:020000040800F2
:100000000845002085010008FD1E0008E1190008D0
:10001000F91E0008CD0200089555000800000000F8
:100020000000000000000000000000004122000865
:100030000B1000080000000009200008F927000844
:100040009F0100089F0100089F0100089F01000810
:100050009F0100089F0100089F0100089F01000800
:100060009F0100089F0100089F0100089F010008F0
:100070009F0100089F0100089F0100089F010008E0
:100080009F0100089F0100089F0100089F010008D0
:10009000D10200089F010008ED0200089F0100083E
:1000A0009F0100089F0100089F0100089F010008B0
:1000B0009F0100081D2900089F0100089F010008FA
:1000C0009F0100089F0100089F0100089F01000890
:1000D0009F0100089F0100089F0100089F01000880
:1000E0009F0100089F0100089F0100080000000018
:1000F0000000000000000000000000000000000000
:1001000000000000000000009F0100089F0100089F
:100110009F0100089F0100089F0100089F0100083F
:100120009F0100089F0100089F0100089F0100082F
:100130009F0100089F0100089F0100089F0100081F
:100140009F0100088D040008C10400089F010008F9
:10015000DFF80CD000F068F800480047A558000808
:1001600008450020EFF30980704780F30988704745
:10017000EFF30880704780F30888704740BA7047F3
:10018000C0BA70470648804706480047FEE7FEE7CA
:10019000FEE7FEE7FEE7FEE7FEE7FEE7FEE7FEE737
:1001A000B12800085101000810B5431A934209D242
:1001B0008318881803E010F8011D03F8011D521E72
:1001C000F9D210BD40EA01039B0703D009E008C93A
:1001D000121F08C0042AFAD203E011F8013B00F80C
:1001E000013B521EF9D210BDD2B201E000F8012B42
:1001F000491EFBD270470022F6E710B513460A46A7
:1002000004461946FFF7F0FF204610BD30B50446FE
:100210000020034600E05B1C934203D2E05CCD5C0F
:10022000401BF8D030BD0000064C074D06E0E068EA
:1002300040F0010394E8070098471034AC42F6D32D
:10024000FFF78AFFB0600008D060000870B58C1816
:1002500010F8015B15F0070301D110F8013B2A11DA
:1002600006D110F8012B03E010F8016B01F8016BC7
:100270005B1EF9D12B0705D40023521E0DD401F8C3
:10028000013BFAE710F8013BCB1A921C03E013F88C
:10029000015B01F8015B521EF9D5A142D8D30020C1
:1002A00070BD10B501214FF0C05001F0D3FE012008
:1002B00001F078FE10BD000010B54FF40061024857
:1002C000FFF799FF10BD000000F8002000BFFEE717
:1002D00000B585B0002005F029FA6A4600210248E1
:1002E00000F095FB05B000BD0064004010B54FF470
:1002F0000071154800F068FA01280DD11349124821
:1003000000F026FA012802D1002005F0CBF94FF4C5
:1003100000710D4800F028F94FF480610A4800F0A0
:1003200053FA01280ED10949891C074800F010FA38
:10033000012802D1002005F0C9F94FF4806102487C
:1003400000F012F910BD0000006400400200F0103F
:1003500000B589B00121092001F09CFE0121480669
:1003600001F078FE0121880601F074FE4FF4005080
:10037000ADF8200003208DF8220018208DF823000E
:1003800008A9404800F073FF4FF48050ADF82000FA
:1003900048208DF8230008A93A4800F068FF0020A3
:1003A0008DF81A0001208DF81B0000208DF81C002C
:1003B0008DF81D008DF81E008DF81F008DF81600B9
:1003C00001208DF8170008208DF8180001208DF805
:1003D00019000620ADF8140005A92B4800F08DFA8D
:1003E0000E208DF80E0000208DF80F0001208DF8F2
:1003F00010000020ADF80400ADF80600ADF80800CC
:10040000ADF80A000120ADF80C008DF8110001A82C
:1004100000F01AF9012210211B4800F065FA412072
:100420008DF8000001208DF8010000208DF80200F9
:1004300001208DF80300684601F068FD012005F0F9
:1004400069F901225102104800F04EFA012291028E
:100450000D4800F049FA0122D1030B4800F044FA9C
:1004600042208DF8000001208DF8010000208DF859
:10047000020001208DF80300684601F047FD0020CE
:1004800009B000BD000C01400068004010B586B006
:100490000024012005F04AF901AA0121074800F0D3
:1004A000B6FA0598009001A80FC804F04BFF14217C
:1004B00001A8FFF7A0FE06B010BD000000680040D4
:1004C00010B54FF40071184800F07EF9012810D1E2
:1004D0001649154800F03CF9012805D105F0E2F86D
:1004E0001249114800F024F84FF400710E4800F052
:1004F0003BF84FF480610C4800F066F9012812D1F6
:100500000A49891C084800F023F9012806D105F0A2
:10051000DDF80649891C044800F00AF84FF48061B0
:10052000014800F021F810BD006800400200F01002
:1005300000220C4B994202D10023836111E0C1F3E8
:10054000130201F000730BB1C2600AE001F0806396
:100550000BB1026105E001F000630BB1826000E0C5
:10056000426070477000F030B1F5007F3AD00FDC88
:10057000202928D006DC01291CD004291DD00829F7
:1005800040D11DE0402921D0B1F5807F3AD126E04D
:10059000B1F5004F31D006DCB1F5806F25D0B1F553
:1005A000006F2FD124E0B1F5803F12D0B1F5003FAC
:1005B00028D111E0154A826025E00822C26022E0BD
:1005C0001022C2601FE0082202611CE010220261BA
:1005D00019E00822426016E01022426013E0042273
:1005E000426010E0042242600DE0042242600AE012
:1005F000002282610422426005E00022826104221E
:10060000426000E000BF00BF704700000101010030
:1006100010B504460B48844209D10121480601F077
:1006200029FD00214FF0007001F024FD08E00121B8
:10063000880601F01FFD00214FF0806001F01AFDD7
:1006400010BD00000064004010B50021837A012233
:1006500002FA03F13D4A126842F001023B4B1A6074
:100660003A4A1C3212688A43384B1C331A60027BA8
:10067000CAB9364A0C3212688A43344B0C331A60BA
:100680004288C38842EA0343304A4032847A42F8BF
:1006900034300288838842EA03432C4A4032847A09
:1006A00002EBC4025360027B012A19D1274A0C32A3
:1006B00012680A43254B0C331A604288038842EAC9
:1006C0000343224A4032847A42F83430C288838815
:1006D00042EA03431D4A4032847A02EBC40253606B
:1006E000C27A3AB9194A121D12688A43174B1B1D68
:1006F0001A6006E0154A121D12680A43134B1B1DAF
:100700001A60028932B9114A143212688A430F4BB7
:1007100014331A600289012A06D10C4A1432126875
:100720000A430A4B14331A60427B012A06D1074A56
:100730001C3212680A43054B1C331A60034A1268C4
:1007400022F00102014B1A6010BD0000006600405B
:1007500010B50246002001F4700343B19369C1F360
:10076000130423400BB101202DE000202BE001F009
:10077000807343B15368C1F3130423400BB10120CC
:1007800021E000201FE001F0006343B19368C1F352
:10079000130423400BB1012015E0002013E001F009
:1007A000007343B1D368C1F3130423400BB101209C
:1007B00009E0002007E01369C1F3130423400BB1E3
:1007C000012000E0002010BD70B504460D46002653
:1007D00060692840002871D0B5F5807F5CD010DCBE
:1007E000082D35D006DC012D20D0022D24D0042D7B
:1007F00072D127E0102D31D0202D35D0402D6BD176
:1008000038E0B5F5004F60D009DCB5F5007F49D080
:10081000B5F5806F4CD0B5F5006F5DD14FE0B5F503
:10082000803F2DD0B5F5003F56D12FE0A0682D496F
:1008300000F022FB064651E0E068032100F01CFBBB
:1008400006464BE0E068082100F016FB064645E04E
:10085000E068102100F010FB06463FE0206903210C
:1008600000F00AFB064639E02069082100F004FB8D
:10087000064633E02069102100F0FEFA06462DE01E
:100880006068082100F0F8FA064627E06068102149
:1008900000F0F2FA064621E0A069012100F0ECFA2E
:1008A00006461BE0A069022100F0E6FA064615E0C4
:1008B000A069042100F0E0FA06460FE00FE0A0690D
:1008C000702100F0D9FA064608E06068042100F0C3
:1008D000D3FA064602E0FFE7002600BF00E000264C
:1008E000304670BD010101001AB143690B434361F9
:1008F00002E043698B434361704730B502460020F4
:100900000023146824F002041460146844F0010405
:10091000146000E05B1C546804F001041CB94FF63D
:10092000FF74A342F6D1546804F001040CB900200E
:100930006CE08C79012C04D1146844F080041460BC
:1009400003E0146824F080041460CC79012C04D1F5
:10095000146844F04004146003E0146824F0400478
:1009600014600C7A012C04D1146844F02004146043
:1009700003E0146824F0200414604C7A012C04D1A4
:10098000146844F01004146003E0146824F01004A8
:1009900014608C7A012C04D1146844F008041460AB
:1009A00003E0146824F008041460CC7A012C04D10C
:1009B000146844F00404146003E0146824F0040490
:1009C00014608C78A407CD7844EA05640D7944EA74
:1009D00005444D7944EA05540D886D1E2C43D461BD
:1009E000146824F001041460002300E05B1C5468C8
:1009F00004F001041CB14FF6FF74A342F6D1546811
:100A000004F001040CB1002000E0012030BD10B55D
:100A100000F5D87303EB01131B6803F00403137292
:100A2000137A53B900F5D87303EB01131B6840F236
:100A3000FF7404EA5353136009E000F5D87303EB25
:100A400001131B686FF0604404EAD303536000F5A0
:100A5000D87303EB01131B6803F00203537200F514
:100A6000D87303EB01135B6803F00F03937200F577
:100A7000D87303EB01135B681B0AD37400F5D873BA
:100A800003EB01139B68D37200F5D87303EB0113DA
:100A90009B681C0A147300F5D87303EB01139B6861
:100AA0001C0C547300F5D87303EB01139B681B0EE9
:100AB000937300F5D87303EB0113DB68D37300F570
:100AC000D87303EB0113DB681C0A147400F5D873A8
:100AD00003EB0113DB681C0C547400F5D87303EBB3
:100AE0000113DB681B0E937421B9C36843F0200324
:100AF000C36003E0036943F02003036110BD10B538
:100B000002460020936803F08063B3F1806F00D148
:100B100010E0936803F00063B3F1006F01D101208E
:100B200008E0936803F08053B3F1805F01D10220A5
:100B300000E00420042874D002F5C07303EB001316
:100B40001B6803F0010402F5C07303EB00131C6083
:100B50000B7A7BB94B7A0C8843EA445302F5C07494
:100B600004EB00142468234302F5C07404EB001462
:100B7000236010E00B7A4C6843EAC4034C7A2343A9
:100B800002F5C07404EB00142468234302F5C0741A
:100B900004EB001423608B7A03F00F038B7202F5D1
:100BA000C07303EB00135B6823F00F0402F5C073FE
:100BB00003EB00135C6002F5C07303EB00135B688A
:100BC0008C7A234302F5C07404EB001463608B7BC2
:100BD0001C064B7B44EA03440B7B44EA0323CC7A98
:100BE000234302F5C07404EB0014A3608B7C1C0645
:100BF0004B7C44EA03440B7C44EA0323CC7B234331
:100C000002F5C07404EB0014E36002F5C07303EB5B
:100C100000131B6843F0010402F5C07303EB0013DB
:100C20001C6010BD10B50246002321B1012907D078
:100C300002290FD109E090681D4C00EA04030BE083
:100C400090681C4C00EA040306E090681A4C00EA25
:100C5000040301E0002300BF00BF184C181BA3428F
:100C600016D007DC83B16FF08060184470B10228A1
:100C700018D111E0B0F5007F10D0114C204448B1DC
:100C8000B0F5003F0ED10BE002230DE000230BE096
:100C9000002309E0002307E0012305E0012303E02E
:100CA000012301E0002300BF00BFD8B210BD000047
:100CB0000300000400030008000003100001000806
:100CC0000001FFF7F0B504460D462946204600F026
:100CD00025F80746615D681C205C41EA002686EA2B
:100CE0000700F0BD0168C943016070474FF0FF3154
:100CF0000160704730B50B4600210AE004785D5C66
:100D00006C40054D55F82440056884EA15240460BC
:100D1000491C9142F2D330BDF85B000870B5024621
:100D20004FF6FF7048F2050517E0491E12F8014B17
:100D300080EA042000230EE000F400462EB14FF6B6
:100D4000FF7606EA4000684003E04FF6FF7606EAC9
:100D500040005E1CF3B2082BEEDB0029E5D170BD2C
:100D60000FB430B585B00024142208A96846FFF7F7
:100D70001BFA012004F0EEFC20B9012005B030BCC4
:100D80005DF814FB69460E48FFF7B9FE05460024DE
:100D900001E0601C84B2012004F0DCFC40B1294673
:100DA0000748FFF73FFF18B940F6FF708442F0DBB9
:100DB00040F6FF70844201DB0120DFE70020DDE721
:100DC00000680040002001207047000010B51C485A
:100DD0000088401C80B21A49088064281DDB00206E
:100DE000088018480078184991F82810884214D0D3
:100DF000154890F828001349087008211148FFF79A
:100E00008DFF84B20F490C7221120E4841720023EB
:100E10000A2201460D4800F061F90B48407801288C
:100E20000CD109488078012808D100200649487073
:100E3000887000F0D1FD01200349487110BD000009
:100E40007C0000207A3A0020243A0020843A0020D6
:100E500010B500240748006850B106480068806853
:100E600030B10449096888688047012800D001240E
:100E7000204610BD640000200246002002EA010363
:100E80000BB1012000E00020704700000020034962
:100E90000978C1F3800101B10120704720070020CB
:100EA000002003490978C1F3400101B101207047D6
:100EB0002007002010B5034600202AB18B4201D044
:100EC000012006E0002004E08B4201D1012000E077
:100ED000002010BD01460020084AD2898A420BD06A
:100EE000064AD28A8A4207D0044A128B8A4203D029
:100EF000024A528B8A4200D10120704732600008BA
:100F000001460020012901D0032900D101207047AA
:100F10000146002001F0800202B90120704702461C
:100F200000208A4200D10120704700200120704734
:100F3000002002490880091D08807047B06C0040FD
:100F40002DE9FC4701A9284800F0B0F8DFF89C9093
:100F5000002420E0264931F8140000F039FB054652
:100F6000FF2D16D0234830F8150000EB0908224861
:100F700030F81460214830F81400019947183146C0
:100F80003846FFF79FFE20B9324639464046FFF704
:100F90000BF9601CC4B2092CDCDB694612480A3824
:100FA00000F084F808210098FFF78CFE98B90098AB
:100FB00000781349087008460078124981F8280023
:100FC000084690F8280003280CDB0A2081F8290045
:100FD0000120C87006E000200A4981F82900C87085
:100FE00081F82800BDE8FC878E3A00202406002006
:100FF00090600008F85F00087E6000086C600008E0
:101000007A3A0020243A00207047704710B5044611
:1010100006E0142004F0C0FA00F0DAFD601E84B28D
:10102000002CF6DC10BD00002DE9F84F83464FF090
:10103000000A00200090584600F0DEFA8046B8F121
:10104000FF0F27D0584600F0C3FA0546FF2D21D0E8
:101050001148445DDFF84490114830F8150000EB6A
:10106000090621463046FFF759FE87B23755641C02
:1010700038123055641C0B4830F818100A4801EB40
:10108000000ABAF1000F05D000232246314650462F
:1010900000F024F8BDE8F88F1E6000082406002048
:1010A000F85F00086C6000088E3A002002460A488B
:1010B000904201D108600DE007487F38904201D18D
:1010C000086007E004488938904201D1086001E0D7
:1010D000002070470120FCE70D3B00202DE9F04186
:1010E00004460D4616461F463B46324629462046D4
:1010F00004F06CFC0120BDE8F081000070B50446EE
:101100000D4600260848006858B107480068006886
:1011100038B105480068294602682046904700B962
:101120000126304670BD00006400002030B5044642
:1011300004250F4800F088F80546042D16D10D4807
:10114000006940F002000B490861084644610069EB
:1011500040F040000861064800F076F80546054872
:10116000006941F6FD71084002490861284630BD1A
:10117000FFFF0F000020024004200B49C96801F066
:10118000010109B101200EE00749C96801F004011D
:1011900009B1022007E00449C96801F0100109B152
:1011A000032000E00420704700200240034800694B
:1011B00040F08000014908617047000000200240B3
:1011C00078B506460C460425002000904FF6FF70C7
:1011D00000F03AF80546042D26D11448006940F085
:1011E00001001249086134804FF6FF7000F02CF8BE
:1011F0000546042D11D1B01C0090200C00990880E8
:101200004FF6FF7000F020F805460848006941F6E7
:10121000FE7108400549086106E00448006941F68E
:10122000FE71084001490861284678BD002002404F
:1012300002480349486003484860704723016745F6
:1012400000200240AB89EFCD00B502460423FFF732
:1012500093FF034603E0FFF78FFF0346521E012B67
:1012600001D1002AF7D102B90523184600BD2DE9A6
:10127000F04102460025002600200023002400271C
:1012800091F803C00CF00F0591F803C00CF0100C9E
:10129000BCF1000F03D091F802C04CEA050591F8AB
:1012A00000C0BCF1000F31D0146800202BE04FF0DB
:1012B000010C0CFA00F3B1F800C00CEA03069E42E0
:1012C00020D183004FF00F0C0CFA03F7BC4305FA52
:1012D00003FC4CEA040491F803C0BCF1280F06D1CA
:1012E0004FF0010C0CFA00FCC2F814C00AE091F8AF
:1012F00003C0BCF1480F05D14FF0010C0CFA00FC03
:10130000C2F810C0401C0828D1D31460B1F800C046
:10131000BCF1FF0F34DD546800202EE000F1080C12
:101320004FF0010808FA0CF3B1F800C00CEA03060C
:101330009E4221D183004FF00F0C0CFA03F7BC43FF
:1013400005FA03FC4CEA040491F803C0BCF1280F31
:1013500005D100F1080C08FA0CF8C2F8148091F8D5
:1013600003C0BCF1480F07D100F1080C4FF0010891
:1013700008FA0CF8C2F81080401C0828CED354603C
:10138000BDE8F081F0B50A460023002400210025C5
:1013900000F00046B6F1004F02D11D4EF16901E0A8
:1013A0001B4E7168C0F3034583B200F44016B6F5D6
:1013B000401F08D121F07061154E766826F07066E6
:1013C000134F7E6012E000F48016B6F5801F06D140
:1013D000032606FA05F4A14341F0706106E0460DCC
:1013E000360103FA06F6B14341F0706122B1460DB1
:1013F000360103FA06F6314300F00046B6F1004F1D
:1014000002D1034EF16101E0014E7160F0BD0000B8
:101410000000014041617047016170473CB50446DE
:101420000B4600210020019035A000680090012C9F
:1014300032D100BF07E0585C1DF80150684001AD93
:101440006854481CC1B20429F5DB9DF8050000F082
:10145000F0009DF8045005F00F0540EA05101070EB
:101460009DF805000007000E9DF8065040EA151093
:1014700050709DF8060000F0F0009DF8075040EA1B
:10148000151090709DF8070000F00F059DF80400FE
:1014900065F31F10D07030E0002107E0585C1DF8A4
:1014A0000150684001AD6854481CC1B20429F5DB05
:1014B0009DF8040000F00F059DF8050065F31F106E
:1014C00010709DF8050000099DF8065005F00F0505
:1014D00040EA051050709DF8070000F0F0009DF8FC
:1014E000065040EA151090709DF8070000F00F00BC
:1014F0009DF8045040EA1510D07000203CBD00005B
:101500009023B02170B5054603F0F4FE4443601CFF
:1015100010B9AA20444303E014B903F0EBFE0444DD
:101520002C70200C6870200AA870EC70002070BD30
:101530002DE9F047064600240027204890F82C00AB
:101540001E4991F82B1000EB012087B26222214640
:10155000641C72543A0A2146641C72542146641C6D
:101560007754DFF85C90002507E0164830F8150046
:10157000B84200D103E0681CC5B2132DF5DB00BFF3
:10158000132D01D1022404E03846FFF7A3FC00B973
:101590000224022C0ED00C4810F805800B4A32F8B9
:1015A000152002EB090130194246FEF7FDFD04EB60
:1015B000080084B22046BDE8F0870000243A0020ED
:1015C00024060020326000081E600008F85F000852
:1015D0000246FF20002108E0064B33F81130934209
:1015E00001D1084603E04B1CD9B21329F4D300BF44
:1015F00070470000326000080246FF20002108E02A
:10160000064B33F81130934201D1084603E04B1CDE
:10161000D9B20929F4D300BF7047000090600008D8
:101620000448007820B1002002490870012070476A
:101630000020FCE7580000200648006806490860C2
:101640000448001F00684860024808380068886045
:1016500070470000F0F7FF1F540100206848008821
:10166000401C80B2664908800A287CDB0020088084
:101670006448B0F84000B0F5FA7F34DA6148B0F859
:101680004000401C5F49A1F840000846B0F8400007
:10169000B0F5FA7F27D1002008720846407F032862
:1016A00003D00846407F02281DD100205549087705
:1016B00001204877002081F8220088714874A1F841
:1016C000400081F8240081F8250081F82700C873C4
:1016D0004D488079012803D100204B494862887128
:1016E000012048490870474890F8240058B14748FD
:1016F000007820F00100454908700846007820F085
:10170000020008700CE04148007820F00100401C05
:101710003E4908700846007820F00200801C0870DE
:10172000384890F8250058B13848007820F0040077
:10173000364908700846007820F0080008700CE070
:101740003248007820F00400001D30490870084637
:10175000007820F00800083008702A48B0F85400DB
:1017600070B1284800E048E0B0F85400401E254918
:10177000A1F854000846B0F8540008B90020C87316
:1017800023480088401C80B221490880642800DA80
:10179000704700201E4908801A4890F82900D8B1E7
:1017A000184890F82900401E164981F8290008467B
:1017B00090F8290080B90846C07801280CD1002093
:1017C000C870084690F82800002805DD084690F803
:1017D0002800401E81F828000A48007A30B10B48E2
:1017E000007820F010000949087006E007480078EA
:1017F00020F0100010300549087000BFC8E7000055
:101800001A010020243A0020E4310020700000205A
:10181000180100207047704770B505460E4608480D
:101820000670002404E0285D06490855601CC4B217
:10183000034800788442F6DB01F030F970BD000007
:10184000250100201C0100200146002004E0054A7B
:10185000125C0A54421CD0B2034A12789042F6DB62
:10186000704700001C0100202501002070B50446CF
:101870000D4601F01FFA064632462946204603F07F
:1018800085FC70BD70B505460E46084806700024FC
:1018900004E0285D06490855601CC4B2034800787E
:1018A0008442F6DB01F07EF970BD000025010020C6
:1018B0001C01002010B501F08FFA10BD10B50446D0
:1018C00003F0F8FC00200149087010BD240100203D
:1018D0000148007870470000250100207FB50546CB
:1018E0000E48006800900E4800788DF8040000242F
:1018F00005E0295D0DF105000155601CC4B20848E2
:1019000000788442F5DB01208DF80D000549487010
:101910009DE80F0002F02CFB7FBD00002801002095
:1019200026010020243A0020014908707047000079
:101930002601002020B940F2B471044A116003E08E
:1019400040F2B471014A1160704700002801002084
:10195000704700002DE9F04105460E4601F0AAF956
:1019600004460A48007878B97F2020706570A67018
:1019700003270020FFF7DEFF01F096FD384601F057
:10198000F9F9012001490870BDE8F0812401002027
:101990002DE9F04105460E4601F08CF980460D48D0
:1019A0000078A8B9A5B1002404E0305D08F804006F
:1019B000601C84B2AC42F8DB2F460020FFF7BAFF70
:1019C00001F072FD384601F0D5F901200149087097
:1019D000BDE8F0812401002010B501F001F810BD30
:1019E00000BFFEE710B54FF400600B49086003F03C
:1019F00052FF4FF480600849091F086003F04BFF55
:101A00004FF480600449086003F045FF4FF4006024
:101A10000149091F086010BD140C014010B54FF4B6
:101A200000600949086003F036FF4FF48060064902
:101A3000086003F030FF4FF480600349091D08601F
:101A400003F029FF10BD0000100C014070B50546E1
:101A50000024002618E06006040E4FF480600F4951
:101A6000086003F018FF0D480838006800F40060B3
:101A700008B1601CC4B24FF480600849091D0860B9
:101A800003F009FF701CC6B2082EE4DB15B9FFF79E
:101A9000C5FF01E0FFF7A6FF204670BD100C014016
:101AA00070B50446002524E004F0800020B14FF416
:101AB00000601149086004E04FF400600E49091D00
:101AC000086003F0E8FE4FF480600B49086003F003
:101AD000E2FE4FF480600849091D0860072D02D11D
:101AE0004000091F08606006040E03F0D4FE681C65
:101AF000C5B2082DD8DB70BD100C014010B54FF4F5
:101B000000600A4908604010086003F0C4FE4FF40A
:101B100000600649091D086003F0BDFE4FF48060B7
:101B20000249091D086003F0B6FE10BD100C01400B
:101B300010B54FF40060074908604010091F0860A5
:101B400003F0A9FE4FF400600249091F086003F08A
:101B5000A2FE10BD140C014010B54FF400600E49F8
:101B6000086003F098FE4FF480600B49086003F0B2
:101B700092FE09480838006800F4006008B10124AA
:101B800000E000244FF480600349091D086003F061
:101B900082FE204610BD0000100C014070B50546C5
:101BA0000C4645F2555000F033F8284600F024F872
:101BB000204600F027F800F017F800F001F870BD9B
:101BC0004CF6CC40014908607047000000300040EE
:101BD00010B500F009F810BD10B540F635410420ED
:101BE000FFF7DCFF10BD00004AF6AA20014908609B
:101BF0007047000000300040014948607047000015
:101C0000003000400149886070470000003000400B
:101C10000149086070470000003000402DE9F0479E
:101C20002D4804682D48844201D0BDE8F0872A4839
:101C3000001D0468B4F5205F02D3B4F5D03F00D98D
:101C4000F3E7A60804F0030000B1761CDFF89080EB
:101C5000244DFFF7EDFA002724E04FF0000AD8F8F2
:101C60000040C5F30A0010B92846FFF75FFA0EE0FE
:101C700021462846FFF7A4FA042800D108E00AF11B
:101C8000010000F0FF0ABAF1030F00DB00E0EFE70C
:101C900000BFD5F800904C4500D005E008F10408DD
:101CA0002D1D7F1CB742D8D300BF0B48FFF73EFA6B
:101CB000FFF77CFA0B4840680B490860084600684B
:101CC0000A49086007490868FEF755FA074800689E
:101CD000804700BFA9E700000058020844332211E2
:101CE0000060020800800008180000201400002096
:101CF0000020054A1188121F128842EA0141034A56
:101D0000914200D101207047B46C00405CBA55AAE2
:101D100010B5FEF7D1FA72B6FFF780FFFFF7E8FFC4
:101D200028B101200F490870FFF702F917E00E48AB
:101D300000680E490840B0F1005F10D100F07EFC51
:101D4000094840680A49086008460068094908606F
:101D500005490868FEF70FFA06480068804762B632
:101D600010BD000058000020008000080000FE2F79
:101D7000600000205C00002008B501211C2000F05C
:101D800089F94FF40070ADF8000010208DF80300C1
:101D900003208DF8020069465348FFF768FA4FF4B4
:101DA00000715148FFF738FB0120ADF8000010200A
:101DB0008DF8030003208DF8020069464A48FFF7BA
:101DC00056FA01214848FFF727FB40F20240ADF8E0
:101DD000000010208DF8030003208DF802006946F2
:101DE0004148FFF744FA02213F48FFF715FB4FF443
:101DF00080613D48FFF70EFBA020ADF800001020E9
:101E00008DF8030003208DF8020069463748FFF77C
:101E10002EFA20213548FFF7FDFA80213348FFF7DD
:101E2000FBFA44F22720ADF8000010208DF80300E3
:101E300003208DF8020069462D48FFF718FA4FF489
:101E400000712B48FFF7E8FA01212948FFF7E2FA71
:101E500002212748FFF7DEFA04212548FFF7DAFAC6
:101E60004FF480412248FFF7D5FA20212048FFF7A0
:101E7000D1FA4FF48070ADF8000048208DF80300CF
:101E800069461948FFF7F3F94FF40070ADF8000008
:101E900048208DF8030069461448FFF7E8F901214E
:101EA000084600F0F7F801211248FFF76BFA1020FE
:101EB000ADF8000001208DF8020010208DF803001D
:101EC00069460B48FFF7D3F910210948FFF7A4FA38
:101ED0004FF40050ADF8000004208DF8030069466F
:101EE0000248FFF7C4F908BD000801400010014096
:101EF000000C01400001300000BFFEE7704710B544
:101F00004FF4A06000F03AF810BD000070B5002159
:101F100000230F22C47804B3154C246804F4E06451
:101F2000C4F5E064210AC1F10403CA40447804FA0C
:101F300003F184781440214309010E4C0678A15521
:101F4000047804F01F050124AC4005786D11AD0044
:101F500005F1E025C5F8004109E0047804F01F050B
:101F60000124AC40044D0678761145F8264070BD3A
:101F70000CED00E000E400E080E100E002490143F4
:101F8000024A1160704700000000FA050CED00E005
:101F900010B54FF400720021014803F096F910BD0E
:101FA000843A0020014908627047000000000E4298
:101FB0001FB50120134908720020A1F840000098C5
:101FC000A0F2347010B1AB2818D10BE040F234709D
:101FD0000C49A1F84E009DF804100DF10500FFF723
:101FE00051FC0CE040F2DF700649A1F84E009DF86C
:101FF00004100DF10500FFF70FFC00E000BF00BF6B
:102000001FBD0000243A0020704700002DE9F04178
:1020100004460D46164600270948006860B1084886
:102020000068406840B10648006832462946436867
:102030002046984700B901273846BDE8F0810000E6
:1020400064000020014802490860704700F8002041
:102050006400002029B1064AD2690243044BDA61C8
:1020600004E0034AD2698243014BDA617047000001
:102070000010024029B1064A12690243044B1A615A
:1020800004E0034A12698243014B1A617047000061
:102090000010024029B1064A92690243044B9A613A
:1020A00004E0034A92698243014B9A617047000041
:1020B000001002402DE9F0410021002200250023FC
:1020C0000026002400278C46DFF86081D8F80480C1
:1020D00008F00C0121B1042907D0082959D109E0E1
:1020E000DFF84C81C0F8008058E0DFF84481C0F888
:1020F000008053E0DFF83481D8F8048008F47012CF
:10210000DFF82881D8F8048008F48035920C0D2A75
:1021100001D0921C00E0062235B9DFF8188102FBDD
:1021200008F8C0F8008033E0DFF80081D8F82C8090
:1021300008F48036DFF8F480D8F82C8008F00F0817
:1021400008F1010446B9DFF8E880B8FBF4F808FBB1
:1021500002F8C0F800801BE0DFF8D080D8F82C80AF
:10216000C8F3031808F10107DFF8C080D8F82C8005
:10217000C8F3032808F1020CDFF8B480B8FBF7F8C5
:1021800008FB0CF8B8FBF4F808FB02F8C0F8008074
:1021900004E0DFF89C80C0F8008000BF00BFDFF8DB
:1021A0008C80D8F8048008F0F0010909DFF88880F5
:1021B00018F80130D0F8008028FA03F8C0F804803D
:1021C000DFF86880D8F8048008F4E061090ADFF8D5
:1021D000688018F80130D0F8048028FA03F8C0F8B5
:1021E0000880DFF84880D8F8048008F46051C90AF4
:1021F000DFF8448018F80130D0F8048028FA03F89A
:10220000C0F80C80DFF82480D8F8048008F440413E
:10221000890BDFF8288018F80130D0F80C80B8FB63
:10222000F3F8C0F81080BDE8F08100000010024013
:1022300000127A0000093D004300002053000020F6
:10224000704700002DE9F04104460D4600260027A6
:102250006078217800EB012087B20F48C08AB8422D
:1022600011D10E48C07AA8420BD10D4890F8220037
:1022700028B12A46A11C0B48FDF796FF04E033263F
:1022800002E0132600E0312616B93846FEF7CCFEF0
:102290003046BDE8F0810000326000081E60000892
:1022A000243A0020F80600202DE9F04F8DB00446B6
:1022B000174698464FF00009CA4600250026AB464F
:1022C0008348B0F84200042803DA13200DB0BDE8BB
:1022D000F08F94F800A0A078617840EA012571227F
:1022E0003046711C8EB20DF8002022783046711CE9
:1022F0008EB20DF8002062783046711C8EB20DF857
:102300000020A2783046711C8EB20DF80020BAF180
:10231000010F7DD1A078617840EA01256C49B1F8C0
:1023200042000421FEF7FBFD18B140F20320854274
:1023300020D06749B1F842000421FEF7F0FD18B142
:1023400040F20220854215D06149B1F842000C21CB
:10235000FEF7E5FD10B1B5F57F4F0BD05C49B1F844
:1023600042000421FEF7DBFD002879D04FF6017012
:10237000854275D1564890F8220000287BD0FEF7A0
:10238000D4FD002874D0A5F20220B8B1012806D0EF
:10239000A0F57C40FE3810B3012867D152E001203F
:1023A0004B49C8734FF4FA70A1F854004FF0000B7A
:1023B0003046711C8EB20DF800B058E0454890F8D8
:1023C0003C08032808D14348007A012804D1414938
:1023D000C8704FF0780901E04FF0220947E03D480E
:1023E000C07B01282BD1E0780006217900EB014069
:1023F000617900EB0120A179084436498861E079D0
:102400000006217A00EB0140617A00EB012000E038
:1024100048E0A17A08442F49C8614FF0780908467E
:1024200080692D49884205D04FF0310901202949A2
:10243000887306E0012027490870887201E04FF098
:10244000220914E0234890F83C0803280BD12148C6
:10245000007A40B901201F4948714FF0780904E023
:102460000CE008E004E04FF0220900E000BF22E0A9
:102470004FF022091FE04FF033091CE040F2032027
:10248000854209D0401E854206D0B5F57F4F03D066
:102490004FF60170854202D14FF013090BE04FF067
:1024A000310908E00A480079012804D100200849D0
:1024B00008714FF01209A8F80060B9F1000F04D1BB
:1024C000324669463846FDF76FFE4846FEE6000094
:1024D000243A0020E4310020008000082DE9F0417A
:1024E00004460E461746984600252078294981F86B
:1024F00035080846D0F838182748B0F84200801E42
:1025000008442449C1F83808FEF7C0FC08B19225F8
:102510003DE0FEF7C5FC08B1932538E01E48B0F851
:10252000420040F60201884201DD13252FE01948E0
:1025300090F83C08012806D0164890F83C0802287C
:1025400001D0242523E0134890F83408114991F86C
:102550003518401A012801DD732518E00D48D0F820
:1025600038080E490968884201D971250FE0012019
:1025700008494870022081F83C080748B0F842003A
:10258000821E074903483430FDF70EFE78252846A1
:10259000BDE8F081E4310020243A00203001002021
:1025A000EC0900202DE9F04104460E4617469846F6
:1025B00000251F49487F00220221FEF77BFC78B3EB
:1025C0001B4890F8220001282BD11949B1F842008C
:1025D0000521FEF7A4FC08B3164890F83C08022831
:1025E0001AD11448D0F8380813490968884213D121
:1025F000012010498870032081F83C0820780006EB
:10260000617800EB0140E178A27801EB02210843F8
:1026100008490862782507E0242505E0132503E032
:1026200001E0332500E07F252846BDE8F081000069
:10263000243A0020E43100203001002003480449FE
:102640000880000C091D088070470000EC59000844
:10265000B86C004010B500F001F810BD0CB50020BA
:10266000019000904048006840F480303E49086086
:1026700000BF3D48006800F4003000900198401C05
:102680000190009820B94FF6FF7101988842F0D16F
:102690003548006800F4003010B10120009001E0DE
:1026A00000200090009801285CD13048006840F07C
:1026B00010002E4908600846006820F003000860FA
:1026C0000846006840F00200086027484068264934
:1026D00048600846406848600846406840F48060AA
:1026E00048600846C06A224908401F49C862084637
:1026F000C06A204908431C49C8620846006840F087
:102700008060086000BF1848006800F00060002882
:10271000F9D01548406820F47C10134948600846F9
:10272000406840F4E81048600846006840F0807057
:10273000086000BF0C48006800F000700028F9D065
:102740000948406820F0030007494860084640688F
:1027500040F00200486000BF0348406800F00C00F1
:102760000828F9D10CBD00000010024000200240F2
:1027700000F0FEFF1408010010B50D4890F8E500C8
:102780000B4991F8E41000EB012084B24FF6FF7082
:10279000844201DA601C84B22012054981F8E40009
:1027A000084680F8E5400349488BFEF73DFC10BD24
:1027B000240600203260000810B50D4890F8E100B2
:1027C0000B4991F8E01000EB012084B24FF6FF7046
:1027D000844201DA601C84B22012054981F8E000CD
:1027E000084680F8E1400349088BFEF71DFC10BD48
:1027F00024060020326000080F480068401C0E4983
:1028000008600E480068401C0C4908600A480068CF
:102810004FF47A71B0FBF1F201FB1200012804D1F0
:1028200007480068401C064908600648007810B94F
:102830000120044908707047340000202C0000205B
:10284000380000203000002030B5164800684FF4F2
:102850007A72B0FBF2F1B1F1807F01D301201DE06B
:1028600021F07F40401E4FF0E022506150170F22B0
:10287000002807DA13071D0E0B4B00F00F04241F6E
:102880001D5503E013071C0E084B1C5400BF00200D
:102890004FF0E022906107201061002008B100BFD6
:1028A000FEE730BD0000002018ED00E000E400E08D
:1028B00010B51648006840F0010014490860084649
:1028C00040681349084011494860084600681149AA
:1028D00008400E4908600846006820F4802008601F
:1028E0000846406820F4FE0048600846006820F072
:1028F000A05008604FF47F0088600020C862FFF796
:10290000A9FE4FF000600449086010BD00100240AD
:102910000000FFF0FFFFF6FE08ED00E010B501211A
:10292000084800F016F858B10121064800F00EF8EA
:102930000548006808B9012000E00020024908604D
:1029400010BD00000004004090012342CA430282EF
:10295000704730B50246002000230024158A05EA9E
:102960000103958905EA010413B10CB1012000E0CF
:10297000002030BD10B51248008888B900201149E8
:1029800008701149087011490870114908701149FF
:1029900008700846017810480088FEF767FF0DE0D0
:1029A0000720094908700D480078401C0B49087041
:1029B00008460078102801D10020087010BD0000E2
:1029C0009A000020B6000020A40000208D00002006
:1029D000B2000020AB0000209200002090000020F8
:1029E00010B50120214908700020214908702148B4
:1029F0000078012805D120480078102801D1FEF781
:102A000009FF1C480078012803D11B4800781028D2
:102A100005D01A48007858B11948007840B9962076
:102A200018490880012018490870022017490870C9
:102A300016480078012802D11548007848B10E48A0
:102A4000007830B10B480078042804D11148008880
:102A500008B900F0FDFC10480078012805D10548B0
:102A60000078062801D100F0F3FC10BDAE00002074
:102A7000B3000020A4000020880000208000002077
:102A80007F000020A0000020B50000207E00002074
:102A900081000020860000208D00002070B536489F
:102AA0000078012866D035480079012804D13448DF
:102AB0000078012800D170BDFEF70AFF3149088077
:102AC0003148FEF7C1FE3048007800F0F0002F4991
:102AD000087000202E4908802E4800882749A1F858
:102AE0004200002008712848007800F00F052248B5
:102AF0000078022803D115B901201F490870204829
:102B00000078012801D100F0A3FC2048007820BB08
:102B10001D48007800F00F001E49088001240CE0D9
:102B20001948005D1C491A4A1288885418480088C0
:102B3000401C17490880601CC4B2164800888442B3
:102B4000EEDD00F03DFA48B9092014490870084646
:102B5000017810480088FEF789FE0BE0012010493B
:102B6000087000200D49087008460178094800885F
:102B7000FEF77CFE00BF9EE77E000020243A002086
:102B80008D00002098000020B80000209400002054
:102B90009600002092000020EA090020AB000020EF
:102BA000AD00002010B51F480078012824D0012076
:102BB0001D490870FEF78CFE1C4908801C48FEF772
:102BC00043FE1B48007800F00F04164800780228E6
:102BD00003D114B901201349087016480078012860
:102BE00001D100F035FC0020134908700120134981
:102BF00008701349087114E00F480078401CC0B2F7
:102C00000D49087002280CDB02F01EFA00F064F88F
:102C1000002009490870034908700A4908700A49E8
:102C2000087010BD7E000020AF000020980000203A
:102C3000B80000208D000020C1000020C00000204E
:102C4000243A0020A40000202401002010B51148DF
:102C5000007838B1104840781049087000F0EAFB5D
:102C60000F4908700D4800780E4908700C4800782C
:102C70000D49087000200D49087000F029FC0B4830
:102C8000007818B904200A49087002E003200849B6
:102C9000087010BDB7000020B800002080000020A0
:102CA000810000207F00002082000020840000209E
:102CB000A400002000487047EA09002010B505482C
:102CC0000078012804D100200249087000F050F972
:102CD00010BD0000AF00002000200D4908700D4914
:102CE00008700D4908700D4908700D4908700D49AC
:102CF00008700D4908700D4908700D4908700D499C
:102D000008700D4908700D4908700D49087070472A
:102D1000A40000207E0000208D000020B1000020D3
:102D2000B2000020AE000020AF000020B300002061
:102D3000B4000020B5000020B6000020AA0000204A
:102D4000B000002010B507480078FEF7EDFD0648FA
:102D5000FEF7C4FD4620054908800120044908709B
:102D600010BD00008C000020B80000209C00002056
:102D7000B300002010B504461148048000880728DD
:102D800003DC00200F49087002E010200D49087094
:102D900001200D49087000200C4908800C4800787B
:102DA000012802D100F052FC09E00C20094908700A
:102DB00008460078FEF782FD00200349087010BD28
:102DC00086000020880000207E0000208A0000206D
:102DD000B1000020AB00002010B500F03BFE00F079
:102DE00037FB10BD10B50A48007820B1012805D086
:102DF000022809D105E000F091FA06E000F0AAFAF5
:102E000003E000F0DDFA00E000BF00BF10BD0000ED
:102E10009100002010B52E4840782D49097801F026
:102E20000F0140EA01202B490880084600882A4902
:102E300008802848008840F60201884213DD0D20F2
:102E4000264908700846017822480088FEF70EFDE2
:102E500002202349087000F083FB002020490870FD
:102E60002049087032E01B48008808282EDB00F05B
:102E7000A7F848B90920194908700846017815488B
:102E80000088FEF7F3FC21E0022411E01048005D09
:102E90001549164A128888540F480088401E0E496A
:102EA000088012480088401C10490880601CC4B289
:102EB000072CEBDD01200E49087006480088FEF75C
:102EC000AAFC01200B49087000F04AFB10BD00006D
:102ED000B8000020920000209A000020AB000020E3
:102EE000AA000020A4000020EA090020960000208B
:102EF000900000208D00002010B51848007800F0E8
:102F00000F001749088001240CE01448005D1549A2
:102F1000154A1288885414480088401C12490880B9
:102F2000601CC4B20E4800888442EEDD00F048F810
:102F300048B909200D4908700846017808480088FA
:102F4000FEF794FC08E00020084908700846017864
:102F500003480088FEF78AFC10BD0000B80000207E
:102F600092000020EA09002096000020AB0000201B
:102F700010B50E48007800F0F0000D4908700020F0
:102F80000C4908800C490870094800780B49C8763C
:102F90000748007810B9FFF7AFFF05E00448007854
:102FA000102801D1FFF736FF10BD0000B800002047
:102FB0009400002096000020AD000020243A00205C
:102FC00000202149097831B1102912D0202918D0C8
:102FD000302935D12CE01D49098849B11C490A889E
:102FE0001A490988491C8A4201DA002000E00120C0
:102FF00027E017490988082901DA002000E00120AC
:103000001FE014490988072907DB114909880829A5
:1030100001DA00200BE0012009E00D490A880D4982
:103020000988491C8A4201DA002000E0012008E0FA
:1030300007490988032901DA002000E0012000E0A7
:1030400000BF00BF704700009400002092000020E5
:10305000980000209A0000202C490988072933DABB
:1030600001212B4A1180012016E02A49095C2A4AD5
:103070002A4B1B88D15429490988491C274A1180A9
:1030800027490988491E264A118021490988491C77
:103090001F4A1180411CC8B21C4909888842E4DDDE
:1030A0001F49098819B901211E4A82F821100121FE
:1030B0001D4A117008211D4A117001211C4A11700E
:1030C0000021164A118020E01049098807291CDBDD
:1030D000012011E00F49095C0F4A104B1B88D154A5
:1030E0000E490988491C0D4A11800D490988491E5D
:1030F0000B4A1180411CC8B20728EBDD084909883A
:1031000019B90121074A82F821107047A600002052
:10311000A8000020B8000020EA0900209600002046
:103120009A000020243A002091000020A4000020F2
:10313000B200002010B52D48008838B903202C4972
:1031400008700846007800F0D1F84EE02948007871
:1031500001284AD1002027490870274908702748CC
:10316000007800F0F000264908700846007818B191
:1031700008460078102809D106201D490870084625
:10318000007800F0B3F8FFF7F3FE2EE01C4800785B
:1031900020282AD1FFF714FF38B9092014490870F4
:1031A0000846007800F0A2F81FE01448007800F00C
:1031B0000F0014490978884210D100201249087084
:1031C000FFF710FE96200949088001200A4908707F
:1031D0000D48007848B9FFF7CDFB06E0042004490C
:1031E00008700846007800F081F810BDA2000020A9
:1031F000AB000020AF000020B6000020B800002087
:1032000094000020900000209100002010B52D4A6D
:1032100012882D4B1B889A4220DB2B4A1178012003
:1032200011E02A4A125C2A4B2A4C24881A55294A52
:103230001288521C274B1A80234A1288521E224B96
:103240001A80421CD0B28842EBDD1F4A1288002A45
:1032500036D10122204B83F8212031E0194A12880F
:10326000194B1B889A422BDA01221C4B1A80012031
:1032700016E0164A125C164B164C24881A55154A4D
:103280001288521C134B1A800F4A1288521E0E4B82
:103290001A80124A1288521C104B1A80421CD0B25B
:1032A000084A12889042E4DD02220D4B1A7008226F
:1032B0000C4B1A7001220C4B1A700022054B1A801D
:1032C00010BD0000A60000209A000020B8000020D9
:1032D000EA09002096000020243A0020A8000020DF
:1032E00091000020A4000020B200002010B5044688
:1032F000214606480088FEF7B9FA00200449087004
:10330000044908700449087010BD000092000020B4
:10331000A40000208D000020B200002010B50A4853
:10332000008840F60201081A084908800848008809
:10333000072802DBFFF790FE05E005480088072814
:1033400001DAFFF763FF10BD96000020A600002001
:103350009A0000201248007808BB16E01148124974
:103360000988405C1149124A128888541048008824
:10337000401C0F4908800F480088401E0D490880F6
:1033800009480088401C0849088007480088072829
:10339000E4DD0020084908700720084908707047DC
:1033A000B2000020B8000020A8000020EA09002098
:1033B000960000209A00002091000020A400002028
:1033C0001449097821BB1449087816E01349144AB6
:1033D0001288895C134A144B1B88D15412490988FE
:1033E000491C114A11800C490988491E0A4A11805A
:1033F0000B490988491C0A4A118009490A88411C5D
:103400008A42E3DD0021094A11700721084A117040
:1034100070470000B20000209A000020B800002091
:10342000A8000020EA09002096000020910000205A
:10343000A4000020054A917831B17F2900DD7F2169
:10344000C8B2421CD0B200E001207047B800002092
:1034500010B514480078092821D2DFE800F00508EB
:103460000B0E1114171A1D00FFF728FC18E000F0CE
:1034700069FC15E000F0D4FB12E000F01BF80FE04F
:1034800000F02EFB0CE000F097FC09E000F02CFCB3
:1034900006E0FFF74FFE03E000F096FB00E000BF00
:1034A00000BF10BDA4000020012001490870704732
:1034B000B100002010B500F00BF80348007810B9F7
:1034C00004200249087010BD84000020A4000020E0
:1034D00010B50A48007820B1012805D0022809D18A
:1034E00005E000F0C9F906E000F0ECF903E000F0B7
:1034F0002BFA00E000BF00BF10BD000084000020D8
:1035000012490988C1F3032141F01001104A1170DA
:103510000E4909785170022011E00E490E4A1288B6
:10352000895C0B4A11540C490988491C0A4A1180CC
:1035300006490988491E054A1180411CC8B207285E
:10354000EBDD0821054A117070470000860000205D
:10355000B8000020EA0900208A0000208C0000202A
:1035600010B51748007840F0300016490870002068
:103570004870887014490880032014490870032497
:1035800004E0CC200F490855601CC4B2072CF8DDBC
:1035900008200E4908700020FEF7CCF90B4800788F
:1035A000FEF7C2F90748FEF799F9062008490870A6
:1035B00046200849088001200749087010BD000016
:1035C000AA000020B80000208E0000208C000020FF
:1035D000A40000209E000020B4000020164A1278AB
:1035E000164B1A70012001210EE0154A154B1B885D
:1035F000D25C124B5A54134A1288521C114B1A8037
:10360000421CD0B24A1CD1B20B4A12889142ECDD66
:10361000094A1278521C0C4B1A7007280ADC04E085
:10362000CC22064B1A54421CD0B20728F8DD0822DF
:10363000054B1A707047000086000020B80000207B
:10364000EA0900208A0000208C00002010B51048F4
:10365000007810B9FFF7C2FF05E00D480078102888
:1036600001D1FFF74DFF01200A4908700A48007890
:10367000FEF75AF90948FEF731F9012008490870A8
:1036800046200849088001200749087010BD000045
:1036900088000020830000208C000020B80000205B
:1036A000A40000209C000020B300002010B52A4890
:1036B000008807282BDA012028490880012416E019
:1036C000274828490988405C27490855254800882B
:1036D000401C2449088025480088401E2349088052
:1036E0001E480088401C1D490880601CC4B21A484E
:1036F00000888442E4DD01201D49087000201D4936
:103700000870FEF725F900201649088023E01248CA
:10371000008807281FDB012411E01148114909889E
:10372000405C114908550F480088401C0D4908802D
:103730000E480088401E0D490880601CC4B2072C4A
:10374000EBDD08200C490870FFF7FCFA04200B4958
:10375000087000F065F910BDA6000020A800002048
:10376000EA0900208A000020B8000020860000201E
:1037700084000020B10000208C000020A400002064
:1037800070B5334800883349098888422DDB01250C
:1037900030480678012413E02F4830490988405CFE
:1037A0002F4908552D480088401C2C49088029487D
:1037B0000088401E27490880681CC5B2601CC4B23E
:1037C000B442E9DD2748067004E0CC20244948557E
:1037D000681CC5B2072DF8DD082022490870FFF7E4
:1037E000B1FA04202049087030E0194800881949CE
:1037F000098888422ADA01201C490880012416E041
:10380000154816490988405C154908551348008831
:10381000401C124908800F480088401E0D4908804E
:1038200012480088401C11490880601CC4B2084836
:1038300000888442E4DD02200D49087000200D4913
:103840000870FEF785F800200449088070BD00006C
:10385000A600002086000020EA0900208A0000203F
:10386000B80000208C000020A4000020A800002048
:1038700084000020B100002010B50D48007840F011
:1038800020000C4908700C48008840F60201081A14
:103890000A4908800A480088072802DBFFF706FF6C
:1038A00005E007480088072801DAFFF769FF10BD27
:1038B00083000020B80000208A000020A60000201D
:1038C0008600002010B517480078012828D116E09E
:1038D000154816490988405C1549164A12888854CB
:1038E00012480088401C1149088013480088401E77
:1038F000114908800F480088401C0E4908800D4877
:1039000000880728E4DD08200C490870FFF71AFA40
:1039100000200B49087004200A49087000F080F864
:1039200010BD0000B1000020EA0900208A0000203C
:10393000B8000020A8000020860000208C00002095
:1039400084000020A400002010B520480078012841
:103950003AD11F48047800781E49097808441E4966
:10396000087018E01D481E490988405C1D49184A26
:10397000128888541A480088401C19490880154844
:103980000088401E13490880601CC4B2104800889B
:10399000401C0F4908800E4800880F49097888426A
:1039A000E0DB04E0CC200F490855601CC4B2072CB2
:1039B000F8DD082008490870FFF7C4F900200A491B
:1039C000087004200949087010BD0000B1000020F3
:1039D000A8000020860000208C000020EA090020BA
:1039E0008A000020B800002084000020A4000020ED
:1039F00010B504462046FDF761FF00200449087019
:103A000004490870044908700449087010BD00009A
:103A1000A40000207E000020B1000020AE000020A5
:103A200009480078401C08490870084600781028AA
:103A300001D1002008700548007820B104480078C2
:103A4000401E03490870704783000020800000205A
:103A50007F0000201A480078012808D11948008802
:103A6000002804DD17480088401E164908801648C3
:103A70000078012808D115480088002804DD134883
:103A80000088401E1149088011480078012808D19B
:103A900010480088002804DD0E480088401E0D49AB
:103AA00008800D480078012808D10C4800880028BB
:103AB00004DD0A480088401E08490880704700005D
:103AC000B30000209C000020B40000209E000020D5
:103AD000B5000020A0000020B6000020A2000020B9
:103AE00010B52C48008838B901202B4908700846C9
:103AF0000078FFF77DFF4CE028480078012803D0CC
:103B000027480078012844D100202649087023491D
:103B100008702548008838B900201F4908700846F9
:103B20000078FFF765FF34E02048007848B120486E
:103B3000007830B900201F49087002201E49087023
:103B400027E01E48007818B11C48007801280CD1E5
:103B5000FFF7BEFC1A48007818B900201049087019
:103B600017E001200E49087013E01448007802287D
:103B700003D10320104908700BE010480078022898
:103B800007DD10480078401E0E49087005200A49DC
:103B9000087010BD9C000020AB000020AE0000208B
:103BA000B0000020B300002086000020800000202C
:103BB0007F000020B7000020A4000020810000202A
:103BC000840000208200002010B51148008838B918
:103BD00003201049087008460078FFF787FB15E0BE
:103BE0000D48007801280AD100200B4908700B20ED
:103BF0000849087008460078FFF778FB06E0FFF7F1
:103C0000F1F80648007808B9FEF7B4FE10BD0000D0
:103C1000A2000020AB000020AF0000209100002097
:103C200010B52B48008838B902202A490870084688
:103C30000078FFF7DDFE49E027480078012845D1EC
:103C40000020254908702548007800F0F00024493C
:103C5000087008460078302838D1002021490870C3
:103C60001E48007800F00F04FFF7AAF938B90920C0
:103C70001849087008460078FFF7BAFE26E0032CC2
:103C800007DB05201349087008460078FFF7B0FEEF
:103C90001CE0022C07D108200E4908700846007865
:103CA000FFF7A6FE12E0012C0DD10720094908708C
:103CB00008460078FFF79CFE952005490880012002
:103CC0000849087002E00CB9FEF7C0FF10BD000003
:103CD000A0000020AB000020AF000020B8000020B2
:103CE00094000020B500002010B50F48007801288E
:103CF0000ED100200C4908700C49087007200C49AF
:103D0000087096200B49088001200B49087009E0D3
:103D10000A48008830B9012009490870084600782F
:103D2000FFF7E4FA10BD0000AE000020B400002050
:103D3000A4000020A2000020B60000209E00002069
:103D4000AB00002010B51548008838B9012014498F
:103D5000087008460078FFF74BFE1DE01148007818
:103D6000012819D100200F4908700F4908700F4829
:103D7000007838B900200A49087008460078FFF733
:103D800037FE09E009480078102805D101200849CC
:103D9000087002200749087010BD00009C00002038
:103DA000AB000020AE000020B300002088000020FF
:103DB000B7000020A400002008480078401E0749F2
:103DC000087008460078012806DC032004490870C2
:103DD0000448007801490870704700008200002004
:103DE000A4000020810000200246002321B90D48D4
:103DF00000681060012070470A4803681068984204
:103E000005D81068181A884209D30120F3E7106812
:103E1000C0F1FF301844884201D30120EBE70020B5
:103E2000E9E70000340000204F48007801280AD15B
:103E30004E484089401C4D494881012008700020AF
:103E40004949087000E0704748484089052190FBC7
:103E5000F1F201FB120030B94448408918B1012049
:103E60004249487000E0EEE7404840890A2190FB53
:103E7000F1F201FB120028B93C48408910B1012041
:103E80003A49887039484089142190FBF1F201FBCE
:103E9000120028B93548408910B101203349C87053
:103EA00032484089322190FBF1F201FB120028B91F
:103EB0002E48408910B101202C4908712B484089B7
:103EC000642190FBF1F201FB120028B927484089D8
:103ED00010B1012025494871244840894FF4FA71F6
:103EE00090FBF1F201FB120028B92048408910B183
:103EF00001201E4988711D4840894FF47A7190FB5A
:103F0000F1F201FB120028B91848408910B10120D4
:103F10001649C8711548408940F2DC5190FBF1F216
:103F200001FB120028B91148408910B101200F4946
:103F300008720E4840894FF4FA6190FBF1F201FBE0
:103F4000120028B90948408910B101200749487278
:103F50000648408941F27071884202DB0020034923
:103F6000488100BF6FE7000030000020840100207E
:103F70000FB5184800880A2802DB00201549088080
:103F800014480288001D00EB0210009901609DF8A2
:103F9000041010480288001D00EB021001719DF80A
:103FA0000D100C480288001D00EB021041730948F7
:103FB0000188001D00EB0110DDF8051040F8051F19
:103FC000DDF80910416003480088401C0149088061
:103FD0000FBD0000EC11002010B51748006800B1BB
:103FE00010BDFCF7EFFE00B9FAE71BE0134840886C
:103FF0000A2802DB00201149488010484188001D32
:1040000000EB011494E80F0001F0B3F901200C4912
:104010008870002081F82A0008484088401C074921
:10402000488005E005480088044949888842DDD178
:1040300000BF00BFD4E700006C000020EC1100209E
:10404000243A002010B50948007F70B10748C07FAE
:1040500010280AD10549887F00F01EFC0020034982
:104060000877FF210248FCF7C6F810BD243A00206B
:10407000EA09002010B50748007F50B10548C07F0D
:10408000112806D103482B3000F0ECFC0020014938
:10409000087710BD243A002010B50648007F40B1D3
:1040A0000448C07F222804D100F044FB00200149CD
:1040B000087710BD243A002010B51548007F28B3BA
:1040C0001348C07F272821D1114890F82B000228DF
:1040D00009D0104A0E492B31012000F025FD0020A7
:1040E0000B49087712E00A4890F82B0002280DD1FE
:1040F000084A07492B3100F017FD002004490877D2
:1041000081F82100034800210160416010BD0000DA
:10411000243A0020E000002010B50A48007F78B162
:104120000848C07F2E280BD107480088401E81B266
:10413000064800F037FB0020024981F8210008778B
:1041400010BD0000243A002096000020EB0900205A
:1041500010B50A48007F78B10848C07F31280BD1DC
:10416000032106482B3000F035FE00200349087774
:10417000FF210348FCF73FF810BD0000243A00205F
:10418000EA09002010B50C48007F98B10A48C07FAA
:1041900034280FD109480088401E81B2084800F039
:1041A00053FE002004490877C877FF210448401EC9
:1041B000FCF721F810BD0000243A002096000020F2
:1041C000EB09002010B50C48007FA0B10A48C07F61
:1041D000362810D109480078401EC1B206482B305D
:1041E00000F0D8FE002004490877C87740F60201A5
:1041F0000348FCF700F810BD243A00209600002088
:10420000EA09002010B50948007F70B10748C07F57
:1042100037280AD106480088401E81B2054800F0C0
:10422000E3FE002001490877C87710BD243A00203A
:1042300096000020EB09002010B50748007F50B120
:104240000548C07F3E2806D103482B3000F0EAFA2B
:1042500000200149087710BD243A00208178064AE1
:104260001170C178517011460978491C11701146BE
:104270004978891C51707047E000002010B509484A
:10428000007801280DD1074840780B2806DA054848
:104290004078054951F82040A04702E0002001493C
:1042A000087010BDE8000020EC00002010B50120CF
:1042B0000249087000F0C8FE10BD0000E8000020B0
:1042C00010B500200249087000F0BEFE10BD0000CD
:1042D000E80000202DE9FE4300240126A046002529
:1042E0000027FCA207CA8DE80700FD4800780128D6
:1042F0001DD10020FA4908700846C07988B901200C
:10430000C87108468069F7490860F548C069F649F0
:1043100008600020F5490860F5490880F0490874F4
:10432000D6E10320EE4908740020C871D0E1EC48C2
:10433000C079012867D1EA490874EB48006890B158
:10434000E9480068B0F5006F08D9E7480068A0F5B3
:104350000060E54908604FF4006704E0E248076840
:104360000020E1490860DF490968E04A12688818BE
:104370003946FCF7C3FE0646DC4800683844DB4992
:104380000860DB480088401CD94908804EB10320F2
:10439000D34908740020C87172213120FDF7DAFA80
:1043A00096E1D148006800BB0220CD490874002086
:1043B000C87171222046611CCCB2CE490A54012238
:1043C0002046611CCCB2CB490A54FF222046611C16
:1043D000CCB2C8490A5400222046611CCCB2C5495F
:1043E0000A542046FDF7D4FA72E1C148008814212E
:1043F00090FBF1F201FB1200002891D178213120CD
:10440000FDF7A8FA64E1B648407801287BD176220E
:104410002046611CCCB2B7490A54B14890F8342800
:104420002046611CCCB2B3490A54B348B0F84200EC
:10443000851EAB48406918B9A9482430FCF756FCE2
:10444000A748007A012815D1A5494969AB4A8818BF
:104450002A46A3493431FBF7A7FEA1484069284406
:104460009F4948612A463431A1F11000FCF742FC13
:10447000002642E09A48407A01283ED1984890F8B8
:104480003508974991F83418884213D0944890F829
:104490003508934981F83408084690F8340895495E
:1044A00008558F48D0F83808401B8D49C1F83808A6
:1044B000002622E02A468A493431A1F11000FCF797
:1044C00019FC8748406948B98548406B8449C862EF
:1044D000FF22042182483430FBF786FE8049496977
:1044E000874A88182A467E493431FDF78FFD0646F3
:1044F0007B48406928447A4948612EB97D49204665
:10450000FDF746FA07E010E000207549C862722105
:104510003620FDF71FFA724890F83408401C7049A5
:1045200081F8340800204870D2E06D488078002877
:1045300052D077222046611CCCB26E490A5400202A
:10454000674988700846007A012802D10020487225
:1045500002E000206249087361482430FCF7C2FB86
:104560005F48406A5E49096A88420BD15C48007A1C
:10457000012804D15A494872FDF764FD02E0012088
:10458000574908735648406A020E2046611CCCB257
:1045900058490A545248406AC0F307422046611CF9
:1045A000CCB254490A544E48808CC0F307222046AE
:1045B000611CCCB24F490A54494890F82420204647
:1045C000611CCCB24B490A542046FDF7E1F90020AA
:1045D0004349486208627BE04148C078012832D1F3
:1045E0003F48407A38B3FCF733FC20BB71222046A9
:1045F000611CCCB23F490A5401222046611CCCB256
:104600003C490A5402222046611CCCB239490A5462
:104610002046611CCCB237490A5400222046611C56
:10462000CCB234490A5401202D49C873314920467F
:10463000FDF7AEF903E022213120FDF78BF90020D0
:104640002749C87044E026484079E8B3002024494F
:10465000487171222046611CCCB226490A540122BD
:104660002046611CCCB223490A54FF222046611C1B
:10467000CCB220490A5401222046611CCCB21D490B
:104680000A5490460C2269461E48FBF7BFFDA0B9AC
:104690001348007B88B11248C06A1B490840B0F13A
:1046A000005F0AD104220E492C311548FDF7AEFCFB
:1046B00018B94FF00008FEF75FF82046611CCCB235
:1046C0000C4901F8008000E002E02046FDF760F9A7
:1046D000BDE8FE83533530385F44435532343031C2
:1046E000E431002044010020480100204C0100205A
:1046F00050010020843C0020243A002000F80020D3
:104700000080000800C000080000FE2F01200849BA
:104710004877002081F8220088714874A1F8400091
:1047200081F8240081F8250081F8270070470000F7
:10473000243A002070B5002400251748407801284D
:1047400028DD1648007900B970BD1449B1F842005F
:104750000321FCF7E4FB98B11148FCF7E9FE05469C
:10476000032D04DB0E492846FDF712F909E00B483A
:104770000079012805D1002008490871312400E0A2
:1047800013241CB121462220FDF7E4F81E20034922
:10479000A1F8460000BFD7E734010020243A0020EA
:1047A000843C00202DE9F04104460D4600260027F8
:1047B0001948407801282CDD18480079012828D1B3
:1047C0001649487F00220221FCF774FBB8B1032D83
:1047D00001DA132714E0A81E81B22046FDF732FD4E
:1047E000064656B96E200E490870207848706078E9
:1047F00088700320FDF7CCF802E0374600E07F2701
:104800001FB139462E20FDF7A5F828200349A1F84D
:104810004600BDE8F081000034010020243A002069
:10482000843C002070B504460025002617484078D7
:1048300001282ADD1649B1F842000221FCF76FFB7E
:10484000C8B1207800F07F0666B92078FCF760FBDD
:1048500090B17E200F490870207848700220FDF743
:1048600097F809E00A480079012805D10020084995
:104870000871122500E013251DB129463E20FDF7E1
:1048800069F80A200249A1F8460070BD34010020F1
:10489000243A0020843C00202DE9F04105460227FF
:1048A000002600246B484078012875DD10206949F6
:1048B0000870002048706848007908B9BDE8F081A8
:1048C0006549B1F842000221FCF729FB00287CD0A1
:1048D00005F07F04012C03D0022C01D0032C75D1EC
:1048E0005D48407F032845D1022C43D15A480079C6
:1048F00001283CD1FCF719FB002839D05648C07B71
:10490000002835D054484477FDF756FF5248447785
:104910000020514981F8220088714874A1F84000B4
:1049200081F8240081F8250081F827002846FCF74B
:10493000EFFA80B1502049490870084645700020C0
:1049400088703220C87001200871F4204871062751
:104950003846FDF71DF800204149087248728872F8
:10496000C87208738873C873487381F83C0862E0A2
:10497000222660E03848407F012801D1022C05D072
:104980003548407F022808D1032C06D132480079EF
:10499000012850D17E264EE05AE0032C0BD0012C8A
:1049A00009D12D48407F022805D101202A490870ED
:1049B000C82081F82000012C02D100202649C873AC
:1049C000254844770020244901E033E029E0A1F89C
:1049D000400081F82200887148740846407F03280F
:1049E00001D1032C07D000201B4981F8240081F855
:1049F000250081F827002846FCF78AFAD8B1502014
:104A00001649087008464570002088703220C8702A
:104A100001200871F420487106273846FCF7B8FFDA
:104A200009E00D480079012805D100200A490871E4
:104A3000122600E013261EB131461020FCF78AFF33
:104A40000A2004498880084680880349A1F8460066
:104A500000BF33E734010020243A0020843C0020CA
:104A6000E431002070B50446002500262A4840782D
:104A700001284EDD112028490870002048701E20B2
:104A800088802648007900B970BD2449B1F84200F9
:104A90000221FCF744FA002831D0207800F07F068C
:104AA0003046FCF72DFA08B3FCF73FFAE0B1207866
:104AB000FCF72EFA38B15120194908702078487057
:104AC0000220FCF765FF17488079012805D10020F6
:104AD0001449887112490870487001200F49087004
:104AE000C82081F820000BE0222509E00B4800795E
:104AF000012805D1002009490871122500E013257D
:104B00001DB129461120FCF725FF0A200349A1F811
:104B1000460000BFB8E7000034010020243A00201E
:104B2000843C0020E43100202DE9F04180460C4611
:104B300015460026FF27A048407801287EDD9F48C3
:104B4000007901287AD19D49487F01221146FCF75E
:104B5000B1F9002873D02078092806D19749487FF9
:104B600000220221FCF7A6F950B9207801284DD186
:104B70009249487F00220321FCF79CF9002845D088
:104B800000208F49087020788E4908708B49B1F851
:104B900042000221FCF7C3F9A8B38848C078012875
:104BA00001D13726FAE067208749087020784870DD
:104BB000824890F82200012808D180488079012895
:104BC00004D108460021C0F802100DE07B48407C6B
:104BD00050B97E48FCF796FC0120784948747A4821
:104BE0007A490968C0F802100120754908707349B4
:104BF000887167207049087000204870724906204B
:104C0000FCF7C6FECAE0FFE71326C7E020780A28B3
:104C100006D16A49487F00220221FCF74BF950B9BE
:104C20002078022876D16549487F00220321FCF7CD
:104C300041F900286ED00020604901E0B9E0ACE005
:104C40004874B1F842000621FCF769F9002875D0D4
:104C50005A4890F82800032802DC5948007880B9A7
:104C6000564890F82800032800DB36265448007880
:104C700028B1217853480078401C814292D02426E4
:104C80008CE04F480078012802D100204C49087080
:104C90004D4800210160818004224C49FBF7B6FA9F
:104CA00000285BD02178491EC8B2494A4749FCF721
:104CB000B5FB0746002F4FD160782870A078687048
:104CC000E078A8702079E870042241492846FBF773
:104CD0009DFA00BB0020394981F8280067203A4935
:104CE0000870207848702078022801D1012000E067
:104CF0000220324981F8230067202F4908700020E4
:104D0000487001202D4981F822002F490220FCF72C
:104D10003FFE24E02AE0294890F82800FF2806DA20
:104D2000264890F82800401C244981F82800234890
:104D300090F82800022802DC352610E014E01F4815
:104D400090F8280003280AD136260A201B4981F84A
:104D500029000120C87002E0122600E024261B482A
:104D600000210160818019E0132617E020780128D6
:104D700008D02078022805D02078092802D0207891
:104D80000A2801D17F2609E00C48B0F84200022829
:104D900001DA132602E0122600E07F261EB131461A
:104DA0002720FCF7D7FD1E20034988800349A1F87E
:104DB0004600BDE8F081000034010020243A0020C4
:104DC0005201002053010020843C00203A010020C1
:104DD0003E010020F8B505460E4600240020009054
:104DE00016484078012827DD3120144908701E201C
:104DF00088801348007901281ED11149487F01227B
:104E00001146FCF757F838B16B460E4A3146284632
:104E1000FDF74AFA044600E07F2424B12146312000
:104E2000FCF798FD04E00749BDF80000FCF7B0FD71
:104E30000A200349A1F84600F8BD00003401002013
:104E4000243A0020843C00202DE9F04104460E461F
:104E5000002748484078012870DD4748007908B9A4
:104E6000BDE8F0814449487F00220221FCF722F886
:104E7000002866D0404890F8220001285FD12578AC
:104E800094F801800A2E57D115B9B8F1440F01D01A
:104E9000312757E0A0780006E17840EA0140217907
:104EA00040EA01206179084334490860A07900068E
:104EB000E17940EA0140217A40EA0120617A084321
:104EC0002F49086074202F4908700846457020203B
:104ED0004870082088700220C87001202A4981F893
:104EE00034080020C1F83808486124480068274980
:104EF000884207D101202449087200204872C873F3
:104F0000C8721FE02048407A012813D11B4800686E
:104F10001F4988420ED11C48807A30B100201A49BE
:104F2000C8724871087208730CE0002014490860C8
:104F3000222707E0702705E0132703E017E0332757
:104F400000E07F2727B139463420FCF703FD07E056
:104F50000C490420FCF71CFD01200B4981F83C089A
:104F60001E200449888014200349A1F8460000BF90
:104F700076E7000034010020243A00202C010020B4
:104F800030010020843C0020E431002000F80020A3
:104F900000800008F8B505460E4600240020009069
:104FA0000E484078012818DD36200C4908701E2074
:104FB00088800B48007901280FD16B46094A314699
:104FC0002846FDF78BFA04461CB121463620FCF733
:104FD000C1FC1E200249A1F84600F8BD34010020A2
:104FE000243A0020843C0020F8B505460E460024F3
:104FF000772012490870002000901148407801285D
:105000001ADD10480079012816D177200C49087064
:105010001E208880002048706B46084A314628468A
:10502000FDF7C0FA04461CB121463720FCF792FC7C
:105030000A200449A1F84600F8BD0000843C002085
:1050400034010020243A002010B5FCF7E9FA0128C9
:1050500027D1FDF7B1FB02201749487701200873DB
:10506000002081F8220088714874A1F8400081F87E
:10507000240081F8250081F8270081F82900C870F4
:1050800050200E4908700C48407F487000208870FE
:105090003220C87001200871F42048710620FCF706
:1050A00077FC0020064908700220487001208870B3
:1050B0000020888010BD0000243A0020843C00209D
:1050C0003401002010B50848007F58B10649C87F58
:1050D00000F014F8002004490877C877FF2103483E
:1050E000FBF789F810BD0000243A0020EA090020EF
:1050F00010B50446FFF7E4F810BD000070B5054692
:10510000002415484078012825DD1448C07F342844
:1051100007D01248C07F362803D01048C07F3728F8
:1051200008D10E49487F00220221FBF7C3FE48B98F
:105130007F2407E009480079012803D100200749AE
:10514000087111241CB121462846FCF703FC0A20F3
:105150000249A1F8460070BD34010020243A002025
:105160001E200149888070473401002070B5054633
:105170000C4605480078272805D16078012802D11F
:105180002046FFF76BF870BD340100202DE9F04197
:1051900007460E4614464EBB3F484078012825D1AD
:1051A0003D48007840302178884207D12146384672
:1051B000FFF7DCFF0220384948706BE020787F2839
:1051C00068D1354800786178884263D1A078782822
:1051D00005D1FFF7C5FF04202F4948705AE0A07899
:1051E000FFF786FF03202C49487053E0002E44D17E
:1051F00029484078022840D12078102805D1022083
:105200002549487060782549887720782349C877F0
:10521000002518E02248405D2049C97F884210D10E
:105220001E48C07F342803D01C48C07F362805D1D3
:105230001C48008820B91C48457001E01A48457098
:1052400003E0681CC5B20B2DE4DB00BF0B2D02D1BF
:105250000A2015494870142110482B30FAF7CBFF6B
:105260001422611C0D482B30FAF79EFF01200B49D8
:1052700008770846A0F842700CE0092E0AD10B48C6
:105280000078012806D1002008490870FF2108484D
:10529000FAF7B1FFBDE8F08134010020243A002084
:1052A000A26000089A000020E8000020C000002052
:1052B000EA090020012001494870704734010020AC
:1052C000704710B500F08CF810BD70B504460D465F
:1052D000164632462946204600F052FA70BD70B597
:1052E00004460D46164632462946204600F08BFA03
:1052F00070BD00001149096851B94FF0E02189697A
:105300000E4A1160114609680D4A51430B4A11605B
:105310004FF0E0218969094A12688818074909682D
:1053200043F285621144054A116080B21146098832
:1053300001EB810140EA014070470000C4000020F9
:105340000DE37A050FB41FB5069800909DF8220072
:105350008DF804009DF804200DF123010DF10500E6
:10536000FAF722FF9DE80F0000F0A8F81FBC5DF8D7
:1053700014FB0FB587B000208DF81000079802903D
:105380009DF820008DF8120000208DF811009DF886
:1053900012200DF121010DF11300FAF705FF069817
:1053A000009002A80FC8FBF7DBFC0BB000BD10B5E6
:1053B0000A20FBF72BFEFCF7EBFD10BD10B50348F0
:1053C000C27903A10548FAF7EFFE10BD1E60000880
:1053D0003030323430313137000000008F06002089
:1053E00010B52F48007850B9FFF7E8FFFBF7A8FD8C
:1053F000FBF70AFEFFF78AF90120294908702948BE
:105400000078F0B1274890F8200038B1254890F88E
:105410002000401E234981F8200011E0002021498E
:10542000087000BF2048006800F4E0601F4908438E
:10543000001D1D490860BFF34F8F00BF00BFFEE78E
:1054400010BD1B480088401C80B219490880022802
:105450000DDB00200880FEF729FF01201149C871EB
:105460000020C87600F068F8002012490880124831
:105470000088401C80B210490880012805DB00200C
:105480000880FEF7FBFEFCF715FAFEF7A5FDFCF71A
:10549000E5F8FBF79BFCFEF71DFF00BFD0E700001F
:1054A000DE000020243A00200CED00E00000FA05A8
:1054B000D8000020DC000020DA0000200FB540F208
:1054C000DF710098884204D040F23471009888421D
:1054D0002FD118480088B0F5FA7F02DB002015496B
:1054E000088014480288001D00EB0210009901603A
:1054F0009DF804100F480288001D00EB0210017196
:105500009DF80D100B480288001D00EB021041733E
:1055100008480188001D00EB0110DDF8051040F877
:10552000051FDDF80910416002480088401C014950
:1055300008800FBD9012002010B51EE01248408870
:10554000B0F5FA7F02DB00200F4948800E488078D2
:105550000E4908700C484188001D00EB011494E8C6
:105560000F00FCF725FD08484088401C064948808C
:1055700007480068401C0649086003480088024943
:1055800049888842DAD110BD90120020C90000205D
:10559000D400002000BFFEE744E032213EE000BF1F
:1055A00000BF00BF00BF00BF00BF00BF00BF00BF03
:1055B00000BF00BF00BF00BF00BF00BF00BF00BFF3
:1055C00000BF00BF00BF00BF00BF00BF00BF00BFE3
:1055D00000BF00BF00BF00BF00BF00BF00BF00BFD3
:1055E00000BF00BF00BF00BF00BF00BF00BF00BFC3
:1055F00000BF00BF00BF00BF00BF00BF00BF00BFB3
:1056000000BF00BF00BF00BF00BF00BF00BF00BFA2
:1056100000BF00BF00BF00BF4A1ED1B20029BEDCE0
:10562000421ED0B20028B8DC704702E008C8121F42
:1056300008C1002AFAD170477047002001E001C17B
:10564000121F002AFBD1704708B501210820FCF782
:1056500021FD03208DF8020014208DF803004FF483
:105660008060ADF8000069460D48FBF700FE03209E
:105670008DF802004FF40060ADF8000014208DF8A2
:10568000030069460648FBF7F2FD4FF480610448C9
:10569000FBF7C2FE4FF400610148FBF7BDFE08BDF9
:1056A000000C0140022808DA074911F8301021B136
:1056B000054911F83010032900D170470221024A30
:1056C00002F8301000BFF8E76001002010B5044672
:1056D000022C03DA0C4810F8340000B910BD032086
:1056E000094901F8340001EBC401081D0021FEF74F
:1056F0007BFB1CB90548FAF78BFF02E00448FAF778
:1057000087FF00BFEAE7000060010020006400405E
:1057100000680040022800DB70470121024A02F8BD
:10572000301000BFF8E7000060010020022803DA13
:10573000074911F8301001B970470121044A02F8F5
:105740003010002102EBC002517000BFF4E70000EE
:10575000600100200146022908DA064810F83100ED
:1057600020B1044810F83100032801D1002070470F
:105770000120FCE76001002010B5FFF765FF10BDB8
:105780002DE9F04107460C461646FCF7B7F9A02074
:10579000FCF786F9FCF7E0F900B130E0A046E1172C
:1057A00004EB1161C1F30720FCF77AF9FCF7D4F997
:1057B00000B124E0E0B2FCF773F9FCF7CDF900B1D9
:1057C0001DE0FCF79BF9A120FCF76AF9FCF7C4F98E
:1057D00000B114E000250BE0711EA94201D00121A7
:1057E00000E000210846FCF731F97855681C85B2C5
:1057F000B542F1DBFCF79CF90120BDE8F081FCF734
:1058000097F90020F9E72DE9F04706460F46904644
:105810003C46002534E035B1E11704EBD161491174
:10582000A4EB411109BB25B1FCF782F90620FBF777
:10583000EDFBFCF763F9A020FCF732F9FCF78CF9DB
:1058400000B124E0A146E11704EB1161C1F3072088
:10585000FCF726F9FCF780F900B118E0E0B2FCF79C
:105860001FF9FCF779F900B111E0705DFCF718F948
:10587000FCF772F900B10AE0601C84B2681C85B2C2
:105880004545C8DBFCF754F90120BDE8F087FCF77B
:105890004FF90020F9E7002001E0411C88B23C28C4
:1058A000FBDB704786B0FDF703F8FAF7FAFCFCF76C
:1058B0002FFAFCF7C9FF01A8FCF7FCFBFCF71FFB64
:1058C000FCF75AFAFFF758FFFCF786F9FAF740FDA4
:1058D0004FF400712648FBF79DFDFFF768FDFBF7CD
:1058E000ABFE43E0FEF7A0FA22480078012805D17C
:1058F000002020490870FFF7E4FC37E01D4840789D
:10590000012805D100201B494870FCF761F92DE002
:1059100018488078012805D1002016498870FFF7C3
:10592000CFFC23E01348C078012803D1002011499F
:10593000C8701BE00F480079012803D100200D49F1
:10594000087113E00B484079012803D10020094970
:1059500048710BE00748C079012807D100200549AC
:10596000C8714FF400710248FBF754FDBAE700001C
:10597000000C0140840100202DE9F04704460F4649
:10598000154699463DB161190E48814203D8A0F5EC
:105990000070844203D24FF0FF30BDE8F08737B18A
:1059A000002602E0B85DA055761CAE42FAD3064848
:1059B000A4EB0008AAB21FFA88F12046FFF78FFC7B
:1059C0000020EAE7843C0020843A00202DE9F041E1
:1059D00004460D4616461F463B463246294620469B
:1059E000FFF7CAFF80464046BDE8F08130303234D0
:1059F00030313137000000000000211042206330B8
:105A00008440A550C660E770088129914AA16BB116
:105A10008CC1ADD1CEE1EFF13112100273325222BE
:105A2000B5529442F772D662399318837BB35AA366
:105A3000BDD39CC3FFF3DEE362244334200401148E
:105A4000E664C774A44485546AA54BB528850995B6
:105A5000EEE5CFF5ACC58DD553367226111630065E
:105A6000D776F6669556B4465BB77AA71997388706
:105A7000DFF7FEE79DD7BCC7C448E5588668A7781E
:105A80004008611802282338CCC9EDD98EE9AFF956
:105A9000488969990AA92BB9F55AD44AB77A966AFE
:105AA000711A500A333A122AFDDBDCCBBFFB9EEBA6
:105AB000799B588B3BBB1AABA66C877CE44CC55CCE
:105AC000222C033C600C411CAEED8FFDECCDCDDDF6
:105AD0002AAD0BBD688D499D977EB66ED55EF44E9E
:105AE000133E322E511E700E9FFFBEEFDDDFFCCF46
:105AF0001BBF3AAF599F788F8891A981CAB1EBA19A
:105B00000CD12DC14EF16FE18010A100C230E32015
:105B10000450254046706760B9839893FBA3DAB3BD
:105B20003DC31CD37FE35EF3B1029012F322D23265
:105B30003542145277625672EAB5CBA5A89589858D
:105B40006EF54FE52CD50DC5E234C324A0148104B5
:105B50006674476424540544DBA7FAB79987B8975D
:105B60005FE77EF71DC73CD7D326F2369106B01605
:105B700057667676154634564CD96DC90EF92FE91D
:105B8000C899E9898AB9ABA9445865480678276855
:105B9000C018E1088238A3287DCB5CDB3FEB1EFBFD
:105BA000F98BD89BBBAB9ABB754A545A376A167AA5
:105BB000F10AD01AB32A923A2EFD0FED6CDD4DCDCD
:105BC000AABD8BADE89DC98D267C076C645C454CF5
:105BD000A23C832CE01CC10C1FEF3EFF5DCF7CDF9D
:105BE0009BAFBABFD98FF89F176E367E554E745E45
:105BF000932EB23ED10EF01E0000000096300777C3
:105C00002C610EEEBA51099919C46D078FF46A70B0
:105C100035A563E9A395649E3288DB0EA4B8DC79D0
:105C20001EE9D5E088D9D2972B4CB609BD7CB17E50
:105C3000072DB8E7911DBF906410B71DF220B06A20
:105C40004871B9F3DE41BE847DD4DA1AEBE4DD6D30
:105C500051B5D4F4C785D38356986C13C0A86B6430
:105C60007AF962FDECC9658A4F5C0114D96C066350
:105C7000633D0FFAF50D088DC8206E3B5E10694C30
:105C8000E44160D5727167A2D1E4033C47D4044B70
:105C9000FD850DD26BB50AA5FAA8B5356C98B24250
:105CA000D6C9BBDB40F9BCACE36CD832755CDF45D0
:105CB000CF0DD6DC593DD1ABAC30D9263A00DE5100
:105CC0008051D7C81661D0BFB5F4B42123C4B356F0
:105CD0009995BACF0FA5BDB89EB802280888055F70
:105CE000B2D90CC624E90BB1877C6F2F114C6858D0
:105CF000AB1D61C13D2D66B69041DC760671DB01BE
:105D0000BC20D2982A10D5EF8985B1711FB5B6068F
:105D1000A5E4BF9F33D4B8E8A2C9077834F9000FCF
:105D20008EA8099618980EE1BB0D6A7F2D3D6D086F
:105D3000976C6491015C63E6F4516B6B62616C1C5F
:105D4000D83065854E0062F2ED95066C7BA5011B8F
:105D5000C1F4088257C40FF5C6D9B06550E9B7122F
:105D6000EAB8BE8B7C88B9FCDF1DDD62492DDA15EF
:105D7000F37CD38C654CD4FB5861B24DCE51B53A0F
:105D80007400BCA3E230BBD441A5DF4AD795D83D0F
:105D90006DC4D1A4FBF4D6D36AE96943FCD96E344F
:105DA000468867ADD0B860DA732D0444E51D03332F
:105DB0005F4C0AAAC97C0DDD3C710550AA4102273F
:105DC00010100BBE86200CC925B56857B3856F200F
:105DD00009D466B99FE461CE0EF9DE5E98C9D9296F
:105DE0002298D0B0B4A8D7C7173DB359810DB42EAF
:105DF0003B5CBDB7AD6CBAC02083B8EDB6B3BF9AFB
:105E00000CE2B6039AD2B1743947D5EAAF77D29D86
:105E10001526DB048316DC73120B63E3843B649466
:105E20003E6A6D0DA85A6A7A0BCF0EE49DFF099366
:105E300027AE000AB19E077D44930FF0D2A30887D6
:105E400068F2011EFEC206695D5762F7CB67658086
:105E500071366C19E7066B6E761BD4FEE02BD38986
:105E60005A7ADA10CC4ADD676FDFB9F9F9EFBE8EE6
:105E700043BEB717D58EB060E8A3D6D67E93D1A126
:105E8000C4C2D83852F2DF4FF167BBD16757BCA606
:105E9000DD06B53F4B36B248DA2B0DD84C1B0AAFA6
:105EA000F64A0336607A0441C3EF60DF55DF67A826
:105EB000EF8E6E3179BE69468CB361CB1A8366BCB6
:105EC000A0D26F2536E2685295770CCC03470BBB06
:105ED000B91602222F260555BE3BBAC5280BBDB206
:105EE000925AB42B046AB35CA7FFD7C231CFD0B5A6
:105EF0008B9ED92C1DAEDE5BB0C2649B26F263EC98
:105F00009CA36A750A936D02A906099C3F360EEBA5
:105F10008567077213570005824ABF95147AB8E265
:105F2000AE2BB17B381BB60C9B8ED2920DBED5E545
:105F3000B7EFDC7C21DFDB0BD4D2D38642E2D4F195
:105F4000F8B3DD686E83DA1FCD16BE815B26B9F625
:105F5000E177B06F7747B718E65A0888706A0FFF85
:105F6000CA3B06665C0B0111FF9E658F69AE62F845
:105F7000D3FF6B6145CF6C1678E20AA0EED20DD745
:105F80005483044EC2B30339612667A7F71660D065
:105F90004D476949DB776E3E4A6AD1AEDC5AD6D9A5
:105FA000660BDF40F03BD83753AEBCA9C59EBBDEC5
:105FB0007FCFB247E9FFB5301CF2BDBD8AC2BACA75
:105FC0003093B353A6A3B4240536D0BA9306D7CDE5
:105FD0002957DE54BF67D9232E7A66B3B84A61C405
:105FE000021B685D942B6F2A37BE0BB4A18E0CC3C5
:105FF0001BDF055A8DEF022D00000E001A0026004F
:1060000040004A0054006B0075008800CA00D400AC
:10601000E000E400E800EC00F000F400F8000C0AF6
:106020000A18080815081140080A020202020202B2
:10603000020087F18AF197F189F189F093F195F1E6
:1060400080F190F110F08CF184F100A001A0802F7C
:10605000812F822F832F842F00000000000000007A
:106060000101010101010001010100000000130014
:1060700055005F006B006F00730077007B0011001C
:10608000400008000A0002000200020002000200B4
:1060900090F110F08CF184F100A001A0812F822FEB
:1060A000832F1011222E273E313436377F00000017
:1060B000D060000800000020540100004C020008DD
:1060C0001C61000854010020B44300003A56000847
:1060D0001184A24A040009330102030406070809D7
:1060E000293B693F051902040608027B1F1345403E
:1060F0001B0875041A99041319411B08B9081339B0
:10610000421B08510C1A85041AC5041A051013C540
:0C611000500914C10A158018F1000000AD
:04000005080001519D
:00000001FF
:020000040800F2
:10800000808700206581000843D3000871C70008FD
:1080100041D3000899970008111B010800000000D7
:1080200000000000000000000000000099E60008C9
:108030005DB200080000000031DB00082DEE0008F2
:10804000FD1B01087F8100087F8100087F810008F7
:108050007F8100087F8100087F8100087F81000800
:108060007F8100087F8100087F8100087F810008F0
:108070007F8100087F8100087F8100087F810008E0
:108080007F8100087F8100087F8100082598000813
:108090009D9700087F810008BD9700087F81000838
:1080A0007F8100087F8100087F8100087F810008B0
:1080B0007F81000861EF00087F8100087F81000850
:1080C0007F8100087F8100087F8100087F81000890
:1080D0007F810008410C0108BD0C01088D0D0108CD
:1080E0007F8100087F8100087F8100080000000078
:1080F0000000000000000000000000000000000080
:1081000000000000000000007F8100087F8100085F
:1081100075FE000869FF00087F8100087F81000864
:108120007F8100087F8100087F8100087F8100082F
:108130007F8100087F8100087F810008ED9A000898
:108140007F810008199A0008559A00087F8100086D
:10815000DFF80CD000F078FC00480047E94901083E
:10816000808700200648804706480047FEE7FEE774
:10817000FEE7FEE7FEE7FEE7FEE7FEE7FEE7FEE7D7
:10818000C1EE000851810008202A04DB203A00FAE1
:1081900002F1002070479140C2F1200320FA03F35E
:1081A000194390407047202A04DB203A21FA02F05C
:1081B0000021704721FA02F3D040C2F12002914021
:1081C00008431946704740EA01039B0703D009E0C2
:1081D00008C9121F08C0042AFAD203E011F8013BB3
:1081E00000F8013B521EF9D27047D2B201E000F80C
:1081F000012B491EFBD270470022F6E710B513464B
:108200000A4604461946FFF7F0FF204610BD30B578
:1082100005462A460B4612F8010B13F8014B08B12C
:10822000A042F8D01CB1002802D06D1CF1E728460E
:1082300030BD421C10F8011B0029FBD1801A704789
:1082400030B504460020034600E05B1C934203D295
:10825000E05CCD5C401BF8D030BDF0B480EA010298
:10826000D40F4200B2EB410F02D20246084611463B
:108270004A0042D0C30DDDB2C1F3C752AD1A202D62
:1082800035DAC1F3160141F4000204B15242C5F1DE
:10829000200602FA06F12A411044B3EBD05F23D046
:1082A000C4B1012DA0EBC35009DCF0BC4FF000427B
:1082B00002EAC352DBB200F5000000F009BB400047
:1082C00000F1807000EBC350A0F1807040EAD170E3
:1082D000490009E0490841EAC071A0EBC35000F52C
:1082E0000000400800EBC350F0BC00F0E8BA614267
:1082F000012202EB4101001BF6E7F0BC704781F060
:108300000041AAE780F00040A7E780EA010210B52B
:1083100002F00043400022D04A001FD0010E01EBC2
:108320001261C0F35600C2F3560240F4000042F45A
:108330000002A0FB022000047F39140400D0401C7E
:1083400050EA124001D44000491EC2B20C0604EBB0
:10835000D010401C4008802A02D003E0002010BD4D
:1083600020F00100002900DA0020184310BD30B4CD
:1083700080EA010202F0004530F0004221F00040A6
:1083800013D090B1C30DD40DC2F31601C0F3160083
:10839000E41A41F4000140F400027D34914201D31B
:1083A000641C00E04900002C02DA30BC0020704759
:1083B0004FF400000023914201D3891A034340087F
:1083C0004FEA4101F7D151B1914202D14FF0004142
:1083D00005E002D24FF0010101E06FF0010103EB73
:1083E000C450284430BC00F06ABA2DE9FE4F8046E4
:1083F00081EA0300C00F0C46009021F0004123F0F9
:108400000045B8EB0200A94105D2404621469046FE
:108410001C460B46024623F00040104347D0270D70
:10842000C7F30A00C3F30A510290401A0190402892
:108430006BDAC3F3130040F4801B0098924620B11E
:108440000023D2EB030A63EB0B0B01985946C0F1F2
:1084500040025046FFF798FE06460D4650465946E4
:10846000019A00F01AFA10EB08006141002487EA33
:10847000115284EAE7731A4340D0009A62B3019A1A
:10848000012A4FEA075215DC001B61EB02014FF095
:10849000004202EA0752CDE90042001C41F580117A
:1084A00032462B4600F051FA03B0BDE8F08F40464B
:1084B0002146F9E7001B61EB0201001C41F5801326
:1084C00000185B412018A2F5001747EB030140EAB2
:1084D000D570B6196D4111E06D084FEA360645EAD0
:1084E000C0754FEA0752001B61EB0201001C41F509
:1084F000801149084FEA30000019514132462B469D
:1085000003B0BDE8F04F00F011BA0098012240001E
:108510000023D0EB020263EBE073009821464FEAA0
:10852000E074B8EB000061EB0401E9E783F000437D
:108530005BE781F0004158E72DE9FE4F81EA030433
:1085400004F0004421F0004100944FF0000B23F0B0
:10855000004350EA01045ED052EA03045BD0C3F347
:108560000A54C1F30A552C44A4F2F3340194A0FB3D
:108570000254C1F3130141F48011C3F3130343F414
:10858000801301FB024400FB034E840A970A44EA6D
:10859000815447EA8357A4FB076802958D0A05FBBF
:1085A00007854FEA932C04FB0C542705029D4FEAE4
:1085B000065847EA1637B5EB08056EEB070C870E31
:1085C000920E47EA811742EA8312A7FB0201B6EB3B
:1085D0000B0164EB00042B0D43EA0C335E1844EBF3
:1085E0001C50DA465146E7FB0201C5F313044FEA7B
:1085F0000B3343EA14534FEA0432019C43EA060367
:10860000A4F10C040294009CCDE900B400F09DF9A3
:1086100003B0BDE8F08F00200146F9E72DE9F04DE9
:1086200081EA030404F0004B21F0004514464FF0AA
:10863000000A23F0004150EA050220D054EA01026A
:108640001DD0C5F30A570246C5F31303C1F3130047
:10865000C1F30A5640F4801543F48013A7EB0608D3
:10866000101BD64608F2FD3873EB050002D308F163
:10867000010801E092185B41B8F1000F03DA002015
:108680000146BDE8F08D00204FF480110646844677
:108690000EE0171B73EB050705D3121B63EB0503F5
:1086A00006434CEA010C49084FEA300092185B413E
:1086B00050EA0107EDD152EA030012D082EA040029
:1086C00083EA0501084305D0101BAB4106D2012205
:1086D000002306E000224FF0004302E06FF00102A9
:1086E00053101AEB06004CEB085110EB0A0041EB5B
:1086F0000B01BDE8F04D00F019B970B521F0004351
:1087000003430CD0C1F30A550024D5EB040564EBF8
:108710000403D617AD1AB34102DB0020014670BD39
:10872000201841EB025170BDC10F80EAE07008448F
:10873000CA079623002100F0CBB8962300221146E9
:1087400000F0C6B80EB540F2334102910021CDE9E8
:1087500000110A460B4600F0F8F803B000BD20F007
:108760000040C10DC0F3160040F400007F2901DA7B
:1087700000207047962903DCC1F19601C84070477C
:1087800096398840704700F0004230F000400AD02F
:10879000C10D01F56071C0F3160042EA0151C20833
:1087A00040071143704700200146704701F0004325
:1087B00030B421F0004150EA010206D00A0DA2F5C2
:1087C0006072C1F31301002A02DC30BC0020704744
:1087D000440F44EAC104C100E01830BC00EBC250B1
:1087E00000F06DB8002801DBC0F10040002901DB7A
:1087F000C1F1004181427047002801DBC0F1004017
:10880000002901DBC1F100418842704730B50B46B9
:10881000014600202022012409E021FA02F59D42B0
:1088200005D303FA02F5491B04FA02F52844151E84
:10883000A2F10102F1DC30BD2DE9F05F0546002018
:1088400092469B4688460646814640241BE02846C1
:10885000414647462246FFF7A6FC53465A46C01AF1
:10886000914110D3114618462246FFF78DFC2D1A70
:1088700067EB01084F46224601200021FFF784FCE8
:1088800017EB00094E41201EA4F10104DFDC48462D
:1088900031462A464346BDE8F09F202A06DBCB1727
:1088A000203A41FA02F043EAE07306E041FA02F3AB
:1088B000D040C2F120029140084319467047002978
:1088C000A8BF7047401C490008BF20F00100704756
:1088D00010B4B0FA80FC00FA0CF050EA010404BFB6
:1088E00010BC704749B1CCF1200421FA04F411FA0C
:1088F0000CF118BF012121430843A3EB0C01CB1D50
:108900004FEA00614FEA102042BF002010BC7047C0
:1089100000EBC35010440029A4BF10BC7047401C9A
:10892000490008BF20F0010010BC704710B5141EAC
:1089300073F1000408DA401C41F1000192185B4118
:108940001A4301D120F0010010BD2DE9F04D9246EF
:108950009B4611B1B1FA81F202E0B0FA80F2203206
:108960009046FFF711FC04460F4640EA0A0041EA30
:108970000B0153465A46084313D0114653EA0100EF
:1089800019D0C8F140025046FFF70DFC05460E46CF
:10899000504659464246FFF7F7FB084305D00120F1
:1089A00004E020463946BDE8F08D0020054346EA44
:1089B000E0762C4337430A986305E40AA0EB0800ED
:1089C0000022FD0A44EA47540A3002D5002001463D
:1089D000E9E7010510196941DDE908450019694118
:1089E000BDE8F04DA2E7C1F30A52C1F3130140F212
:1089F000FF3341F480119A4202DA002001467047A9
:108A000040F233439A42A2F2334202DC5242FFF771
:108A1000CABBFFF7B9BB000030B5041E71F10004FA
:108A200004DB4FF00044404264EB0101141E73F17B
:108A3000000405DB1C464FF00043524263EB040385
:108A4000994208BF904230BD064C074D06E0E068F1
:108A500040F0010394E8070098471034AC42F6D385
:108A6000FFF77AFB1C7F01083C7F010870B58C186A
:108A700010F8015B15F0070301D110F8013B2A1132
:108A800006D110F8012B03E010F8016B01F8016B1F
:108A90005B1EF9D12B0705D40023521E0DD401F81B
:108AA000013BFAE710F8013BCB1A921C03E013F8E4
:108AB000015B01F8015B521EF9D5A142D8D3002019
:108AC00070BD0078704700002DE9F0411E4804F0A9
:108AD0007FFB1E4D0126002769791D4C884205D079
:108AE000207818B9042002F061FE88B1164804F01D
:108AF0006FFB6979884202D1207800B12770154850
:108B000004F066FBA97988420BD0607828B108E0B0
:108B10002670042009F0B6FDF1E7032002F046FEBE
:108B200058B10C4804F054FBA979884203D160780D
:108B3000002800D06770BDE8F0816670BDE8F041A4
:108B4000052009F09FBD00009C090020882300201B
:108B50003C070020A40900200029816802D041F0D0
:108B6000010101E021F00101816070470029816865
:108B700002D041F4807101E021F48071816070477E
:108B8000014600208968490700D501207047014649
:108B900000208968090700D50120704710B5426898
:108BA0000E4B0C791A400B6842EA042213434360CF
:108BB00083680B4A1340D1E9024222434C7943EACD
:108BC00044031A438260C26A097C22F47002491E7F
:108BD000C9B242EA0151C16210BD0000FFFEF0FFC0
:108BE000FDF7F1FF70B5072409290AD9C568A1F17D
:108BF0000A0606EB4606B440A543B3401D43C560D4
:108C000007E0056901EB4106B440A543B3401D43AD
:108C100005611F23072A09D2446B521E02EB820210
:108C200093409C4391400C43446370BD0D2A09D28C
:108C3000046BD21F02EB820293409C4391400C4391
:108C4000046370BDC46A0D3A02EB820293409C43F8
:108C500091400C43C46270BD816841F0080181609D
:108C600070470029816802D041F4A00101E021F49D
:108C7000A00181607047816841F004018160704704
:108C800038B590228DF8002001228DF801208DF852
:108C900002108DF803000B480024C0F8982103F05F
:108CA00031FE6D46285D03F06BFE0A20401E000475
:108CB000000CFBD1641CE4B2042CF3D303F044FE9B
:108CC00038BD00000080214208B50121082005F0D0
:108CD0003DFBC020ADF8000003208DF802001020FD
:108CE0008DF803006946054802F044FF044801215D
:108CF000C0F89C11C0F8981108BD0000000C01409C
:108D00000080214210B5084C207B18B1002060740F
:108D1000012010BD607C20B90120607405F0FCFBCF
:108D2000A060002010BD00002824002070B50121A3
:108D300092B0084605F0E6FA012140F2112005F054
:108D400005FB4FF4004005F0D3FA3920ADF84000A0
:108D500000248DF8434010A9334802F00BFF4FF474
:108D600060200B94CDE90D0401208DF831002F4EC9
:108D700004258DF830008DF83C500BA93046FFF7E4
:108D80000DFF052301220A213046FFF72BFF0523A3
:108D900002220D213046FFF725FF052303220E2175
:108DA0003046FFF71FFF052304220F213046FFF74F
:108DB00019FF1E4869464C300090801506901C48EB
:108DC0000190280207908020CDE9044020200890DF
:108DD000CDE90245C001CDE90904164C204602F058
:108DE00094F90121204602F085F901213046FFF770
:108DF000BDFE01213046FFF7AFFE3046FFF72CFFE6
:108E000034462046FFF7C3FE0028FAD12046FFF77C
:108E100032FF2046FFF7B4FE0028FAD10121204698
:108E2000FFF71FFF12B070BD001001400024014089
:108E3000500000200800024070B504460D460C208A
:108E40000CF010F82988018069684160216809B137
:108E5000626806E00121217260608060206070BD60
:108E600019468B689342FBD188602168816070BD90
:108E700010B50D4C0D49207851F8200080470B4962
:108E80002078203151F8200080472178074A01EBF3
:108E90004101C03A02EBC10151F82010002901D074
:108EA0008847207010BD0000602300205406002079
:108EB00000F00F01000900EB800001EB4000C0B2A0
:108EC000704710B5012005F04DFABDE810400020B4
:108ED00005F048BA00B50D48A1B041F20401A0F870
:108EE00005102021418000F5C371087C401C0874E6
:108EF00007A008F0DFFE20AA6946044802F022F924
:108F00000021084806F0C4FE21B000BD221F002049
:108F100073656E6420436861726765206461746183
:108F20000A0D0000DC01002010B50C4C94F86C0018
:108F3000642809D0206F0169884738B1206F8169A2
:108F4000884728B1012010BD062002E01C2000E067
:108F5000212002F039FC002010BD0000C8060020CE
:108F600000B50B48A1B041F20901A0F8051012218B
:108F7000418000F5C371087C401C087405A008F00E
:108F800099FE20AA6946024802F0DCF821B000BD33
:108F9000221F002053656E64204368617267696E0A
:108FA0006744617461200A0D0000000000B5A1B0A3
:108FB0000020ADF880000F4841F20301A0F8051031
:108FC0000D49097881720421418000F5C370017C4C
:108FD000491C017409A008F06DFE20AA69460548E5
:108FE00002F0B0F804480021503006F051FE21B0E4
:108FF00000BD0000221F00208801002073656E6400
:109000002073746174652064617461200A0D00002E
:1090100010B5242002F0BAFB0021044806F038FE07
:10902000BDE81040002001F01BBE0000942300208A
:1090300010B5124CA2B041F22100A4F80500A4F230
:1090400046404069E071010A2172010C6172000E14
:10905000A072042004F5C3716080087C401C087471
:1090600007A008F027FE20AA6946204602F06AF809
:109070000421E01D0AF076FE22B010BD221F002060
:109080000A0D7368656E676A6979696E6764612045
:109090000A0D000010B50F4CA2B04FF48150A4F897
:1090A00005005520E071AA202072022004F5C3714A
:1090B0006080087C401C087407A008F0FBFD20AA13
:1090C0006946204602F03EF80221E01D0AF04AFE01
:1090D00022B010BD221F00204F54412041434B209D
:1090E0000A0D000000B51848A1B041F20801A0F82F
:1090F000051016A100F2BE220B6816A1D362096802
:109100001163A0F1420242F8493F516000F2EA22A5
:109110009168C1730B0A03740B0C4374090E8174BC
:10912000117BC1740D21418000F5C371087C401C86
:1091300008740AA008F0BEFD20AA6946024802F0A1
:1091400001F821B000BD0000221F00205332303151
:1091500000000000574C494E4700000073656E64E4
:1091600020626D732076657273696F6E0A0D000060
:109170000549088A401C80B20882C82801D3AA2069
:1091800070470020704700006023002010B50121C7
:109190004FF0C05005F0C2F8BDE81040012004F0C7
:1091A000A7B9000070B5094D130AD2B205F5807653
:1091B00006E000BF10F8014B5C402B5D5340325D70
:1091C000491E89B2F6D242EA032070BDC07301087D
:1091D00070B5094DFF22134605F5807606E000BF05
:1091E00010F8014B54402A5D5A40335D491E89B244
:1091F000F6D243EA022070BDC0730108022101A02B
:1092000005F060B9415400000A2101A005F05AB9E7
:1092100041542B53544154453D3F000010B588B094
:10922000044620216846FEF7E7FF20216846FEF746
:10923000E3FF224606A1684608F04CFD6846FEF7AB
:10924000F8FF0146684605F03DF908B010BD000082
:1092500041542B4E414D453D25730000092101A08D
:1092600005F030B941542B4E414D453D3F000000C3
:109270000D2101A005F026B941542B554152545FF0
:109280004346473D3F0000000B2101A005F01AB9FD
:1092900041542B564552494F4E3D3F0070B5214D2C
:1092A000687801283DD1204C2078062830D2DFE8AC
:1092B00000F003130B2F1A2307221CA11D48FEF7F1
:1092C000BFFF28BB022015E00A221BA11948FEF7A8
:1092D000B7FFE8B901200DE01A491648FEF797FFDD
:1092E000B0B1042006E00B2217A11248FEF7A8FF38
:1092F00070B9052020700BE00E486060E88920817D
:109300000C480188A1F5B442A53A01D10BF0FCFD4F
:1093100000206870E881BDE8704080210548FEF7B4
:109320006BBF70BD88010020A820002041542B4F46
:109330004B0D0A00CC1B002041542B4F4B0D0A3023
:10934000333033003015002041542B4F4B0D0A3081
:10935000310D0A0010B5114C2078062819D2DFE82B
:1093600000F0030B07180F19BDE81040FFF746BFC8
:10937000BDE8104000F0F0B9BDE8104000F0B0B911
:1093800000F0D6F9064890F8760008B1012800D11F
:10939000A07010BDBDE8104000F004B8A820002067
:1093A000201500202DE9F041424E4348002596F853
:1093B000A810037C01290DD0404C4FF47A7132463D
:1093C0002186012792F87620142B0CD942B1012A6C
:1093D00008D008E00A2B01D386F8A850BDE8F08138
:1093E000857000E087708378052BF7D2DFE803F003
:1093F00004080B035500F1E7BDE8F04100F040B967
:1094000000F0FEF8E8E72D48403006F041FC012866
:10941000E4D1E08D401C80B2E085092800D9E585C3
:1094200026480021403006F033FCE08DA8B1012829
:1094300017D0022819D00328D0D0042819D0052825
:109440001BD006281DD007281FD0082821D00928A6
:10945000C4D1BDE8F04109F023BABDE8F04100F005
:10946000A3B8BDE8F041FFF735BDBDE8F041FFF717
:109470009DBDBDE8F04100F023B8BDE8F041FFF725
:1094800031BEBDE8F041FFF76BBDBDE8F04109F02A
:109490003BBABDE8F04109F0D9B9417C4B1C43749B
:1094A00014299BD905701AB1012A97D1877095E7C5
:1094B000857093E720150020A82000208801002057
:1094C00030B5A1B000202F4CADF8800041F207006C
:1094D000A4F805002C4842F21075818BC28BE17113
:1094E00001FB02F393FBF5F3090A21726272110A80
:1094F000A172E37290F82910217390F8281061731B
:109500002021A1735F21E173C27E2274C18C61743A
:10951000090AA174E274B0F809102175090A61758D
:10952000B0F80B10A175090AE175B0F801102176A9
:10953000090A6176B0F80510A176090AE176C179C9
:109540002177418A6177090AA17790F82A10E1779B
:1095500090F82B0084F820000CA008F0ABFB1A2038
:10956000608020AA6946204601F0ECFD04F5C37036
:10957000017C491C01740021094806F089FB21B0D7
:1095800030BD0000221F0020780C002073656E643F
:10959000204443444320646174610A0D00000000CC
:1095A000E001002004F082BF00B5A1B00020ADF8BA
:1095B00080000AA008F07EFB0E493A2020AA4880CD
:1095C00069460C4801F0BEFD0B48017C491C017442
:1095D00000210A4806F05CFB21B000BD73656E6493
:1095E00020686561727462656174206461746120D1
:1095F0000A0D0000221F0020A8200020D401002016
:1096000010B592B00020ADF8400040F6B8311348D4
:1096100006F03EFB01281FD1114C41F20100A4F8D5
:10962000050010A008F046FB1349A4F14200CA6EE1
:1096300040F8492F096F416010490A688260496803
:10964000C1601020608010AA6946204601F07AFDB2
:109650000021024806F01CFB12B010BDD001002012
:10966000221F002073656E64204C6F67696E206452
:109670006174610D0A00000020150020D0720108FD
:1096800010B592B00024ADF8404041F288310C484A
:1096900006F0FEFA012810D101030A48A0F80510CF
:1096A000448009A008F006FB10AA6946054801F0AD
:1096B00049FD0021024806F0EBFA12B010BD00008F
:1096C000CC010020221F002053656E642052656784
:1096D0006973746572656420646174610A0D0000C9
:1096E00010B54FF47A71104806F0D2FA012819D15A
:1096F0000D4C383CA07A20B1012804D0022807D0B4
:109700000AE0012007E00948FFF788FD022002E097
:10971000FFF7A4FD0020A072BDE810400021024820
:1097200006F0B6BA10BD0000C001002030150020C0
:1097300010B540F6B831074806F0AAFA012807D15B
:10974000FFF762FDBDE810400021024806F0A0BA14
:1097500010BD0000C401002010B54FF47A710D480F
:1097600006F096FA012814D10A4C343C607A10B104
:10977000012804D007E0FFF787FD012002E0FFF792
:1097800077FD00206072BDE810400021014806F01E
:109790007FBA10BDBC010020FEE7000000B585B017
:1097A0006A460021044800F089FD6946002009F05E
:1097B000D1FE05B000BD00000064004070B5174C3C
:1097C0004FF400752946204600F0B0FB01280CD16B
:1097D0001349204600F08FFB012802D1002009F038
:1097E00059FF2946204600F0D1F94FF480652946FB
:1097F000204600F09BFB01280FD109492046891C17
:1098000000F079FB012802D1002009F05BFF294616
:109810002046BDE8704000F0B9B970BD006400405A
:109820000200F01010B51A4C0021204600F0F6FDA1
:10983000022806D0012824D000220021084609F081
:10984000B5FE0121204600F0E9FD022806D00128DE
:1098500019D000220121002009F0A8FE0221204693
:1098600000F0DCFD022806D001280ED000220221E3
:10987000002009F09BFE2046BDE81040012100F0C9
:1098800085B90122D9E70122E4E70122EFE70000D0
:109890000064004070B58AB004F0FFFE0121092089
:1098A00004F054FD0121480604F038FD012188062A
:1098B00004F034FD504E0021304600F0B9FC701425
:1098C000ADF8200003208DF8220018204B4C8DF8B5
:1098D000230008A9204602F04DF9A014ADF820009D
:1098E00048208DF8230008A9204602F043F90024FF
:1098F00001258DF80A408DF80B5008208DF80800DE
:109900008DF80C408DF806408DF80D408DF807500D
:1099100006208DF80E40ADF804008DF80F508DF83C
:10992000095001A9304600F05DFB3548407BB0B1DD
:109930000E208DF81A008DF81B408DF81C50ADF8E4
:109940001040ADF81440ADF81240ADF81640ADF837
:1099500018508DF81D5004A800F0AAF903E0294919
:10996000002000F0B7FA01221021304600F032FB4F
:1099700041208DF800008DF801508DF802408DF8DF
:109980000350684603F0EEFC01221146304600F019
:1099900021FB01225102304600F01CFB0122910202
:1099A000304600F017FB0122D103304600F012FBD5
:1099B0000121304600F03CFC3F208DF800008DF87E
:1099C00001508DF802408DF80350684603F0CAFC40
:1099D00042208DF800008DF801508DF802408DF87E
:1099E0000350684603F0BEFC04F059FE06A008F0E0
:1099F00061F90AB0002070BD00680040000C014011
:109A0000282400200C05002063616E2032206F7036
:109A1000656E210A0000000000B50B4985B00120E9
:109A200088730A4804F078FE6A460121084800F06D
:109A300045FC9DF80900002803D16946012009F082
:109A400089FD05B000BD000028240020B4340020AA
:109A50000068004070B5214C4FF40075294620463F
:109A600000F064FA012810D11D4E2046314600F066
:109A700042FA012805D109F00DFE3146204600F0DA
:109A80006DF82946204600F081F84FF4806529469C
:109A9000204600F04BFA01281ED1114E2046B61C7C
:109AA000314600F028FA0F4A012807D00020107430
:109AB00029462046BDE8704000F068B8107C401C84
:109AC0001074094804F028FE012009F0FBFD31461E
:109AD000204600F043F8EBE770BD0000006800404E
:109AE0000200F01028240020BC34002010B51A4CCD
:109AF0000021204600F092FC022806D0012824D044
:109B000000220021012009F051FD0121204600F032
:109B100085FC022806D0012819D000220121084620
:109B200009F044FD0221204600F078FC022806D00E
:109B300001280ED000220221012009F037FD204625
:109B4000BDE81040012100F021B80122D9E701222F
:109B5000E4E70122EFE70000006800400A4A914272
:109B600002D1002181617047C1F313028B0101D53D
:109B7000C26070474B0101D502617047090101D5F0
:109B800082607047426070477000F03030B5082343
:109B900010240422B1F5007F1DD010DC202929D02B
:109BA00007DC012921D0042922D0082900D1C46072
:109BB00030BD402920D0B1F5807FF9D10BE00025E0
:109BC000B1F5004F06D008DCB1F5806F03D0B1F5D8
:109BD000006FEDD18561426030BDB1F5803F0DD0A1
:109BE000B1F5003FF8D1446030BD0549816030BD1A
:109BF000C36030BD036130BD046130BD436030BD22
:109C000001010100094910B588424FF0010101D15D
:109C10004C0601E04FF08064204604F08BFB2046A8
:109C2000BDE81040002104F085BB00000064004046
:109C300030B41446002819D000220272026042603B
:109C4000B1F5006F03D304250572416001E0027293
:109C5000016043B13CB142728372214630BC1A4666
:109C60000B30FEF7B0BA82720221417230BC7047ED
:109C700030B41446002819D00022027202604260FB
:109C8000B1F5006F03D304250572416001E0027253
:109C9000016043B13CB142728372214630BC1A4626
:109CA0000B30FEF790BA82720221417230BC7047CD
:109CB000F0B5827A012191402E4A136843F00103E6
:109CC00013602C4B1C331C688C431C60294D067B95
:109CD000294C0C35A6B92E688E432E604688C7885D
:109CE00046EA0746877A04EBC707C7F84066068846
:109CF000878846EA0746877A04EBC707C7F84466B1
:109D0000067B012E12D12E680E432E60867A0568DE
:109D100004EBC6064FEA3545C6F84056867A4568D4
:109D200004EBC6044FEA3545C4F84456114CC57AD5
:109D3000241D002D256806D00D4325600D4C058996
:109D4000143415B104E08D43F7E725688D43256091
:109D50000589012D02D125680D432560407B01282E
:109D600002D1186808431860106820F001001060E4
:109D7000F0BD000000660040006000402DE9FF419A
:109D8000064601250F460024284600F0DFFA012090
:109D90008DF80A508DF80B008DF80C00ADF8080016
:109DA0008DF80D0000254FF0040831E004EBD4706D
:109DB00020F00100201A401C012802D002281BD1EB
:109DC0000DE056F8351008EBC101090CADF8001094
:109DD00036F8351008EBC100ADF802000CE056F87B
:109DE000351008EBC101090CADF8041036F8351038
:109DF00008EBC100ADF80600641CE00707D1684617
:109E0000FFF756FF9DF80A00401C8DF80A006D1CF4
:109E1000BD42CBDBE00702D06846FFF749FFBDE853
:109E2000FF812DE9FF41804601250E46002428468A
:109E300000F08CFA01208DF80A5000218DF80B00FB
:109E40008DF80C10ADF808008DF80D000D464FF69A
:109E5000FF7736E0E01704EB907020F00300201A43
:109E6000401C012806D002280BD0032810D004285B
:109E70001BD114E038F8350007EA4010ADF80000B7
:109E800013E038F8350007EA4010ADF802000CE0A6
:109E900038F8350007EA4010ADF8040005E038F85E
:109EA000350007EA4010ADF80600641CA00707D192
:109EB0006846FFF7FDFE9DF80A00401C8DF80A0079
:109EC0006D1CB542C6DBA00702D06846FFF7F0FE66
:109ED000BDE8FF8110B50A46102118B1012805D050
:109EE000002010BD1046FFF79CFF02E01046FFF770
:109EF00045FF012010BD0246002011F4700F03D071
:109F0000926904E001207047CB0104D552680A40F1
:109F10001103F7D170470B0101D59268F7E78B0168
:109F200001D5D268F3E71269F1E70000024600208C
:109F300053690B424AD0B1F5807F3BD013DC08292E
:109F40002ED007DC012926D0022927D004293DD1B3
:109F5000D0682BE0102925D0202926D0402935D1E2
:109F60001069102130E0B1F5004F2BD00BDCB1F5BA
:109F7000007F22D0B1F5806F22D0B1F5006F25D1DE
:109F80009069702120E0B1F5803F11D0B1F5003F1C
:109F90001CD15068E5E790680D4915E0D06802E0F3
:109FA000D068DEE7106903210EE0106908210BE09C
:109FB0005068FBE79069012106E09069022103E007
:109FC000906900E05068042100F0C4BD70470000B3
:109FD00001010100002A426901D00A4300E08A43DE
:109FE0004261704710B50368002223F0020303604A
:109FF000036843F0010303604FF6FF7300E0521C57
:10A000004468E40701D19A42F9D14268D2073ED0B0
:10A010008A79012A02683CD022F080020260CA7963
:10A02000012A026838D022F0400202600A7A012A2E
:10A03000026834D022F0200202604A7A012A0268C3
:10A0400030D022F0100202608A7A012A02682CD0F5
:10A0500022F008020260CA7A012A026828D022F09F
:10A06000040202608A78CC78920742EA04620C7992
:10A0700042EA04424C79098842EA0452491E0A43E2
:10A08000C261016821F001010160002114E000209B
:10A0900010BD42F08002C1E742F04002C5E742F045
:10A0A0002002C9E742F01002CDE742F00802D1E7F2
:10A0B00042F00402D5E7491C4268D20701D0994218
:10A0C000F9D14068C007E2D1012010BD10460B0055
:10A0D00001D00021184770470846D1B2C0B20AF03B
:10A0E00063BA000070B58AB00121052004F02EF992
:10A0F0000121480604F012F9474E0021304600F0D5
:10A1000097F8B014ADF8200003208DF82200182035
:10A11000424C8DF8230008A9204601F02BFDE014E5
:10A12000ADF8200048208DF8230008A9204601F052
:10A1300021FD00248DF81A4001258DF81B500C20BC
:10A140008DF818008DF816408DF817400920ADF8ED
:10A15000140007948DF8195005A93046FFF742FF07
:10A160008DF80E408DF80F408DF81050ADF804407A
:10A17000ADF80840ADF80640ADF80A40ADF80C4027
:10A180008DF8115001A8FFF793FD012202213046FE
:10A19000FFF720FF14208DF800008DF801508DF896
:10A1A00002408DF80350684603F0DCF801221146A6
:10A1B0003046FFF70FFF012251023046FFF70AFF3A
:10A1C000012291023046FFF705FF0122D1033046FC
:10A1D000FFF700FF0121304600F02AF813208DF828
:10A1E00000008DF801508DF802408DF8035068464C
:10A1F00003F0B8F816208DF800008DF801508DF8A6
:10A2000002408DF80350684603F0ACF804A007F054
:10A2100051FD0AB0002070BD0064004000080140FC
:10A2200063616E2031206F70656E210A00000000AE
:10A2300000234FF6FF7221B1012917D0022924D043
:10A240003AE0016821F0020141F00101016000E003
:10A25000521E416801F00301012901D0002AF7D103
:10A26000406800F00300012823D124E0016821F0B8
:10A270000301016000E0521E4168890701D0002AF5
:10A28000F9D14068800714D115E0016821F001017F
:10A2900041F00201016000E0521E416801F003013B
:10A2A000022901D0002AF7D1406800F003000228FB
:10A2B00001D0002300E001231846704710B500EBE1
:10A2C0000113D3F8B04114F004041472D3F8B04170
:10A2D00034D0E408C2F80440D3F8B04104F00204DA
:10A2E0005472D3F8B44104F00F049472D3F8B4411B
:10A2F000240AD474D3F8B841D472D3F8B841240AEC
:10A300001473D3F8B841240C5473D3F8B841240E15
:10A310009473D3F8BC41D473D3F8BC41240A1474A9
:10A32000D3F8BC41240C5474D3F8BC311B0E937485
:10A3300039B1016941F02001016110BD640D146063
:10A34000CAE7C16841F02001C16010BD09490A682F
:10A3500042F001020A600A6843F60E739A430A60EB
:10A360000A6842EA00200860086820F001000860DE
:10A37000704700000066004030B502460020936838
:10A380005B0108D49068000101D5012003E09068CA
:10A39000C00037D5022002EB0012D2F8803103F062
:10A3A0000103C2F880310B7A73B3D2F880414D6853
:10A3B0001C434B7A43EAC5031C43C2F880418B7AA5
:10A3C00003F00F038B72D2F8843123F00F03C2F82D
:10A3D0008431D2F884318C7A2343C2F88431CB7A29
:10A3E000CC6843EA0423C2F88831CB7B096943EA8D
:10A3F0000121C2F88C11D2F8801141F00101C2F89C
:10A40000801130BD042030BDD2F880314C7A234316
:10A410000C8843EA4453C2F88031D0E7002221B1CE
:10A42000012905D0022906D112E08268114801E015
:10A430008268114802401149501A8A4214D00ADC3D
:10A44000A2B16FF0806010180FD002280CD10FE07D
:10A4500082680B48EEE7B0F5007F09D00949401843
:10A4600003D0B0F5003F03D00020704702207047B2
:10A4700001207047030000040003000800010008E9
:10A48000000003100001FFF770B512488188828830
:10A49000A0F1300400253038616AC06971B13C21F7
:10A4A000B0FBF1F0C000FEF748F90B49FDF75FFF84
:10A4B0000A4908606562E561256270BDA16A3C29B0
:10A4C00004D2491C1044A162E06170BD0120C4E9BE
:10A4D000090570BD5000002000401C46380C0020CB
:10A4E000054810B590F8210008B1012010BD2920C1
:10A4F00001F06AF9002010BDFC0C002010B50178B5
:10A50000427801EB0221144AA2F81B108178C3782B
:10A5100001EB032109B2B1F57A6F02DDA1F57A6191
:10A5200001E0C1F57A6109B20B4C8BB23D34A2F85F
:10A530001D300A2902DBA4F8073002E00021A4F84C
:10A5400007100179437901EB032122F81F1F80795D
:10A550009070012010BD0000FC0C002000B50246E8
:10A560000078FEF7A5FC134BD8725078FEF7A0FCDC
:10A5700018739078FEF79CFC5873D078FEF798FC1F
:10A5800098731079FEF794FCD8735079FEF790FC1D
:10A5900018749079FEF78CFC064958744839D1F844
:10A5A000532041F8012FB1F856208A80887101208C
:10A5B00000BD0000FC0C002010B508A007F07AFBDD
:10A5C00000F0A0F900F074F900F092F902F06CFFCD
:10A5D000044802F00EFE012010BD000054310D0AA7
:10A5E000000000008409002010B502A007F062FB03
:10A5F000022010BD5431300D0A00000010B502A039
:10A6000007F058FB062010BD5431310D0A00000040
:10A6100010B502A007F04EFB062010BD5431320DDC
:10A620000A00000010B504A007F044FB02F01CFF74
:10A6300000F068F9002010BD5431330D0A0000000D
:10A6400010B503A007F036FB00F05CF9012010BD47
:10A650005431340D0A00000010B509A007F02AFBA0
:10A6600002F002FF084C01202072084802F0C1FDF0
:10A670000020E071064802F09CFD072010BD00009C
:10A680005431350D0A000000882300207C09002089
:10A690006C09002010B509A007F00CFB094802F076
:10A6A00088FD00F025F902F0FFFE07490020087040
:10A6B000064908700649087010BD00005431360D77
:10A6C0000A00000084090020210000202000002052
:10A6D0000C0B002010B503A007F0ECFA02F0E4FE2A
:10A6E000022010BD54320D0A0000000010B502A077
:10A6F00007F0E0FA032010BD54330D0A00000000FB
:10A70000044810B50021C174018203A007F0D2FAF9
:10A71000042010BD6023002054340D0A0000000006
:10A7200010B502A007F0C6FA052010BD54350D0A79
:10A730000000000010B502A007F0BCFA062010BD12
:10A7400054360D0A0000000010B506A007F0B2FA5A
:10A7500006490020487100F0D5F802F085FE00207F
:10A7600010BD000054370D0A0000000074230020C3
:10A7700010B502A007F09EFA022010BD54380D0A51
:10A780000000000010B502A007F094FA022010BDEE
:10A7900054390D0A0000000010B5252000F0F6FF26
:10A7A0000021044805F074FABDE81040012000F0D3
:10A7B00057BA00009823002010B5154C606A002895
:10A7C00001DA14A01CE0606A400001D515A017E072
:10A7D000606A800001D518A012E0606AC00001D54F
:10A7E0001AA00DE0606A000101D51BA008E0606AB4
:10A7F000400101D51CA003E0606A800102D51DA0C4
:10A8000007F058FA606A40F08070606210BD000086
:10A8100000100240B5CDB9A6BAC4B8B4CEBB0D0A7B
:10A8200000000000B4B0BFDABFB4C3C5B9B7B8B454
:10A83000CEBB0D0A00000000B6C0C1A2BFB4C3C5A4
:10A84000B9B7B8B4CEBB0D0A00000000C8EDBCFE1D
:10A85000B8B4CEBB0D0A0000C9CFB5E72FB5F4B52B
:10A86000E7B8B4CEBB0D0A00D2FDBDC5B8B4CEBBAF
:10A870000D0A0000424F52B8B4CEBB0D0A000000D2
:10A8800010B5094802F095FC012000F0E8FC0748EB
:10A8900002F0AFFC4FF4FA7000F0E1FCBDE81040AC
:10A8A000024802F086BC0000C4090020CC09002048
:10A8B00010B502F0AFFB4FF4FA7000F0D0FC02F0DC
:10A8C000C5FB044901204871BDE8104002A007F013
:10A8D000F1B9000088230020434C4F53455F3132CB
:10A8E00056506F7765725265616C790D0A000000F1
:10A8F000024900200872024802F05BBC8823002055
:10A900007C090020024900208871024802F051BCF5
:10A91000882300205C090020024900208871024839
:10A9200002F047BC882300205C09002030B50C46AB
:10A93000054600F005F8024628190088504030BD51
:10A9400070B504464FF6FF7048F2050503460EE069
:10A9500014F8012B80EA02200022491E060403EAB3
:10A96000400000D56840521CD2B2082AF6D3002914
:10A97000EED170BD0A48026FB0F84630B0F848001A
:10A98000118801EB81014900B1FBF3F1494201EB70
:10A9900081014FF2600303EB41010844508070478E
:10A9A000C80600200120704770B5124D124C28785F
:10A9B000072811D011480069804702280CD00020D8
:10A9C00020702878801E042801D8012020700620DD
:10A9D00000F0ECFE48B901E00320F1E728780628F2
:10A9E00005D1074802F0F4FB08B902202070207856
:10A9F00070BD0000602300208C050020580000205E
:10AA0000A40900200088322801D8012070470020C6
:10AA10007047000010B506480649C08F898A8842F1
:10AA200004D2282000F0D0FE002010BD012010BD6F
:10AA3000C8060020FC0C00201D4810B5007920B18C
:10AA4000012807D002280CD108E01121194801F093
:10AA50002FF806E0174801F057F802E0112001F046
:10AA600063F8134832213038044605F011F9012803
:10AA700005D108F089F80021204605F009F90E49B2
:10AA8000886BC20612D520F0100088630848FA21AE
:10AA90002838044605F0FCF8012807D108F0CEFA62
:10AAA0002046BDE81040002105F0F2B810BD0000BE
:10AAB00074230020B52C0108FC0C002070B5204D3B
:10AAC0000026A889401C80B2A8810A2802D3AE8142
:10AAD00001F0EAFA1B491C4CA1F1FC008A88130A18
:10AAE00000F8E83F42708A790274C9794174688934
:10AAF000401C80B26881642814D36E81134D94F891
:10AB00002800297881420DD0287008212846FFF7B7
:10AB100017FF2872000A687200230A2229460C488F
:10AB200000F062FD6078012808D1A078012805D1E5
:10AB30006670A67001F016FE0120607170BD000005
:10AB4000100B0020CC350020A0440020F64400204B
:10AB500000450020024600200A4200D00120704734
:10AB6000034900200978490700D5012070470000FB
:10AB7000CC350020034900200978890700D5012041
:10AB800070470000CC350020034600201AB18B42EC
:10AB900000D0012070478B42FBD070470349002052
:10ABA000497A002900D0012070470000CC350020F0
:10ABB0000021012801D0032800D101210846704757
:10ABC0000021012805D0022803D0042801D00A283A
:10ABD00000D101210846704701460020090600D433
:10ABE00001207047024600208A4200D101207047B0
:10ABF0000120704770B517490020174E08601439BE
:10AC00000446C87004EBC40006EB40050C35102167
:10AC10002846FDF7F1FA10212846FFF791FE287427
:10AC2000000A641CE4B26874122CEBD30A494FF496
:10AC3000A2740C3122460D4601F5A270FDF7C3FA4D
:10AC4000002322462946054800F0CEFCBDE87040AE
:10AC500006F0ECB9240B0020E435002089450020E3
:10AC6000024A012110440172704700009423002021
:10AC7000044810B500698047022801D0002010BDAB
:10AC8000012010BD5800002070B58F4805210646F0
:10AC900003F030FD8D4C002518B12573304603F0CC
:10ACA0003BFD894805210830064603F023FD18B115
:10ACB000A573304603F030FD834805211030064669
:10ACC00003F018FD18B12574304603F025FD804CC3
:10ACD000E06880477F49884203DA2A2000F066FD59
:10ACE00040B3E06880477C49884206DB2A2000F0B8
:10ACF0005DFD10B12A2000F049FDE06880477749EA
:10AD0000884203DD322000F051FDB8B1E068804791
:10AD10007349884206DC322000F048FD10B1322031
:10AD200000F034FD6F4C94F84C00C0F30100032890
:10AD300008D00AE02A2000F047FDDEE7322000F0CC
:10AD400043FDEFE72E2000F03FFD606CC0F3816013
:10AD5000032802D10B2000F037FD606CC0F30170B6
:10AD6000032802D12B2000F02FFD606C800F0328F8
:10AD700002D12C2000F028FD606CC0F301400328B4
:10AD800002D12D2000F020FD606CC0F3815003281B
:10AD900002D10C2000F018FD94F84400C0F300002C
:10ADA00010B10D2000F010FDB4F84400C0F3813064
:10ADB000032802D10E2000F007FD94F84400C0F3F0
:10ADC000800010B10F2000F0FFFC94F84400C0F3A5
:10ADD000C00010B1102000F0F7FC94F84400C0F35C
:10ADE000001010B1112000F0EFFC94F84400C0F303
:10ADF000401010B1122000F0E7FC94F84400C0F3BA
:10AE00008110032802D1132000F0DEFC206CC0F377
:10AE1000806010B1142000F0D7FC206CC0F30060FB
:10AE200010B1152000F0D0FC206CC0F3406010B1D0
:10AE3000162000F0C9FC206CC0F3007010B1172080
:10AE400000F0C2FC206CC00F02D0182000F0BCFC47
:10AE5000206CC0F3404010B1192000F0B5FC206C0C
:10AE6000C0F30150032802D11A2000F0ADFCB4F861
:10AE70004000C0F3C02010B11B2000F0A5FC94F8E6
:10AE80005C00C0F3800010B11D2000F09DFC94F820
:10AE90005C00C0F3C00010B11E2000F095FC94F8D7
:10AEA0005C00C0F3401010B11F2000F08DFC94F83E
:10AEB0005C00C0F3C010002804D0BDE87040202022
:10AEC00000F082BC70BD0000AC34002028240020BB
:10AED000580000200000084100001041000094418B
:10AEE00000009041B022002070B51949194800F0C7
:10AEF00079FD0546174818490C3000F073FD1649D6
:10AF0000164C1D39B1F81D10B9B1012D05D0B1F5A0
:10AF1000A07F12D9032804D00FE0012000F054FCD8
:10AF200012E00321204603F0E5FB30B1052000F0DC
:10AF30004BFC204603F0F0FB06E0204603F0ECFB60
:10AF4000032000F033FC08B1002070BD012070BD6B
:10AF5000440C0020B8230020190D00209C34002050
:10AF600010B52A2000F022FC08B9FDF7ADFD114C08
:10AF700060688047552803DB302000F025FC06E0A0
:10AF800060688047502802DC302000F0FFFB0A4850
:10AF900090F90000552804DBBDE81040312000F096
:10AFA00013BC502804DCBDE81040312000F0EEBB9B
:10AFB00010BD000058000020882300200A4810B56A
:10AFC0000078002448B1411E032901D8012404E07F
:10AFD000052801D0072800D1022400F0C9FB00B1E8
:10AFE0000324204610BD00006023002010B541F26C
:10AFF000883421460D4804F04BFE012808D00B4848
:10B000002146001F04F044FE012806D0012010BD97
:10B01000252000F0D9FB012003E0242000F0D4FB20
:10B02000002003F0A9FD002010BD0000982300209F
:10B03000007870472DE9FE4F01A9264800F0C4FAB8
:10B04000254D264E264FDFF89C80DFF89C9000248B
:10B0500036F8140000F0A2FFFF2813D037F81000D4
:10B0600001992844029039F8140038F814B00844C3
:10B0700082465946FFF75AFC20B95A465146029873
:10B08000FDF7A1F8641CE4B2092CE1D306F0A6F99F
:10B09000104869460A3800F097FA08210098FFF72F
:10B0A00045FC124938B1002081F82900C87081F8A8
:10B0B0002800BDE8FE8F00980D4A0078107081F8D6
:10B0C00028000328F5D30A2081F829000120C87040
:10B0D000EFE700000A450020D03400203478010852
:10B0E000D47701085878010846780108A044002068
:10B0F000F64400200029016802D041F0010102E07D
:10B100004FF6FE7211400160704730B5036847F694
:10B11000F07293430C6A8A682243D1E904452C43B8
:10B1200022438C692243CC6922434C6A22438C6AB5
:10B1300022431A430260CA6842600A688260496812
:10B14000C16030BD70B50C46050033D08CB3688843
:10B15000A52121705A2161701930A070000AE07099
:10B1600020202071601D10221349FDF72CF868790A
:10B170006075B5F805001726000AA0756A88022ACE
:10B1800007D304F11700E91DFDF71DF8A878173063
:10B19000C6B231462046FEF71BF8A055761CF1B228
:10B1A000000A6054491CC9B22046FEF7FBF9012091
:10B1B00070BDFFE70020FBE720150020F8B56946C9
:10B1C000214800F001FA1226204F0024009804EBD9
:10B1D000C40500EB4500B11EFFF7A8FB88B9009835
:10B1E000324600EB450107EB45000C30FCF7EBFF66
:10B1F0000098324600EB4501154800EB4500FCF78E
:10B20000E2FF07EB4500007B092805D11148012129
:10B21000A14002680A430260641CE4B2122CD5D338
:10B2200006F0F2F80B494FF4FA701439888018319F
:10B230004FF0FF30A1F1150208600749A1F5227017
:10B2400003F078FDF8BD000089450020E4350020BA
:10B2500034370020240B002078380020704710B5C8
:10B26000044606E0142006F0DDFC01F0ABFC641E91
:10B27000A4B2002CF6D110BD70B5044600F0A2FEB9
:10B280000646FF2822D0204600F088FEFF281DD069
:10B290000F49114A0C5C0F4932F81000451821463D
:10B2A0002846FFF74DFB2855641C000A28550B481B
:10B2B000621C30F816100A48081803D000232946EB
:10B2C00000F092F9BDE8704006F088B870BD00004B
:10B2D000FA770108D0340020D477010846780108B5
:10B2E0000A4500202DE9F8411C46002688468DF8C5
:10B2F0000060217815464A1C592322706B5421782E
:10B30000194F4A1C227068546A463946404603F079
:10B3100011FD22E037F816002178020A13484B1C71
:10B3200050F8220023704FEA104C05F801C0217834
:10B330004FEA102C4B1C237005F801C021784B1CE0
:10B340002370685402EBC20108EB41004278207878
:10B35000411C2170761C2A54F6B29DF800008642EA
:10B36000D8D30020BDE8F881783800206477010840
:10B370002DE9F0434FF05908DDE90754002694F811
:10B3800000C04FF001090CF10107277005F80C808F
:10B39000277807F1010C84F800C0E855224F21F00E
:10B3A0007F4000BF57F826C0604536D120784FEA6D
:10B3B000114C471C277005F800C020784FEA112C6B
:10B3C000471C277005F800C02078471C27702954B7
:10B3D00006EBC601267813F81170701C2070AF556B
:10B3E000012A01D0FF2A1CD103EB41014FF00009D3
:10B3F000487BB0B120780123421C22702B54227864
:10B400000823501C2070AB542078891C284403F07A
:10B410004DFC21780844207003E0761CF6B2122E11
:10B42000C0D34846BDE8F08364770108524B10B59D
:10B43000524A18781168C40602D541F0200101E093
:10B4400021F0200111608106116802D541F0400110
:10B4500001E021F0400111604106116802D541F080
:10B46000800101E021F080011160000602D541F465
:10B47000807001E021F4807010605878C107116875
:10B4800002D041F4007101E021F4007111608107E4
:10B49000116802D541F4806101E021F480611160FE
:10B4A0004107116802D541F4006101E021F4006117
:10B4B00011600107116802D541F4805101E021F4C7
:10B4C00080511160C106116802D541F4005101E0BC
:10B4D00021F4005111608106116802D541F48041C8
:10B4E00001E021F4804111604106116802D541F468
:10B4F000004101E021F400411160000602D541F451
:10B50000803001E021F4803010609878C007106826
:10B5100002D040F4003001E020F400301060FFF76A
:10B520003DFB28B3587A082803D3106840F0100078
:10B530001060FFF733FB002819D110481438C18878
:10B54000491C8BB20021C380C82B04D9136843F077
:10B5500001031360C18003895B1C9BB20381B3F5B7
:10B56000967F04D9136843F002031360018110BD74
:10B57000106820F01000DBE7CC350020240B002001
:10B5800030B50C460F4A00EBC00102EB41030C4DF5
:10B590000C33122813D21878A0420FD0092C0DD1E9
:10B5A000184603F0B9FB587818B92878401C287061
:10B5B0005870587BFF2801D0401C58731C7030BD58
:10B5C000130B0020E4350020064A824205D07F3A62
:10B5D000824202D00A3A824202D101200A607047B8
:10B5E000002070478945002010B50BF02FFB01208B
:10B5F00010BD000001A006F05DBB00004556454EA1
:10B60000545F410D0A00000070B515A006F052FB12
:10B61000164D00244FF4FA766879D0B101F024FF7A
:10B620003046FFF71CFE6879B0B101F01DFF3046CF
:10B63000FFF715FE0E4801F0CBFD697988420ED068
:10B64000641CE4B2052CE7D3BDE87040042000F090
:10B65000BBB8FFF72DF9E3E7FFF72AF9E7E770BD7D
:10B660004556454E545F41430D0A00008823002093
:10B670009C09002001A006F01DBB00004556454E68
:10B68000545F420D0A00000001A006F013BB000049
:10B690004556454E545F430D0A00000070B516A094
:10B6A00006F008FB174D00244FF4FA76A87901281C
:10B6B0001BD001F00DFF3046FFF7D1FDA87901281E
:10B6C00016D001F005FF3046FFF7C9FD0E4801F026
:10B6D0007FFDA97988420ED0641CE4B2052CE5D325
:10B6E000BDE87040032000F06FB8FFF715F9E2E7FE
:10B6F000FFF712F9E7E770BD4556454E545F4443E6
:10B700000D0A000088230020A409002010B5102194
:10B710000548FCF771FD05490020086008710839EB
:10B720000860486010BD0000182400202C0800208C
:10B7300070B50A4C052604F1080520686168884246
:10B740000BD0295C06A006F0B5FA2068401C90FBDF
:10B75000F6F106FB11002060F0E770BD2408002020
:10B76000457272204E554D2069732025640D0A00E4
:10B77000054900200A5C0AB101207047401CC0B294
:10B780001028F7D3002070471824002010B5034676
:10B7900000F00CF830B1DC08184600F079F90249E5
:10B7A00000200855012010BD18240020C20800F018
:10B7B00007010448805C01228A40104000D001202B
:10B7C000704700001824002010B50346FFF7EEFF75
:10B7D000A0B90B4AA2F10801486813540522401C85
:10B7E00090FBF2F402FB140048600649D80803F00D
:10B7F00007030A5C01249C4022430A54012010BD27
:10B800002C080020182400200149C860704700005F
:10B810000020024070B50D4E0546304600F088F815
:10B82000042811D10A4C206940F0020020616561B2
:10B83000206940F040002061304600F079F821692D
:10B8400041F6FD721140216170BD0000FFFF0F0045
:10B850000020024008490420CA68D20701D0012014
:10B860007047CA68520701D502207047C968C906E7
:10B87000FBD5032070470000002002400248016908
:10B8800041F080010161704700200240F0B506469A
:10B890004FF6FF770D46384600F04AF804280DD1E0
:10B8A000074C206940F0010020613580384600F0E7
:10B8B0003FF8216941F6FE7211402161F0BD0000A0
:10B8C000002002402DE9F841064600204FF6FF77A0
:10B8D00000900D46384600F02BF8042817D10D4C87
:10B8E000206940F0010020613580B846384600F0FC
:10B8F0001FF841F6FE77042806D1B61C280C0096E6
:10B900003080404600F014F8216939402161BDE8DB
:10B91000F8810000002002400348024941600349C9
:10B92000416070472301674500200240AB89EFCD9D
:10B9300000B50346FFF78EFF03E000BFFFF78AFF65
:10B940005B1E012803D0002B00D1052000BD002B79
:10B95000F4D1FAE70A290FD801EB4102074903881D
:10B9600021F8223001EB820183788B70C278CA7093
:10B9700002790A718068886070470000A023002067
:10B9800000B501211648FFF7E5FF154802210C30EC
:10B99000FFF7E0FF124803211830FFF7DBFF1048E4
:10B9A00004212430FFF7D6FF0D4805213030FFF782
:10B9B000D1FF0B4806213C30FFF7CCFF0848072198
:10B9C0004830FFF7C7FF064808215430FFF7C2FF91
:10B9D0000348092160305DF804EBFFF7BBBF0000AE
:10B9E000B807002010B504468268084690472179C0
:10B9F0000022814202D0A27020710CE0E3788342E1
:10BA000001D1A27007E0A078401CC0B2A0702288CB
:10BA1000904200D3E170E07810BD00002DE9F047BE
:10BA200081461A48184C00278088401E86B204EBD5
:10BA3000C60041684846FCF7D5FE04D34846616815
:10BA4000FCF7DAFE18D240F6FF70BDE8F087B819AF
:10BA5000450804EBC5084846D8F80410FCF7CCFEAE
:10BA600002D26D1EAEB207E04846D8F80410FCF7CB
:10BA7000B9FE06D26D1CAFB2B742E8D934F937002F
:10BA8000E3E734F93500E0E7546D010820000020B9
:10BA9000064A0021535C834202D100205054704773
:10BAA000491CC9B20529F5D3704700002C080020B5
:10BAB0002DE9F041074612480E466421804604F005
:10BAC000E7F800250F4C012806D1B847E5720021A0
:10BAD0004046656004F0DCF8E07A11280ED1607C05
:10BAE000B0420BD1606841F6EC41B1EB104F05D18B
:10BAF00003490120E572403165600871BDE8F081BD
:10BB0000342300204C0D002010B501460220884748
:10BB100004490220087103480021BDE810403C3868
:10BB200004F0B6B87423002070B50F4900240F4DFF
:10BB3000CA7A0F4E132A0CD14A7C824209D1486836
:10BB400041F6EC42B2EB104F03D1CC724C602C7139
:10BB5000B463064832213C3804F09AF8012801D138
:10BB60002C71B46370BD00004C0D002074230020C4
:10BB7000FC0C0020F0B5CA78002502F00F03D206B5
:10BB800001D58A7813430A784FF00F0E12F0FF0F99
:10BB90004FF001021CD004680F8802FA05F6374006
:10BBA000B74211D14FEA850C0EFA0CF724EA0707C9
:10BBB00003FA0CF43C43CF78282F02D0482F02D050
:10BBC00002E0466100E006616D1C082DE4D30460CC
:10BBD0000C88FF2C1ED944685FF0000606F10807A8
:10BBE00002FA07F50F882F40AF420FD14FEA860CBB
:10BBF0000EFA0CF7BC4303FA0CF73C43CF78282F1E
:10BC000000D14561CF78482F00D10561761C082E00
:10BC1000E4D34460F0BD0000F0B5144C002801DA14
:10BC2000E36900E06368420D120185B2C0F3015779
:10BC30009540C0F30346032F05D0C2020AD5032264
:10BC4000B240934307E023F07062636823F07063AF
:10BC5000636002E0AB4343F0706201B12A43002805
:10BC600001DAE261F0BD6260F0BD00000000014059
:10BC70000246002092680A4200D0012070474161CC
:10BC800070470161704700787047000070B50C4C38
:10BC9000206980470B4D02280BD10B480321064633
:10BCA00002F028FD28B1304602F036FDA06880473A
:10BCB00004E020698047022801D00020287070BD70
:10BCC0005800002088230020A43400200C4810B520
:10BCD00040880B4A01211C3A05F04AFF08483038D9
:10BCE0004069FCF750FD02460B4606480649FCF742
:10BCF00095FCFCF75BFDFFF791FE0449488110BD00
:10BD0000500000209A99999999991340380C002075
:10BD10007CB5002328A40093246801946D4601ACEF
:10BD2000012825D0C85CE65C7040E8545B1CDBB29F
:10BD3000042BF7D39DF800109DF8010001F00F04CB
:10BD4000034664F31F13137003099DF8020043EACE
:10BD5000001353709DF8033003F0F00444EA101010
:10BD6000907003F00F0040EA1110D07000207CBDED
:10BD7000C85CE65C7040E8545B1CDBB2042BF7D374
:10BD80009DF801109DF8000001F0F00343EA001354
:10BD900013700B019DF8021043EA1113537001F068
:10BDA000F0039DF8031043EA111301F00F019370A3
:10BDB00061F31F10D9E700009023B02170B505464C
:10BDC00005F01AF94443601C01D01CB105E06FF086
:10BDD000A90402E005F010F904462C70200C6870EC
:10BDE000200AA870EC70002070BD0000FEB500268F
:10BDF00004468DF8086053783D480D460B2974D2EF
:10BE0000DFE801F0730606596073717373730600FF
:10BE10000A4602A9204600F0F9F802004FF0590046
:10BE20004FF0090115D18DF8086020709DF80820A9
:10BE3000521CD2B28DF80820A5549DF80820521C3F
:10BE4000D2B28DF80820A1549DF80820521C8DF81C
:10BE50000820012D49D18DF8086020709DF8080058
:10BE6000401CC0B28DF8080025549DF80800401C05
:10BE7000C0B28DF8080021549DF80800401CC0B2E3
:10BE80008DF8080026549DF80800401CC1B21848DF
:10BE90008DF808100C38C27A62549DF80810491CBD
:10BEA000C9B28DF80810807A60549DF80800401CD3
:10BEB0008DF8080019E0014602AB22462846FFF73C
:10BEC00011FA12E063F31741937863F30F21D378EB
:10BED000127963F3070102ABCDE90043034628461C
:10BEE000FFF746FA08B18DF808609DF80800FEBD1E
:10BEF000F035002070B516490324164B91F82C201C
:10BF000091F82B10144D02EB01218AB262210170CD
:10BF1000110A41708270002135F81160964203D0F9
:10BF2000491CC9B21329F7D313290ED0022C0AD009
:10BF30000A4A2044555C0A4A32F811102A4619442C
:10BF4000FCF741F92C44204670BD0224FBE70000B9
:10BF5000A0440020D03400200E780108FA770108B0
:10BF6000D477010800B5FEF7FBFD0B4A00281068E6
:10BF700002D040F0080001E020F008001060FEF759
:10BF8000F9FD0028106802D040F0040001E020F024
:10BF90000400106000BD0000240B0020024610B514
:10BFA000FF20074B002100BF33F81140944201D11C
:10BFB000084610BD491CC9B21329F5D310BD0000B5
:10BFC0000E780108024610B5FF20074B002100BF84
:10BFD00033F81140944201D1084610BD491CC9B242
:10BFE0000929F5D310BD000034780108007A7047A4
:10BFF000007970470148B0F90A007047380C0020FA
:10C00000533530385F444355323430312DE9F043F5
:10C01000224C002759256781057042700925894601
:10C02000857039465FF0030501EBC10604EB460C51
:10C030009CF80C601E4203D19E4201D00A2A23D1F3
:10C04000174E3668CE40F6071ED066890127761C4B
:10C050006681144E56F821804FEA184800F8058092
:10C060006D1C36F82180EDB24FEA182800F80580E3
:10C070006D1CEDB216F8216046556D1CEDB29CF8B2
:10C080000C6046556D1CEDB2491CC9B21229CBD3C8
:10C0900089F800503846BDE8F0830000E435002000
:10C0A000280B0020647701082DE9F0412F4DA88866
:10C0B00018B1401EA880BDE8F081FFF753FFFFF7DD
:10C0C000B5F92B4890F827000028F4D12748294FCC
:10C0D00014300024D0F8006026FA04F0C00701D024
:10C0E000092106E004EBC40007EB4000007B20F0D0
:10C0F00001012046FFF744FA641CE4B2122CEBD392
:10C100002878122600EBC00007EB40041A4F14F801
:10C110000C1F17F81000814214D010212046FEF7A2
:10C120000FFC2074000A60742878217800EBC002AC
:10C13000002307F812101149324606FB0010214671
:10C14000FFF752FA2878401CC1B20020297012294A
:10C1500000D328706978491CC9B269706429AAD3D0
:10C160006870BDE8F04105F04FB90000100B0020E9
:10C17000A0440020E4350020343700208945002009
:10C1800000210D4A0CE0834206D101EB410000EB97
:10C19000C10002EB00107047491CC9B2022908D245
:10C1A00001EB410303EBC10302EB03131B78FF2BED
:10C1B000E9D10020704700003C1300202DE9F04732
:10C1C0000026DFF80C81DFF80C91DFF80CA1434C5E
:10C1D0004FF400474FF6FF75012804D0022817D00E
:10C1E000032854D070E0EB21822008F0DDFBA0F59D
:10C1F0000041E080B94202D2281AE08002E0A84261
:10C2000000D3E680E088FCF79DFA42464B4652E0B8
:10C21000E321B22008F0C8FBE080B84204D301213A
:10C220006180281AE08000E0668080B2FCF78AFA1C
:10C2300042464B46FCF780F900225346FCF7EEF9E4
:10C24000FCF7B4FAFCF79FFA4FF03332244BFCF7BB
:10C2500073F9244A244BFCF7E1F9FCF7A7FAA06133
:10C260006088012830D11D484FF4FA61143003F082
:10C270000FFD012807D11DA005F01CFD1748002166
:10C28000143003F005FDA06980F000401BE0E321BD
:10C29000B42008F089FBA0F50041E080B94202D249
:10C2A000281AE08002E0A84200D3E680E088FCF78C
:10C2B00049FA4246164BFCF73FF900225346FCF779
:10C2C000ADF9FCF773FAA061A069BDE8F087000042
:10C2D000FCA9F1D24D622040E0FFEF407C0000203D
:10C2E000F308CA40F6285C8FC2F513404E656761BB
:10C2F0007469766520766F6C746167652073616D13
:10C30000706C65206661756C74210D0A0000000078
:10C310004D621040C079032801D0002070470120F1
:10C3200070478079012802D0002800D00020704793
:10C330000148406870470000380C00202DE9F84F94
:10C3400005462D4800248DF80040006F016B88479A
:10C35000DFF8A89003462A4999F8008001260220B8
:10C360000322284F6FF0814CDFF89CA02944AC4495
:10C37000B8F1000F0AD0B8F1010F1ED0234BB8F16D
:10C38000020F1FD0B8F1030F2CD120E0DFF880801E
:10C39000B94203D298F80F10022910D31D4929443D
:10C3A0001D4DA94203D298F80F10022911D2D4458D
:10C3B00015D3BBB188F80F4014E0B94212D28DF802
:10C3C000006011E0994204D3D44508D30AE09942B1
:10C3D00002D28DF8002007E010498C4502D28DF87A
:10C3E000000001E08DF8004069460D48FFF7FAFAB9
:10C3F00089F80000BDE8F88FC80600200C0B00206B
:10C40000F528DCC3285C4F04FFFF3F00F5289C03A0
:10C4100060230020CCCCCCC0CCCC8C00FFFF5F00D4
:10C42000AC2300202DE9F04114480468144821464B
:10C43000FBF765FF054613492046FBF766FF2946D3
:10C44000FBF795FFFCF79FF90F4D88460446002245
:10C450002B46FCF76EF806460F4620464146002262
:10C460002B46FCF769F832463B46FCF7D7F8FCF759
:10C470009DF906490860BDE8F0810000380C0020F5
:10C480000000A0403333A3400000244058000020A7
:10C490000148B0F908007047380C002040790128A5
:10C4A00002D0002800D000207047000001484078EA
:10C4B000704700002000002070B53F4E7088401C7F
:10C4C00080B270800A286FD33C4C00257580B4F888
:10C4D00040004FF4FA71884224D2401C80B2A4F884
:10C4E000400088421ED12572607F032801D00228B7
:10C4F00018D125770120607784F82250A5716574E2
:10C50000A4F8405084F824502C4884F8255084F82E
:10C5100027503838E5730179012901D1856105710A
:10C5200000F04EFB94F8241025480029017802D031
:10C5300021F0030101E041F00301017094F825109E
:10C540000029017802D021F00C0101E041F00C013A
:10C550000170B4F8541031B1491E0904090CA4F853
:10C56000541000D1E5733188491C89B231806429A7
:10C570001AD3358094F8291079B1491E11F0FF01C2
:10C5800084F8291009D1E178012906D1E57094F8E1
:10C59000281011B1491E84F82810217A0029017849
:10C5A00003D021F01001017070BD41F01001017045
:10C5B000BDE8704000F004BBB00B0020A044002098
:10C5C0002C0B002000F00F00092801D937307047EC
:10C5D000303070470009092801D9373070473030B2
:10C5E0007047704770470000074A30B45170064BDF
:10C5F0000022083303E0845C9C54521CD2B28A426D
:10C60000F9D330BC02F0B4BDF00B0020064A10B5DF
:10C61000054B00215278083303E05C5C4454491C0C
:10C62000C9B29142F9D310BDF00B002070B50C4691
:10C63000054602F053FE024621462846BDE87040FA
:10C6400004F07CBA074A30B45170064B002208331C
:10C6500003E0845C9C54521CD2B28A42F9D330BCB1
:10C6600002F0DEBDF00B002002F08EBE10B504F02B
:10C67000E1FA02490020087010BD0000F00B002014
:10C680000148407870470000F00B00207FB50D494D
:10C690006B464A6800928A788DF80420002104E0F5
:10C6A000445C5D18491C6C71C9B29142F8D30649CB
:10C6B00001208DF80D0048709DE80F0003F07EFB0F
:10C6C0007FBD0000F00B0020A044002001498870CD
:10C6D00070470000F00B0020024A40F2B471516034
:10C6E00070470000F00B00207047000070B50D4649
:10C6F000064602F0F3FD0A4C217800290ED17F2175
:10C7000001704670857003250020FFF7E5FF03F0F8
:10C7100071F8284602F008FE0120207070BD00006C
:10C72000F00B002070B50E46044602F0D7FD0C4D0C
:10C730002978002913D1002C11D0002203E0B15C2C
:10C740008154521C92B2A242F9D30020FFF7C4FFD9
:10C7500003F050F8204602F0E7FD0120287070BD7C
:10C76000F00B002002F0CABC0078704700787047D8
:10C77000FEE700002DE9F0410427044600F17006B1
:10C780004FF001085FF0000594F89100062876D27A
:10C79000DFE800F0031975424E5C94F8540003285A
:10C7A0006DD330460AF00CF9002868D104F19401E9
:10C7B00030460AF021F970B384F8918084F89050E3
:10C7C00084F8AC5050E0D4F808C094F89930207840
:10C7D00004F19A02D4F89410E04784F8980094F891
:10C7E0009010491C84F89010FF280CD0022084F887
:10C7F000910084F8AC5094F854008128C4D10320EF
:10C8000084F85400C0E794F84400C9B2814236D39A
:10C8100084F891702CE027E094F8900094F844108C
:10C82000884202D384F891701EE084F891801BE066
:10C8300084F89150D4F8A82022B10121D4F8A400A2
:10C84000904711E0226D002AF7D10DE084F8915055
:10C85000D4F8A81029B10220D4F8A42006F0E8FFEB
:10C8600002E0216D0029F6D194F8910004288BD1C3
:10C870002278BDE8F0410421012006F0D9BFBDE8CF
:10C88000F081000030B500201D4902460446012514
:10C89000C1F8985105235B1E1B041B0CFBD14006FD
:10C8A000D1F81C31000E0BB140F00100C1F89841E5
:10C8B00005235B1E1B041B0CFBD1521CD2B2082AA1
:10C8C000E6D3C1F898410522521E1204120CFBD186
:10C8D000C1F89C410522521E1204120CFBD1C1F872
:10C8E00098510522521E1204120CFBD1C1F8984136
:10C8F0000522521E1204120CFBD1C1F89C5130BD0E
:10C90000008021420F480122C0F89C210521491EC8
:10C910000904090CFBD1C0F898210521491E09041E
:10C92000090CFBD10022C0F89C210521491E0904F5
:10C93000090CFBD1C0F898210520401E0004000C12
:10C94000FBD17047008021420C480021C0F89C11A7
:10C950000521491E0904090CFBD10122C0F89821C8
:10C960000521491E0904090CFBD1C0F89C210520B2
:10C97000401E0004000CFBD17047000000802142E3
:10C9800030B516490024C1F8984122460123050616
:10C9900002D5C1F89C3101E0C1F89C41C1F8983141
:10C9A00005256D1E2D042D0CFBD1C1F898410525E0
:10C9B0006D1E2D042D0CFBD14006521C000ED2B270
:10C9C000082AE4D3C1F89C31C1F898310520401EF3
:10C9D0000004000CFBD1C1F8984130BD0080214219
:10C9E0002DE9F041084D4FF400642C6007F0E9FE9A
:10C9F0002F1F66103E6007F0E4FE2E6007F0E1FE98
:10CA00003C60BDE8F0810000140C014070B5084C9A
:10CA10004FF40060206007F0D4FE2515256007F074
:10CA2000D0FE201D0560BDE8704007F0CABE0000C2
:10CA3000100C01402DE9F047144F0024DFF84C8022
:10CA400082462546A8F108083E1507F1040960064C
:10CA5000040E3E6007F0B5FED8F80000000501D5D1
:10CA6000641CE4B2C9F8006007F0ABFE6D1CEDB2C7
:10CA7000082DECD3BAF1000F04D0FFF7B1FF204628
:10CA8000BDE8F087FFF7C2FFF9E70000100C014096
:10CA90002DE9F047DFF84890054600244FF4806701
:10CAA0004FF40068A9F104062806404601D530601D
:10CAB00001E0C9F8000007F084FE376007F081FE4E
:10CAC000C9F80070072C01D1C6F800806806050E71
:10CAD00007F077FE641CE4B2082CE5D3BDE8F087CC
:10CAE000140C014070B509484FF400650560041549
:10CAF000046007F066FE054E361D356007F061FEE6
:10CB00003460BDE8704007F05CBE0000100C0140CE
:10CB100070B507484FF400640460054D00152D1FE3
:10CB2000286007F04EFE2C60BDE8704007F049BE5B
:10CB3000140C014070B50C4C4FF40060206007F0FD
:10CB400040FE2515256007F03CFE074808380068C0
:10CB5000000501D5012400E000240348001D056004
:10CB600007F02FFE204670BD100C0140064A0188D8
:10CB70000020B2F835308B4204D3B2F8432014328F
:10CB80008A4200D803207047C806002070B50B4DBC
:10CB900006680024B5F83900FBF7CFFD3146FBF7F6
:10CBA00021FE01D2012407E0E88FFBF7C6FD3146E4
:10CBB000FBF722FE00D20224204670BDC8060020EA
:10CBC0007047000003497F20086003490020087077
:10CBD00070470000002C0040740100200C48C1691F
:10CBE00041F40061C1610B4940F2FF30086009481F
:10CBF0007F21001F0160016841F0800101604FF05A
:10CC0000E020002180F800140121C0F800117047D5
:10CC100000100240042C00402DE9FE4342F20F7840
:10CC2000224CADF80080694621480194FCF704F9D4
:10CC300040F6C315ADF8005069461D480194FCF755
:10CC4000FBF841F64B561B4FADF80060694618489B
:10CC50000197FCF7F1F842F22730ADF80000694681
:10CC600013480194FCF7E8F840F2E730ADF8000013
:10CC70001148019069460E48FCF7DEF8ADF80060F7
:10CC800069460B480194FCF7D7F8ADF800506946A7
:10CC900007480197FCF7D0F8ADF8008069460448D2
:10CCA0000194FCF7C9F8BDE8FE83000025D8000810
:10CCB000C434002035D90008F9EA00082DE9F04114
:10CCC0000024154E5FF0FF0704EB440000EBC400A6
:10CCD00006EB00100546B021FBF78EFA641CE4B2A7
:10CCE0002F70022CF0D30D4C206818B90C4806F0B8
:10CCF00019FE206006F075FE18B90A21206806F0BA
:10CD000069FE0849012006F0ABFDBDE8F041064987
:10CD1000022006F0A5BD00003C130020D00000203A
:10CD2000F16C0108D9A00008CDA0000810B5482179
:10CD30000F48FBF761FA0E4828214830FBF75CFAF0
:10CD40000C4801F06DFC010004D009481422483061
:10CD5000FBF739FA0748203001F062FC010006D0E9
:10CD600003481422BDE810405C30FBF72CBA10BD1C
:10CD7000440F00208472010810B5284800F0B3F970
:10CD80002648083000F0AFF92448103000F0ABF925
:10CD90002248183000F0A7F92048203000F0A3F90D
:10CDA0001E48283000F09FF91C48303000F09BF9F5
:10CDB0001A48383000F097F91848403000F093F9DD
:10CDC0001648483000F08FF91448503000F08BF9C5
:10CDD0001248583000F087F91048603000F083F9AD
:10CDE0000E48683000F07FF90C48703000F07BF995
:10CDF0000A48783000F077F90848803000F073F97D
:10CE00000648883000F06FF90448903000F06BF964
:10CE10000248BDE81040983000F065B95C09002078
:10CE200070B51A4C1B491C486278194D0978006985
:10CE3000052A18D2DFE802F003091E101800E87B6B
:10CE400008B103200EE001200CE0072902D0804742
:10CE50000228F8D1022005E00729F2D080470228F5
:10CE6000EFD00420607070BD0729F3D080470228FE
:10CE7000F7D1EFE700F022FB00266E606E7301F041
:10CE80004BFBA8606670267070BD0000340800205F
:10CE90002824002060230020580000202DE9F041C4
:10CEA00016460D46FFF76CF9040007D035B12EB1D8
:10CEB000287818B194F85400012802D00020BDE869
:10CEC000F08195F82000C00702D0A86A0028F6D0AB
:10CED00095F8250084F8450010B9322084F8450003
:10CEE000C0B200EB4000C00004F036FFC4F88C0074
:10CEF000011EE4D094F84530182204F1700009F0C6
:10CF00006FFD95F82000C0070FD194F8450000018F
:10CF100004F022FFC4F88800011E2ED094F845309A
:10CF2000102204F1580009F05BFD286A206404F126
:10CF3000200007462021FBF75FF91F2229463846CB
:10CF4000FBF741F9E86AF862A86AB86295F824002C
:10CF500087F82400286B38630B4830610B48F06079
:10CF60000B48B0600B4870600B4830600B48706134
:10CF7000022084F854000120A1E754F88C0F04F03B
:10CF8000BDFE0020206099E7C14D0108314C010829
:10CF9000A34C0108B34C0108274D01089D4B010823
:10CFA00038B5044601213C2001F0D0F901210846A2
:10CFB00001F0CCF901211248FEF72EFEA468B4B1AD
:10CFC0002088ADF8000010208DF8030002208DF8B5
:10CFD000020069466068FEF7CDFD207A01280AD07C
:10CFE000002803D121886068FEF749FE38BD05A0FE
:10CFF00004F060FE38BD21886068FEF742FE38BD4F
:10D00000000230004F5053206973204E554C4C0D98
:10D010000A00000010B5044800F0CBF8BDE810404D
:10D02000024800F0E6B80000C4090020CC09002046
:10D0300010B5044800F0BDF8BDE81040024800F00B
:10D04000D8B80000CC090020C409002010B504485D
:10D0500000F0AFF8BDE81040024800F0AAB80000A8
:10D06000C4090020CC09002010B5054800F0A1F843
:10D07000044800F09EF8BDE8104003A004F01ABE7A
:10D08000C4090020CC090020414320C8ABB5CD0025
:10D0900010B5054800F0ADF8044800F0AAF8BDE866
:10D0A000104003A004F006BEC4090020CC090020F3
:10D0B000414320C8ABB8DF0038B504460121102039
:10D0C00001F044F9A06800280CD00188ADF80010E8
:10D0D00004218DF8031003218DF802104068694681
:10D0E000FEF748FD38BD00680168002900D00847F8
:10D0F0007047000038B5044601213C2001F026F9B4
:10D10000A468B4B12088ADF8000010208DF80300A9
:10D1100002208DF8020069466068FEF72BFD207A38
:10D1200001280AD0002803D121886068FEF7A7FDF6
:10D1300038BD04A004F0BEFD38BD21886068FEF74C
:10D14000A0FD38BD4F5053206973204E554C4C0DF7
:10D150000A00000038B504460121042001F0F6F869
:10D16000A468002C15D02088ADF8000010208DF8A0
:10D17000030003208DF8020069466068FEF7FAFCA0
:10D18000207A012806D0002803D121886068FEF7A4
:10D1900076FD38BD21886068FEF773FD38BD10B597
:10D1A000044601884068FEF76AFD002020720120D5
:10D1B00010BD10B500684168496819B1806888479A
:10D1C000012010BD002010BD01884068FEF750BD51
:10D1D00000684168896809B1806808470320704782
:10D1E00010B5044601884068FEF74BFD012020720F
:10D1F00010BD10B500684168096819B1806888479A
:10D20000012010BD002010BD38B5044601211020BA
:10D2100001F09CF8A06800280CD00188ADF800103F
:10D2200048218DF8031003218DF8021040686946EB
:10D23000FEF7A0FC38BD00000A4810B5C088094AB6
:10D240000221203A04F094FC06480749303800696E
:10D25000FBF75BF84FF07A51FAF7FFFF034948609C
:10D2600010BD00005000002000003041380C0020AC
:10D2700030B504465FF0000014F8015B8D4203D125
:10D28000012A08D0521ED2B2002B04D0401C5B1ED3
:10D2900080B29BB2F0E730BD124810B5C07E124C90
:10D2A000012813D04FF47A700146A0600E4802F0B6
:10D2B000EFFC012814D1606810F0010F00F10100AB
:10D2C00060600A4804D0FFF774FF03E06420EBE7D6
:10D2D000FFF78FFFBDE810400021034802F0D8BCE3
:10D2E00010BD0000780C00200000002094090020F0
:10D2F000094B9A7A72B1094841780B44DB7A03B141
:10D300008380491CC9B241708A4201D80021417012
:10D3100000797047002070472C0B00208C050020FE
:10D3200003A004F0C7FC04F05DFC00F003FC000067
:10D33000476F20746F20536C6565700D0A00000004
:10D34000FEE770474FF4A06000F03EB800F01F0207
:10D35000012191404009800000F1E020C0F88011D7
:10D360007047000070B50F23C47801780122F4B132
:10D37000144C2468457804F4E064C4F5E064240A9D
:10D38000C4F10406E3408478B5401C402C4301F10D
:10D39000E021230181F80034007800F01F018A4069
:10D3A0004009800000F1E020C0F8002170BD01F0CC
:10D3B0001F0082404809800000F1E020C0F8802171
:10D3C00070BD00000CED00E002490843024908600E
:10D3D000704700000000FA050CED00E0024A114021
:10D3E000014302480160704780FFFF1F08ED00E025
:10D3F00004480168044A01F4E06111430160BFF38D
:10D400004F8FFEE70CED00E00400FA0504480168C8
:10D41000044A01F4E06111430160BFF34F8FFEE75E
:10D420000CED00E00400FA054FF400720021014801
:10D4300003F0DEBD0045002010B50948FFF7D9FE16
:10D440000120FDF70CFF0748FFF7D3FE4FF4FA70F9
:10D45000FDF705FFBDE810400248FFF7AABE000037
:10D46000C4090020CC09002010B5FFF7E1FD4FF4FE
:10D47000FA70FDF7F4FEFFF7E9FD0449002048715A
:10D48000BDE8104002A004F015BC00008823002075
:10D490004F50454E5F313256506F7765725265611D
:10D4A0006C790D0A0000000002490120C871024891
:10D4B000FFF79FBE882300206C090020024901204D
:10D4C000C8710248FFF795BE882300206C09002030
:10D4D0000249012088710248FFF78BBE8823002093
:10D4E0005C090020007808B10020704701207047D7
:10D4F000014908627047000000000E4202490A68B4
:10D5000042EA8000086070470070004000B50B30B0
:10D51000034609F0D1FA18680D49C0F309300A2210
:10D5200021F83C0F1868C0F3093090FBF2F081F845
:10D5300030005868800C48805868800C4881186812
:10D540001A79800D62F38D208881012000BD0000D2
:10D55000C806002070B50B30044609F0ADFA0A4D3C
:10D560006068296FC0F3C260496A8847296F2068E4
:10D57000C96AC0F3026088472068C0F3407085F82C
:10D580005900012070BD0000C806002000B50B3016
:10D59000034609F091FA98880A2280B290FBF2F0D3
:10D5A0000A49A1F866005868000C90FBF2F0A1F857
:10D5B00068005868000C90FBF2F040F4805021F8AD
:10D5C0004A0F1868000C4871012000BDC8060020F1
:10D5D00000B50B30034609F06FFA98880B49000A32
:10D5E0000A3081F86A005868000E0A3081F86B0032
:10D5F0009888000A01F8500F5868000E8870586823
:10D60000000C48701879C870012000BDC8060020C1
:10D6100010B50446FBF7FCFC0B34204609F04CFA2D
:10D6200060684FF6FF71C0F3892000EB800001EACB
:10D630004000044921F8410F6068000D4880012036
:10D6400010BD0000C806002000B500F10B0318460D
:10D6500009F032FA034819680163596841630120EF
:10D6600000BD0000B022002000B500F10B031846F9
:10D6700009F022FA0348196881635968C1630120DF
:10D6800000BD0000B022002000B500F10B031846D9
:10D6900009F012FA034819680164596841640120CD
:10D6A00000BD0000B022002070B500F10B04204640
:10D6B00009F002FA2068154DC0F340400A2185F8B0
:10D6C00045006068000C90FBF1F0A5F83300A088DD
:10D6D000C0F38D002880207868712088000A85F8C2
:10D6E0003B00A088C0F38D00A5F83900296F2068A1
:10D6F000C968C0F3004088472068C0F3004085F83F
:10D700005A002068800C2881012070BDC8060020C6
:10D7100000B50B30034609F0CFF998880549C0F3EE
:10D720008D00C8805868000DC0F57A60A1F83500FA
:10D73000012000BDC806002000B50B30034609F0EB
:10D74000BBF918680549C0F38930A1F837000448CF
:10D75000196881655968C165012000BDC8060020AF
:10D76000B02200202DE9F0472348244F0122868A69
:10D7700007F2FA2500206F602870334620213846D2
:10D78000FFF776FD687004461DA0696804F092FA00
:10D79000B4422AD0022025E0385D202828D02978FC
:10D7A000A14605EB810107EB09008860334642463C
:10D7B00020211248FFF75CFD2A7815490446A0EBAA
:10D7C00009005054297805EB8100826811A004F00B
:10D7D00071FA2878401CC0B22870042805D208F1DC
:10D7E0000100C0B28046B442D6D10120BDE8F08726
:10D7F000641CA4B2F7E7000088010020921D0020FD
:10D80000696E6F757420636D643A25730A000000B9
:10D81000A4200020256420706172616D3A25730A8E
:10D82000000000002DE9FC4100203E4C00904FF428
:10D830004571019021606160207260720820A072C1
:10D84000E84600F093FF054600F0A4FF019A65F357
:10D85000196265F39B6260F31D72334D60F39F7232
:10D860000192287A10B3002060F311420192E87906
:10D87000F0B1002060F393420192FDF79FFB009905
:10D8800060F38B210091FDF78FF8DDE9006760F30D
:10D89000155726480197C068FAF761FF80B20A2140
:10D8A000B0FBF1F0C82805D2002004E00120DBE73E
:10D8B0000120DFE7C83860F35D561D48CDE90067F9
:10D8C000006FB0F9020090FBF1F000F5FA7060F320
:10D8D00014360096FDF7CCF9009960F3DF7124202F
:10D8E0000091FDF763FFDDE9001260F39E71687A35
:10D8F00060F34F32CDE90012687808B9A87800B11A
:10D90000012060F3D7524046019209F0DCF80098FC
:10D9100044F80B0F01986060024806F08BF8BDE8F0
:10D92000FC8100001823002088230020380C0020F0
:10D93000C80600202DE9FC410024374E00944FF426
:10D940007A70019430607060347274720820B07222
:10D95000E8462820FDF72AFF58B92620FDF726FFC4
:10D9600038B91C20FDF722FF18B92120FDF71EFF52
:10D9700008B1012200E00022019962F38E31274AAA
:10D98000019113781B1F022B05D8D27C1AB10122FA
:10D9900062F3CF310191FDF707F8022803D0FDF7BC
:10D9A00003F8032803D1019864F3CF3001901C4F92
:10D9B00078688047DDE90054283060F31F64194817
:10D9C00019490078283060F3174401943868FAF751
:10D9D0009CFCFAF7C4FE42F21071884200D9084656
:10D9E00060F30D041148807A60F30B25CDE90054F3
:10D9F000FFF77EFC009960F307014046009109F0B3
:10DA000062F8009846F80B0F01987060024806F023
:10DA100011F8BDE8FC8100001823002060230020DD
:10DA2000580000208823002000007A442C0B00209E
:10DA30007CB50021144B009140F23F4001911860E9
:10DA400058601972114C597208209872A278684671
:10DA5000521CD2B2A270102A00D3A17000990125E5
:10DA6000A47865F3CF3164F30B21641C64F30701E0
:10DA7000009109F028F8009843F80B0F01985860BE
:10DA8000014805F0D7FF7CBD182300208C0500203D
:10DA90001FB5104A012010720020A2F84000009B20
:10DAA0009DF80410A3F5E0636846343B09D0AB2B26
:10DAB00006D140F2DF73A2F84E30401DFEF794FD10
:10DAC0001FBD40F23473A2F84E30401DFEF7BAFD80
:10DAD0001FBD0000A044002000B50B30034608F035
:10DAE000EBFF0648196801615968416104495868AB
:10DAF000096F000C0880012000BD0000B02200204A
:10DB0000C806002070B50B30044608F0D5FF074D5D
:10DB10002068296FC0F30360C9698847296F60686E
:10DB20004969800F8847012070BD0000C8060020A9
:10DB3000704700004FF0E020016921F0020101610F
:10DB40000220FFF703FC0320FFF700FC0420FFF78F
:10DB5000FDFB0520FFF7FAFB0620FFF7F7FB072088
:10DB6000FFF7F4FB0820FFF7F1FB0920FFF7EEFBBE
:10DB70000A20FFF7EBFB0B20FFF7E8FB0C20FFF779
:10DB8000E5FB0D20FFF7E2FB0E20FFF7DFFB0F2088
:10DB9000FFF7DCFB1020FFF7D9FB1120FFF7D6FBC6
:10DBA0001320FFF7D3FB1420FFF7D0FB1520FFF75E
:10DBB000CDFB1620FFF7CAFB1720FFF7C7FB182085
:10DBC000FFF7C4FB1920FFF7C1FB1A20FFF7BEFBCC
:10DBD0001B20FFF7BBFB1C20FFF7B8FB1D20FFF746
:10DBE000B5FB1E20FFF7B2FB1F20FFF7AFFB202085
:10DBF000FFF7ACFB2120FFF7A9FB2220FFF7A6FBD4
:10DC00002320FFF7A3FB2420FFF7A0FB2520FFF72D
:10DC10009DFB2620FFF79AFB2720FFF797FBFEF7D7
:10DC2000D1FF2820FFF792FB2920FFF78FFB2A2046
:10DC3000FFF78CFB3220FFF789FB3320FFF786FBD1
:10DC40003420FFF783FB3520FFF780FB3620FFF7FA
:10DC50007DFB3720FFF77AFB3820FFF777FB392071
:10DC6000FFF774FB3A20FFF771FB3B20FFF76EFBD9
:10DC70003C20FFF76BFB3D20FFF768FB3E20FFF7E2
:10DC800065FB3F20FFF762FB4020FFF75FFB412071
:10DC9000FFF75CFB4220FFF759FB4320FFF756FBE1
:10DCA0000020411E820002F1E022C2F88011401CD7
:10DCB0000828F7DB0120FFF721FCFEF783FF094866
:10DCC000FFF797FA0848C07B0028084802D0FFF702
:10DCD00090FA01E0FFF76DFA41F28830FDF7BFFAE4
:10DCE000FFF794FBF409002028240020EC09002011
:10DCF00070B56249624E634C4868634D401C486091
:10DD00000521B0FBF1F201FB120005287AD2DFE811
:10DD100000F0033347728F005CA003F0CBFF287A3A
:10DD200008B165A105E0306980475449083151F8D0
:10DD3000201064A003F0BEFF206F016A88474F499E
:10DD40004C3151F8201066A003F0B4FF6A484B49EB
:10DD500094F86C200078143151F8201067A003F07B
:10DD6000A9FF94F8450008B16CA100E06FA173A071
:10DD7000BDE8704003F09EBFB4F84320B4F84110F2
:10DD800074A003F097FF7E48B0F81D20B0F81B1078
:10DD90007CA003F08FFF206FB0F9021084A0E7E7AA
:10DDA000B06880470446706880470146224686A0D6
:10DDB00003F080FF8C48FFF70BFA08B18BA400E05A
:10DDC0008DA48F48FFF704FA08B18BA100E087A16A
:10DDD00022468CA003F06EFF287A08B191A200E0E1
:10DDE00091A2E87908B191A100E091A1BDE870404D
:10DDF00090A003F05FBF974C6068FAF7C4FC02463E
:10DE00000B4600E038E094A003F054FFE068FAF716
:10DE1000BAFC02460B4695A003F04CFF3068FAF7B7
:10DE2000B2FCBDE8704002460B4696A003F042BF2C
:10DE3000206F016B88471149343151F8201097A0A9
:10DE400003F038FFA87808B19AA200E09BA2687896
:10DE500008B198A100E099A19AA003F02BFFFAF76E
:10DE600051FF28B99D48D0E900219DA003F022FF71
:10DE7000BDE8704000F04AB970BD00003C070020CA
:10DE800058000020C8060020882300200D0AA1AAFF
:10DE9000A1AAA1AAA1AAA1AAA1AAA1AAA1AAA1AA2A
:10DEA000A1AAA1AAA1AAA1AAA1AAA1AAA1AAA1AA1A
:10DEB000A1AAA1AA0D0A000041435F4368617267ED
:10DEC000696E67000D0A4443555F576F726B696E48
:10DED000674D6F6465203C25733E0D0A000000000D
:10DEE0005643555F576F726B696E674D6F6465205F
:10DEF0003C25733E0D0A00006023002043686172D8
:10DF000067696E675F5374616765203C25733E09DE
:10DF1000534F43203C25643E0D0A0000436F6E734F
:10DF200074616E74566F6C7461676500436F6E73D5
:10DF300074616E7443757272656E740043686172C9
:10DF400067696E675F4D6F646520203C25733E0DE9
:10DF50000A00000044656D616E645F766F6C7461E9
:10DF60006765203C25643E0944656D616E645F63AE
:10DF7000757272656E74203C25643E0D0A000000C7
:10DF8000FC0C00204F75747075745F766F6C746153
:10DF90006765203C25643E094F75747075745F6336
:10DFA000757272656E74203C25643E0D0A00000097
:10DFB0004368617267696E6743757272656E74203B
:10DFC0003C25643E0D0A000054656D703120202010
:10DFD000203C25643E092047554E5F54454D502056
:10DFE0003C25643E0D0A00009C09002044697363CF
:10DFF0006F6E6E65637400004F70656E0000000008
:10E00000A409002044435F52656C6179203C25736C
:10E010003E202041435F52656C6179203C25733E70
:10E020000D0A0000434300004343320043433100E4
:10E030004350000043502D4343312020203C2573A2
:10E040003E092043432D4343322020203C25733E8C
:10E050000D0A0000380C00204B4C33305F566F6CBB
:10E0600074203C25663E0D0A0000000053616D706F
:10E070006C5F766F6C74616765202020203C25669C
:10E080003E0D0A0043435F52206973202020202068
:10E0900020202020203C25663E0D0A004F42435F91
:10E0A00047756E436F6E6E6563742020203C257348
:10E0B0003E0D0A004E4F5F4C6F636B004C6F636BFD
:10E0C000000000004856494C203C25733E2048562D
:10E0D000494C5F32203C25733E0D0A002824002065
:10E0E000456E7465722046616C7365536C6565702E
:10E0F0002049646C6520636F756E74202564204D23
:10E1000041582069732025640D0A00002DE9F0476D
:10E11000DFF84880DFF848900025464618F80500EB
:10E12000B0B1FDF705FB3327B04600244FEA0906DE
:10E1300018F8052016F83410914205D106EBC400FA
:10E14000416808A003F0B6FD641CE4B2BC42EFD302
:10E150006D1CEDB2052DE0D3BDE8F0872C08002042
:10E16000C07501084572726F7220436F6465204963
:10E170006E466F2069732025732D25640D0A0000FB
:10E180002DE9F041264C207860B10026254D01286C
:10E190000DD0022827D003283FD0BDE8F04122A0AF
:10E1A00003F088BDFAF7AEFD80F0010014E008F03E
:10E1B0005BFC012798B1012813D002280DD11D481E
:10E1C00006721D48FEF7F5FFFFF72CFB4FF4FA70BF
:10E1D000FDF745F86F7302202070BDE8F0812770CD
:10E1E000FBE72670F9E76068401C6060A97B0129A5
:10E1F00005D0052803D303206660207003E00128C2
:10E2000001D1FBF747FBFEF70BFE287B0028E4D08B
:10E21000FFF754F96E606E73E3E7FFF781F80000D3
:10E22000340800202824002045525220536C656594
:10E23000700D0A00882300207C090020F0B52948D1
:10E24000807A00EB80004200B2F5AF7F43D32649CD
:10E25000264B00240878012703EBC0060546B6F8D4
:10E2600002C094450CD316E033F830C0944505D273
:10E2700003EBC00CBCF802C0944504D8401CC0B2EB
:10E280000528F1D301E0052800D30420CC708B7859
:10E29000EBB98F7016E033F830C094450CD814E019
:10E2A00033F830C0944505D203EBC00CBCF802C073
:10E2B000944503D8401EC0B20028F1D18C70CB78B1
:10E2C0002BB9CF70F3888B8001E0CC708C708B8879
:10E2D00013B15B1E8B80F0BD8542FCD0322AFAD987
:10E2E0000870F0BDCC350020900B0020AC77010801
:10E2F000034A516821F440410143516070470000D6
:10E3000000100240044A0029516901D0014300E095
:10E31000814351617047000000100240044A002907
:10E32000D16901D0014300E08143D1617047000011
:10E3300000100240044A0029116901D0014300E0A5
:10E34000814311617047000000100240044A002917
:10E35000916901D0014300E0814391617047000061
:10E36000001002400149086070470000400442422A
:10E37000F0B52A4A51682A4B11F00C014FF00F05F5
:10E3800003D0042901D0082901D0036026E0516898
:10E39000546805EA914104F480340D2901D0891CA8
:10E3A00000E00621BCB1D46A14F4803FD46A04F0C2
:10E3B0000F0404F101040AD0D66AD76AC6F3031623
:10E3C000761CB3FBF6F3C7F30327BF1C7B43B3FBF9
:10E3D000F4F34B43D9E7134B594301605168124C96
:10E3E00005EA1111635C0168D94041605368072553
:10E3F00005EA1323E35C21FA03F38360536805EA1B
:10E40000D323E35CD940C1605268032303EA92320C
:10E41000231F9A5CB1FBF2F10161F0BD00100240D4
:10E4200000127A0000093D00F80400200246002096
:10E4300053090949012B0BD0022B0BD0D1F8241022
:10E4400002F01F02012393400B4200D001207047CD
:10E450000968F5E7096AF3E700100240014908601E
:10E460007047000080044242014908607047000084
:10E470003C04424202490A6A02430A6270470000B1
:10E480000010024010B5084C44F22001A06B084275
:10E4900001D1400605D52F20FDF796F90020A06395
:10E4A00010BD012010BD0000FC0C002070B50D4611
:10E4B0000646002403E0305D02F0F4FB641CAC422D
:10E4C000F9DB70BD70B50D460646002403E0305DF3
:10E4D00002F0E8FB641CAC42F9DB0D2002F0E2FB29
:10E4E0000A2002F0DFFB002403E0305D01F0B6FCFF
:10E4F000641CAC42F9DB70BD0248018841F0100198
:10E5000001807047042800400248018821F0100172
:10E510000180704704280040034800880249091F11
:10E52000098840EA014070471C28004010B50121CD
:10E530004FF0C050FFF7F2FE4FF400742046FFF793
:10E5400099FF0120FFF790FF0120FEF7D1FFFAF7B6
:10E55000B8FC0120FFF782FF6120FFF767FF00286A
:10E56000FAD02046FFF786FF0120FFF77DFF00F07D
:10E5700023F800F019F849F63F4000F005F8BDE82F
:10E58000104000F011B8000000B50246FFF7B4FFDC
:10E590000449C2F303400880081D02805DF804EBC3
:10E5A000FFF7B2BF08280040024801888906FCD561
:10E5B00070470000042800400448018821F0080149
:10E5C000018001880907FCD570470000042800403D
:10E5D000114910B50120C1F89801FEF793F9902078
:10E5E000FEF7CEF90020FEF7CBF9FEF7ADF9FEF706
:10E5F00089F99120FEF7C4F9FEF744F9074C208011
:10E60000FEF740F96080FEF79FF96088218840EAB4
:10E6100001202080208810BD00802142840000203D
:10E6200010B510B3416801B38168F1B1037818499E
:10E63000002200BF02EB420404EBC20401EB04140D
:10E6400024789C4211D0521CD2B2022AF2D300226A
:10E6500002EB420303EBC20301EB03131B78FF2B16
:10E6600005D0521CD2B2022AF2D3002010BD02EB18
:10E67000420303EBC20201EB0214014620222046B2
:10E68000F9F7A1FD012084F85400024810BD0000F4
:10E690003C130020D4000020704772B6704762B669
:10E6A0007047000070B5FDF7BDFEFDF747FE002284
:10E6B000012804D0022804D0032802D002E001225D
:10E6C00000E002220A4900230C78A24202D08B61AA
:10E6D0000A7070BD4D78AA4201D18B6170BD8A6904
:10E6E000521C8A61022AF9D34C708870F5E7000049
:10E6F0002000002070B50D460446FFF70DFF21688D
:10E7000009B1616802E04119C4E90001814201D800
:10E71000012070BD002070BD00210160416001201A
:10E720007047000070B50F4D0224B5F8410028B1C4
:10E73000B5F8430010B10024204670BD0A483C21C2
:10E740000646FFF7D7FF0028F6D03046FFF7E4FF74
:10E75000B5F8410020B10A20FDF736F80124EBE7B7
:10E760000920F9E7C806002094340020084810B5B5
:10E77000C0780324012807D040B10420FDF716F823
:10E7800000B10224204610BD0124FBE70024F9E774
:10E7900088230020084810B500790324012807D0F9
:10E7A00040B10320FDF702F800B10224204610BD5D
:10E7B0000024FBE70124F9E7882300202DE9F0413C
:10E7C00042780378284E02EB032295B2284A378A12
:10E7D0000024264B92F82220AF4207D11B7A8B42AD
:10E7E0003CD1C2B30A46811C22482EE0778AAF4250
:10E7F00008D15B7A8B4231D16AB30A46811C1D482D
:10E80000133022E0F78BAF4208D1DB7B8B4225D15E
:10E810000AB30A46811C1748773016E0378CAF429E
:10E8200008D11B7C8B4219D1AAB10A46811C114820
:10E830007B300AE0768CAE4212D15B7C8B420DD1EC
:10E840004AB10A46811C0B487F30F9F7BCFC2846C8
:10E85000FCF712FD05E0FFE7332402E0132400E09B
:10E8600031242046BDE8F0810E780108FA770108CE
:10E87000A0440020453500202DE9FF4F8046604828
:10E8800000248DB0B0F842201F46A146042A03D2CE
:10E89000132011B0BDE8F08FB8F8013098F80010DF
:10E8A0005DBA71238DF8003098F800308DF8013092
:10E8B00098F801308DF8023098F8023004268DF86F
:10E8C00003304FF0050B4FF4017A012907D00329DB
:10E8D0005ED002297AD00179012974D03BE0B8F8E2
:10E8E000011083464DBA04211046FCF77BF918B19C
:10E8F000A5F50070033812D0BBF842000421FCF7E4
:10E9000071F908B155450AD0BBF842000521FCF762
:10E9100069F9010040F207202ED085422CD19BF8E6
:10E920002210584631B3A5F50075033D1BD0012DCB
:10E930000AD0042D0BD198F80300012802D83149E0
:10E94000887001E04FF001098DF8049005262D49EB
:10E9500001201C3988703E80324669460F98F9F7CD
:10E9600032FC204695E70121C1734FF4FA71ABF8F0
:10E970005410E9E7332441E0A5F50071033903D0D1
:10E98000554501D0854201D1132437E0312435E0CB
:10E99000B8F8011080464DBA04211046FCF722F960
:10E9A00030B35545F2D198F822000028E2D015483E
:10E9B0001C38817841B1002181701348007A8DF8AC
:10E9C000040011E002E016E0242417E08046042150
:10E9D0001046FCF707F958B15545D7D198F82200F1
:10E9E0000028C7D08DF804900526A7F800B0B3E73B
:10E9F0005545CBD1C8E70021017112243E80B0E714
:10EA0000A04400202C0B0020CC35002004494BF6FC
:10EA10005C200880091D4AF65520088070470000D8
:10EA2000B06C00400CB500212E48019100910268A5
:10EA300042F4803202604FF6FF72036803F4003341
:10EA40000093019B5B1C0193009B13B9019B9342B4
:10EA5000F3D10268920342D50121009122490A684C
:10EA600042F010020A600A6822F003020A600A6893
:10EA700042F002020A6041684160416841604168B9
:10EA800041F480614160C16A184A1140C162C16AA3
:10EA9000174A1143C162016841F080610160016859
:10EAA0000901FCD5416821F47C114160416841F4C1
:10EAB000E8114160016841F08071016001688901DD
:10EAC000FCD5416821F003014160416841F0020139
:10EAD00041604168C1F381010229FAD10CBD009166
:10EAE0000CBD0000001002400020024000F0FEFFBC
:10EAF00014080100FFF78ABF0A4810B500780728FC
:10EB000004D0094800698047022809D10748D0E9A4
:10EB100001100A30814203D2BDE81040FEF788BFE1
:10EB200010BD000060230020580000202824002091
:10EB300001490872012070479406002001490871BC
:10EB40000120704794060020032803D0042801D038
:10EB5000002070470149C8710120704794060020C9
:10EB6000012802D008B100207047024988710120B5
:10EB70007047000094060020024A002110440172F0
:10EB80007047000094230020012802D008B1002023
:10EB90007047024948710120704700009406002028
:10EBA00070B5FEF7DFFD002818D0124C0020124D82
:10EBB000124E608380B200EB400005EB800041689C
:10EBC0007068F9F724FB0028608B08D000EB400048
:10EBD00005EB8000806800B18047012070BD401CBB
:10EBE00080B260831328E5D305A003F063F800200A
:10EBF00070BD000088010020DC7201088C2000201C
:10EC0000416E20756E7265636F676E697A65642008
:10EC1000434D4420210A00001FB51E48FEF7D8FAD4
:10EC200000B101208DF800001B48FEF7D1FA00B1B9
:10EC300001208DF804001948FEF7CAFA00B101203E
:10EC40008DF808001648FEF7C3FA00B101208DF8D0
:10EC50000C0069461348FCF7C5FE00B10120124CB8
:10EC600001A9E0700F480C38FCF7BCFE00B1012090
:10EC700020710C4802A90C30FCF7B4FE00B1012051
:10EC80006070084803A91830FCF7ACFE00B1012001
:10EC9000A0701FBD9C090020A4090020DC090020F1
:10ECA000E4090020DC23002088230020F0B5CF22D7
:10ECB0000270002343700C7884700126C2700671C4
:10ECC0004F78477191F802C080F806C00223C271E4
:10ECD0000372CB7843720B7983720324C27204737C
:10ECE0004B79437304258273C5738B7903740526AE
:10ECF00042748674CB79C3740627027547750B7A04
:10ED000083754B7AC3754FF0070C027680F819C0F3
:10ED1000897A81761B20F0BD054951F8062F40F80D
:10ED2000022F4A6842600A890281897A817270479B
:10ED3000D0350020F0B5002382F8003003EBC30487
:10ED400000EB4404647834B144EA03251478660087
:10ED5000641C14708D535B1CDBB2122BEED3107845
:10ED600000281DD0002317E000200EE001EB400535
:10ED700031F810606C88F7B204F0FF0C674502D9D7
:10ED80006E8021F81040401CC0B21478E41A641E52
:10ED90008442EBDC5B1CDBB21078401E9842E3DC63
:10EDA000F0BD000010B5FAF7BFF888B1FCF71EF906
:10EDB00000280CD0FCF798F8002808D0084890F8F4
:10EDC0003800C00602D5FBF78BFB18B1012010BD3F
:10EDD00004A000E00EA002F06DFF002010BD0000B6
:10EDE000FC0C0020424D532054686520436861723A
:10EDF00067696E672050686173652053746F707324
:10EE00002041626E6F726D616C6C790A0D000000BA
:10EE1000434353204E6F204368617267696E6720D9
:10EE2000416C6C6F7765646E0D0000000C48816862
:10EE3000491C81604168491C416081684FF47A72C5
:10EE4000B1FBF2F302FB1311012902D1C168491C85
:10EE5000C1600178002901D10121017070470000D3
:10EE6000780100200C484FF47A710068B0FBF1F093
:10EE7000B0F1807F0ED220F07F414FF0E020491E9C
:10EE80004161064AF02182F8141D002181610721A9
:10EE900001617047FEE700000C0000200FE000E079
:10EEA00010B5FDF78FFEBDE810404FF41F72024908
:10EEB000024804F0EFBA00002015002000F001081D
:10EEC000124810B5016841F0010101604168104A23
:10EED0001140416001680F4A11400160016821F44E
:10EEE00080210160416821F4FE014160016821F048
:10EEF000A05101604FF47F0181600021C162FFF7E2
:10EF000091FD05494FF00060086010BD00100240FF
:10EF10000000FFF0FFFFF6FE08ED00E00C4810B522
:10EF200000880B4A0021243A02F022FE08483038BB
:10EF3000C068F9F728FC02460B4606480649F9F76F
:10EF40006DFBF9F733FCFCF769FD0449088110BD3E
:10EF5000500000209A99999999991340380C0020F3
:10EF600010B5084C0121204600F04BF8002807D0CE
:10EF700000F0A4FE2046BDE81040012100F034B8A6
:10EF800010BD0000000400407FB50C46054601217D
:10EF90000220FFF7C3F9ADF800400020ADF804509F
:10EFA000104CADF80600ADF802006946204600F0AE
:10EFB0003FF801221146204600F02FF81D208DF861
:10EFC0000C0001218DF80D1003208DF80E008DF836
:10EFD0000F1003A8FEF7C6F90121204600F007F83C
:10EFE0007FBD000000040040C94301827047002932
:10EFF000018802D041F0010101E021F0010101800E
:10F00000704702460020138A92890B4202EA0102ED
:10F0100002D0002A00D001207047002A828901D046
:10F020000A4300E08A43828170478185704700006F
:10F0300030B502881B4B1C4C98420DD0A0420BD01F
:10F04000B0F1804F08D0194DA84205D0184DA84204
:10F0500002D0184DA84203D122F070054A882A43F5
:10F06000154DA84206D0154DA84203D022F4407594
:10F07000CA882A4302808A8882850A880285984243
:10F080000AD0A04208D00E4A904205D00D4A9042C4
:10F0900002D00D4A904201D1097A01860121818274
:10F0A00030BD0000002C014000340140000400404D
:10F0B00000080040000C0040001000400014004018
:10F0C0000040014000440140004801400A4800213E
:10F0D000428D4AB10722C273027B521CD2B2027324
:10F0E000102A00D1017370470177C173C172017694
:10F0F0004174808CFDF79ABA500B002070B51B4C00
:10F100000125002025756076E07B01280AD1607A10
:10F11000102807D1FDF765FAE07B012802D1607A5B
:10F12000102807D0207908B1E07818B1A07801281C
:10F1300006D007E096202086E5760220A07001E048
:10F14000607930B1607A20B1E07B042803D1E08B94
:10F1500008B900F0F3FAE07A012806D1E07B06282E
:10F1600003D1BDE8704000F0E9BA70BD500B00203B
:10F170002DE9F041274CA078012849D0264F387955
:10F18000012802D1E07A012842D0FDF779FA2085E2
:10F1900020483830FDF73AFA1E4E002538363078D0
:10F1A00000F0F001A173E584A18CA7F842103D7135
:10F1B000A178012700F00F00022901D100B9A77042
:10F1C000E07A012801D100F0B9FAA07B00281FD114
:10F1D0003078124B00F00F01A184012009E000BF3C
:10F1E000E28C16F800C003F802C0521C401CE284F6
:10F1F000C0B28842F4D900F06BF938B1E7742946FF
:10F200006174A08CBDE8F041FDF710BA0921F7E761
:10F21000BDE8F081500B0020A04400209C38002065
:10F2200070B5194C0026A07801281CD00125657501
:10F23000FDF726FA208504F13800FDF7E7F904F11F
:10F240003800A1780078022900F00F0001D100B940
:10F25000A570E07A012801D100F070FA0B486677BA
:10F260006570057170BD607F401CC0B26077022878
:10F27000F8D301F02BFC00F035F866770448A6704F
:10F28000E673067070BD0000500B0020A044002003
:10F29000F00B002010B5104C207868B104F1380054
:10F2A00041782171807828B17F2800D97F20401CC7
:10F2B000C0B200E0012060712079E0706079A07137
:10F2C0000020207200F09CFA207A10B10320E07335
:10F2D00010BD0420FBE70000500B002000487047E1
:10F2E0009C38002007480021C1738170C172C1752C
:10F2F00001760175417541768176C1760177017499
:10F3000081757047500B002010B5064CA07AFDF7B0
:10F31000DDF904F13800FDF7B9F94620A085012098
:10F32000607610BD500B002070B5164C00260728E3
:10F33000E08301D8667201E0102060720125A5709B
:10F340002684E07D012805D00C206074FDF78EF93D
:10F35000A67070BD607A10B1102803D004E000F0F0
:10F36000B9FA01E000F06CFAE571A07AFDF7AEF9A8
:10F3700004483830FDF78AF9E5734620A0856576A4
:10F3800070BD0000500B002010B500F0D3FBBDE8AD
:10F39000104000F0D3B900000B48417B29B101298E
:10F3A0000FD002290FD100F0A7B9C18CA1F602013C
:10F3B00049428186408D072801D300F0A9B800F0AA
:10F3C0002DB900F079B97047500B002070B51F4D72
:10F3D000A5F138042978687801F00F0140EA01208E
:10F3E000A08440F60201608588420BD90D2161742A
:10F3F000FDF71CF90220207400F042FA002020746E
:10F40000E07370BD0828FCD300F062F8B8B1104B6F
:10F410000220E18C2A5C401C5A54628D491C521E09
:10F420006285C0B2E1840728F3D901252573A08C39
:10F43000FDF7D8F8E572BDE8704000F021BA092167
:10F440006174A08CBDE87040FDF7F0B8880B002017
:10F450009C38002070B50F4B0F4DA3F1380418787D
:10F4600000F00F01A184012006E0E28C1E5CAE5486
:10F47000521C401CE284C0B28842F6D900F028F841
:10F4800030B100216174A08CBDE87040FDF7CEB8AA
:10F490000921F7E7880B00209C3800200A480A4918
:10F4A0004FF000020078A1F1380110F0F0008873ED
:10F4B000CA84CA740549C87603D0102803D1FFF75F
:10F4C00085BFFFF7C7BF7047880B0020A04400200E
:10F4D0000E4A00201146937B098D43B1102B0ED0AC
:10F4E000202B0FD0302B09D1032907D305E0928CB4
:10F4F000002A03D0521C914200D3012070470829F2
:10F50000FCD3FAE7528D072AF9D2F3E7500B00201B
:10F51000F0B51E481E4E0121838E1E4C00F1380CA2
:10F52000072B1ED2C18601220EE000BFC58C1CF83D
:10F53000027067556D1CC584458D6D1E4585C58E51
:10F540006D1C521CC586D2B29A42EFD9428D0AB9BF
:10F5500086F8211041730822C27301760021C1840C
:10F56000F0BD0122C38C1CF80250521CE5545B1CF8
:10F57000C384438DD2B25B1E4385072AF2D9180497
:10F58000000CEDD186F82110F0BD0000500B0020DA
:10F59000A04400209C38002070B51F4C608E38B30A
:10F5A000607D002836D00025657504F13806257782
:10F5B000307810F0F000A0731CD010281AD020284A
:10F5C00028D1FFF785FFE8B13078217B00F00F00EC
:10F5D000884219D16573FFF7DFFE9620608601200F
:10F5E0002077607B002815D1BDE87040FFF76EBD25
:10F5F00003200AE00620607400F050F8BDE8704077
:10F60000FFF74CBF092000E004206074BDE87040A3
:10F6100000F044B870BD0000500B0020F0B51C484D
:10F6200001231C4D868E418D00F138048E4215D386
:10F63000CEB2012109E0C28C675CAF54521CC28477
:10F64000428D521E491C4285C9B2B142F3D9408D48
:10F65000002802D1104880F82130F0BDC386012176
:10F660000CE0C28C675CAF54521CC284428D521EA7
:10F670004285C28E521C491CC286C9B2B142F0D921
:10F68000022141730821C17303760021C184F0BDBA
:10F69000500B00209C380020A044002010B5054CE1
:10F6A0000146A08CFCF7C2FF0020E073E0722076D8
:10F6B00010BD0000500B002030B50D48017E002920
:10F6C00014D10C4C00F13803C18E07290AD8C28C22
:10F6D0005D5CA554521CC284428D521E4285491C59
:10F6E000C186F1E7002141730721C17330BD0000DD
:10F6F000500B00209C38002070B50E48017E002978
:10F7000017D190F82A1000F138040B4D491C09E07C
:10F71000C28CE65CAE54521CC284428D521E42859D
:10F720005B1CC386C38E8B42F2D900214173072133
:10F73000C17370BD500B00209C38002070B52C4C5C
:10F7400000212246E37B0320527D092B1CD2DFE8F7
:10F7500003F0050C10141C202A383C00002A13D09A
:10F760006175BDE87040FFF799BEBDE8704000F0DC
:10F7700075BABDE8704000F037BA00F041F8207A61
:10F78000002801D10420E07370BDBDE8704000F096
:10F79000F3B9A179491EC9B2A1710129F4D8E07366
:10F7A0006079A07170BD227D01203AB12175A176EA
:10F7B0000721E17396216186207770BDE18D49B103
:10F7C00070BDBDE87040FFF7E7BE638E13B132B184
:10F7D00061750B206074BDE87040FFF75FBFFFF7F5
:10F7E000DBFD607B0028EBD1BDE87040FFF76EBC0D
:10F7F000500B002001490120C8757047500B0020B4
:10F800000E48017A29B1012915D0022915D100F03D
:10F810003DB90A4AC179383241F020011170018C9A
:10F82000A1F6020149428186C08B072801D300F06E
:10F8300079B800F0B7B800F001B97047500B00205C
:10F8400030B50D480D4CC18BC1F3032242F01003BB
:10F8500000F13802137051700221038CE55C55549D
:10F860005B1C0384C38B491C5B1EC9B2C38307297D
:10F87000F3D90821817230BD500B00209C38002044
:10F8800010B5134C142204F13801207C40F03000F4
:10F890000870002048708A7060840320A072CC2217
:10F8A0000A54401CC0B20728FAD90820A0720020D0
:10F8B000FCF712FFA07AFCF709FF05483830FCF787
:10F8C000E5FE0620E0734620E0850120A07610BD0D
:10F8D000500B0020F0B51149012001F13804CA8B0A
:10F8E000227003460E4F08E00D8C401CC0B27E5DB6
:10F8F000E6546D1C5B1C0D84DBB215469342F3D9B4
:10F900006A1C8A72072807D8CC222254401CC0B235
:10F910000728FAD908208872F0BD0000500B00209B
:10F920009C3800202DE9F0411C4C1D4904F138029F
:10F93000A38E072B1AD20125E58628460CE0268CDB
:10F940008F5D1754761C2684E68B761EE683E68E42
:10F95000761C401CE686C0B29842F0D9257200257C
:10F96000E575FCF7C1FE2584BDE8F0810120238CFC
:10F97000CD5C15545B1C2384E38B401C5B1EC0B222
:10F98000E3830728F3D90820A072FFF7BDFC042009
:10F99000E073BDE8F04100F0BBB80000500B002060
:10F9A0009C3800202DE9F041224C234B04F1380112
:10F9B000A28EE58B4FF00100AA4220D3EDB20122C6
:10F9C0000BE0268C401CC0B29F5D8F54761C2684B1
:10F9D000E68B761E521CE683D2B2AA42F1D9A572FA
:10F9E000CC2202E00A54401CC0B20728FAD90820F1
:10F9F000A072FFF789FC0420E073BDE8F081E08687
:10FA000001200CE0258C5E5D0E546D1C2584E58B79
:10FA10006D1EE583E58E6D1C401CE586C0B29042EC
:10FA2000F0D9022020720025E575FCF75DFE2584E3
:10FA3000E3E70000500B00209C38002070B5114C0B
:10FA4000E07D01281CD1104A04F13803E08E07281C
:10FA50000AD8218C555C1D54491C2184E18B491E18
:10FA6000E183401CE086F1E70820A072FFF74CFC20
:10FA7000002020720420E073BDE8704000F048B818
:10FA800070BD0000500B00209C3800202DE9F04193
:10FA9000174CE07D012828D194F83600A17FC2B22E
:10FAA0000844C1B2A17204F13803124E0BE0258C58
:10FAB000521CD2B2775D1F546D1C2584E58B6D1EE0
:10FAC000E583401CE086E08E8842F0D3CC20072AF4
:10FAD00003D89854521CD2B2F9E70820A072FFF75D
:10FAE00013FC002020720420E073BDE8F0810000C8
:10FAF000500B00209C38002010B5FCF7B7FD0348E0
:10FB00000021C1738170C175017510BD500B0020BB
:10FB10000748C179491CC9B2C171102901D100211E
:10FB2000C1710179002902D0C178491EC1707047A6
:10FB3000500B00200F48417E012903D1818D09B16E
:10FB4000491E8185817E012903D1C18D09B1491EDC
:10FB5000C185C17E012903D1018E09B1491E0186EB
:10FB6000017F012904D1418E002901D0491E41861F
:10FB700070470000500B002070B51A4C0126A08D74
:10FB8000D0B1207DA17D084326D00025657625755E
:10FB9000E08B98B1207908B1E078A8B16079B0B174
:10FBA000012814D002281AD016D9A079A0F101009A
:10FBB000A0714FF0050013E0304600E02846607465
:10FBC000BDE87040FFF798BF2570022008E0FFF7FE
:10FBD00017FE207A08B1A67570BDA57570BD03200B
:10FBE000E07370BD500B002070B51B4C208EB0B17F
:10FBF000607D00282FD0002004F13801607509785D
:10FC000001F0F002A273302A25D1E07601F00F0551
:10FC1000FFF75EFC28B1032D05D305200EE002207E
:10FC20000CE009200AE0022D07D0012D0BD0002D99
:10FC300011D1BDE87040FFF72DBB08206074BDE80E
:10FC40007040FFF759BF07206074FFF755FF9520FC
:10FC500020860120E07670BD500B00200B49012268
:10FC6000888D68B1087D002809D000200875487685
:10FC70004B7A43B1102B02D10A700220C87370472F
:10FC80004A74104600E04874FFF736BF500B00205E
:10FC9000094A29B192680068904204D8101A04E019
:10FCA0009168016003E0C0431044884201D3012001
:10FCB0007047002070470000780100200D4810B503
:10FCC000407B012815D03220FBF770FD002810D1B1
:10FCD0002A20FBF76BFD00280BD1074C2068018818
:10FCE0000648FFF7A2F920684068804720688068CE
:10FCF000206010BD28240020C434002000040040EF
:10FD000030B52C4C2078012852D12B490122C868EB
:10FD1000401CC8600A70002323700524B0FBF4F572
:10FD200004FB1504002C43D1002841D00A24B0FB69
:10FD3000F4F504FB15044A7004B98A701424B0FB6E
:10FD4000F4F504FB150404B9CA703224B0FBF4F5D1
:10FD500004FB150404B90A716424B0FBF4F504FB38
:10FD6000150404B94A714FF4FA74B0FBF4F504FBBE
:10FD7000150404B98A714FF47A74B0FBF4F504FBEE
:10FD8000150404B9CA7140F2DC54B0FBF4F504FB6D
:10FD9000150404B90A724FF4FA64B0FBF4F504FBDD
:10FDA000150404B94A7241F27072904200D3CB60DC
:10FDB00030BD000078010020101500200FB512485A
:10FDC00001880A2901D3002101800288009900EBF3
:10FDD0000212516002889DF8041000EB02121172A9
:10FDE00002889DF80D1000EB021251740188DDF8B5
:10FDF000052000EB011141F8092FDDF809204A60C8
:10FE00000188491C01800FBDA040002070B510483A
:10FE1000006800281BD1FAF7C5FD002817D00D4C4B
:10FE200021886088814212D000250A2800D365808D
:10FE3000608804EB0010001D0FC801F02AF9064885
:10FE40000121817080F82A506088401C608070BD5C
:10FE50004C0B0020A0400020A044002010B5044C12
:10FE60000146204601F0A8F820880006FCD510BD08
:10FE7000004C00402DE9F041384C40F225573946FE
:10FE8000204601F007F8364D002690B1204601F0DB
:10FE90008FF8C1B2A88AC82804D2324A1154401C33
:10FEA000A88200E0AE820A292FD03946204600F011
:10FEB000DAFF40F224473946204600F0EBFF38B124
:10FEC000AE82204601F074F83946204600F0CBFFA0
:10FED00040F227752946204600F0DCFF18B129467C
:10FEE000204600F0C0FF40F226652946204600F07B
:10FEF000D1FF18B12946204600F0B5FF0821204661
:10FF000000F0C1FF012805D00BE0FEF749FEAE82EC
:10FF1000BDE8F0810821204600F0A2FF204601F054
:10FF200047F80421204600F0AEFF012806D1042145
:10FF3000204600F095FF204601F03AF802212046C5
:10FF400000F0A1FF0128E3D10221204600F088FF44
:10FF50002046BDE8F04101F02BB80000004C004005
:10FF600088010020921D002070B5314D40F22556C9
:10FF70003146284600F08EFF2E4C98B1284601F0FD
:10FF800017F8C2B2208B0021C82804D22A4B1A5479
:10FF9000401C208300E02183E182E1703146284645
:10FFA00000F061FF40F224463146284600F072FF1F
:10FFB00040B1284600F0FCFF0120E07031462846A1
:10FFC00000F051FF40F2266631462C46284600F0EC
:10FFD00061FF18B13146204600F045FF0821204658
:10FFE00000F051FF012806D10821204600F038FF1B
:10FFF000204600F0DDFF0421204600F044FF0128E8
:020000040801F1
:1000000006D10421204600F02BFF204600F0D0FF4F
:100010000221204600F037FF012808D102212046A6
:1000200000F01EFF2046BDE8704000F0C1BF70BD6B
:1000300000500040880100205A1E002010B5094CD5
:10004000207F00280DD0E07F10280AD1A07F00F08B
:1000500037FA00202077BDE81040FF210248F8F76A
:10006000CBB810BDA04400209C38002010B5074C30
:10007000207F002808D0E07F112805D104F12B0053
:1000800000F0AAFA0020207710BD0000A044002054
:1000900010B50A4C207F00280FD0E07F14280CD127
:1000A000032104F12B0000F0E7FA00202077BDE8DF
:1000B0001040FF210248F8F79FB810BDA04400206F
:1000C0009C38002010B5064C207F002806D0E07F29
:1000D000192803D100F0F6F80020207710BD0000A9
:1000E000A044002010B5064C207F002806D0E07FF9
:1000F000222803D100F04CF90020207710BD000029
:10010000A044002070B5104C207F00280ED0E07F66
:1001100027280BD194F82B0000250C4A04F12B0161
:10012000022804D0012000F0E1FA257770BD0220FA
:1001300000F0DCFA05482577801F84F8215040F84C
:10014000065F456070BD0000A0440020B60B002093
:1001500010B50A4C207F00280FD0E07F28280CD152
:10016000022104F12B0000F0B7FB00202077BDE84E
:100170001040FF210248F8F73FB810BDA04400200E
:100180009C38002010B5094C207F00280DD0E07F5E
:100190002E280AD106480088401E81B2054800F08A
:1001A00021F9002084F82100207710BDA044002010
:1001B000760B00209D38002010B50A4C207F0028C7
:1001C0000FD0E07F31280CD1032104F12B0000F087
:1001D000F3FB00202077BDE81040FF210248F8F72C
:1001E0000BB810BDA04400209C38002010B5074C6F
:1001F000207F002808D0E07F3E2805D104F12B00A5
:1002000000F028F90020207710BD0000A044002055
:1002100010B50A4C207F00280FD0E07F85280CD134
:10022000012104F12B0000F0FDFB00202077BDE848
:100230001040FF210248F7F7DFBF10BDA0440020A7
:100240009C380020044A81781170C078491C1170D4
:10025000801C507070470000B60B002006480178E3
:10026000012908D141780C2903D20C3050F8210023
:100270000047002101707047B40B002002490120A3
:10028000087000F023BC0000B40B002002490020DD
:10029000087000F01BBC0000B40B00207047000089
:1002A000074801214177002180F8221000F8061F3D
:1002B000C17241878177C17780F8211070470000B3
:1002C000A044002070B52F484178012959D919213F
:1002D00001702D4C00214170B4F8420002281BD35C
:1002E00094F82B0004F12B0600F07F050B2D3DD276
:1002F000DFE805F03C060627143C143C3C3C270094
:100300002846FAF75DFC80B3B4F8420003211FE0F1
:100310001E49FCF707FA31E013212CE02846FAF7D2
:100320004FFC10B3B4F842000621FAF75BFC00283A
:10033000F2D0324629461548FBF758FD0328E7D886
:1003400011E02846FAF73CFC78B1B4F842000221EB
:10035000FAF748FC0028DFD0324629460B48FBF765
:1003600045FD0028D4D1312101E0FFE71221207999
:10037000012803D111B11920FCF7B8F90A20A4F81B
:10038000460070BD0A0C0020A04400200047002059
:10039000114810B5407801281DD9104C0321B4F83C
:1003A0004200FAF71FFC78B10D48FBF7A3FD0328C4
:1003B00003D30B49FCF7B6F90AE02079012807D1ED
:1003C00000202071312100E013212220FCF78EF95A
:1003D0001E20A4F8460010BD0A0C0020A0440020F6
:1003E0000047002070B5064617480D4640780128A2
:1003F00028D9164C2079012824D1607F00220321BE
:10040000FAF7C2FBB8B1032D01D2132114E0AD1EDF
:10041000A9B23046FEF7D2F908B101460CE00C480B
:100420006E2101703178417071788170014603202E
:10043000FCF778F903E07F212E20FCF757F92820FC
:10044000A4F8460070BD00000A0C0020A044002063
:100450000047002070B5054616484078012827D986
:10046000154C0221B4F84200FAF7BCFBC8B1297858
:1004700011F07F0F03D0207901280ED015E0084637
:10048000FAF7AAFB88B10D487E21017029784170E6
:1004900001460220FCF746F907E0002020711221F6
:1004A00000E013213E20FCF721F90A20A4F84600C1
:1004B00070BD00000A0C0020A0440020004700206E
:1004C0002DE9F04707464148417801297BD91021A1
:1004D00001703F4C002580464570B4F8420002216F
:1004E000FAF780FB002865D007F07F06012E07D0C1
:1004F000022E05D0032E03D02079012856D05DE0CE
:10050000607F4FF00109032804D001281AD0022887
:100510001FD019E0022E17D1207901284ED1FAF709
:1005200067FB68B1E07B58B16677FEF7E3FA84F8C1
:100530000C90C82084F8009084F8200078213AE0DC
:10054000222138E0022E06D0032E0CD0012E07D037
:1005500009E0032EFAD1207901282FD17E212AE04B
:10056000FCF72EFBE5736677A4F8405084F8225020
:10057000A5716574032E05D084F8245084F82550A5
:1005800084F827503846FAF727FBB8B111485021B4
:100590000170477085703221C17080F80490F42199
:1005A000417106200B49FCF7BDF807E025711221C7
:1005B00001E008E013211020FCF798F80A20A8F8C1
:1005C0000400A4F84600BDE8F08700000A0C0020F3
:1005D000A0440020004700202DE9F04107462248B2
:1005E000417801293ED911210170002545701E2155
:1005F0001E4C81800221B4F84200FAF7F3FA50B39E
:10060000387800F07F00FAF7D3FAF0B1FAF7F0FA91
:10061000C8B13878FAF7E0FA154E38B15120307089
:100620003878707031460220FCF77CF81148017967
:10063000012902D105713570757001202070C82024
:1006400084F820000BE0222106E02079012806D161
:100650002571122100E013211120FCF747F80A2030
:10066000A4F84600BDE8F0810A0C0020A044002058
:10067000004700206844002070B519494A78012AD3
:100680002CD914220A701E228A800178427809042B
:10069000807801EB0221134C0D180421B4F84200BC
:1006A000FAF7A0FA98B16FF07F40854208D1FAF7C7
:1006B000A1FA0D49542008700120FCF733F80AE034
:1006C0002079012807D100202071312100E0132179
:1006D0001420FCF70BF80A20A4F8460070BD0000B7
:1006E0000A0C0020A0440020004700202DE9F05F04
:1006F000DFF8D8A1002490469AF801000E460128A0
:1007000076D973480179012972D181460122407F4F
:100710001146FAF739FA00287ED0307800254FF0DC
:10072000010BAAF10A07012807D002283FD0B9F827
:100730004200022871D2132451E03D70A8464C4675
:10074000B9F842000221FAF74DFA0028F3D0E07818
:10075000012809D05F4D672028703078687094F8C0
:100760002200012802D004E0372438E0A0790128D3
:1007700002D0607C18B10CE0C5F8028009E0534853
:100780000938FBF71BFB84F811B0D7F80100C5F856
:10079000020087F800B084F806B067218AF80010DC
:1007A0008AF801804B490620FBF7BCFF1BE089F863
:1007B0001150B9F842000621FAF714FA0028BAD00D
:1007C00099F82810032906D8387810B1012813D0D9
:1007D00013E0032900D33624387858B11CB12146E0
:1007E0002720FBF783FF1E20AAF80400A9F8460083
:1007F000BDE8F09F2424F2E73D70364C33490422D3
:100800002560A58009392046F7F71AFD88B33078AE
:100810002E4A401EC0B201E056E053E0521F111FA5
:10082000FBF776FA20B1122447F8015FBD80D6E7C6
:10083000717888F80010B17888F80110F17888F89C
:100840000210317988F80310204940460422491FDC
:10085000F7F7F6FC002848460CD090F82810FF293E
:1008600002D2491C80F82810C9B202291BD83524AD
:10087000DAE725E080F8285067212170327862702D
:100880003278022A0DD0022280F823208AF8001044
:100890008AF8015089F822B00E490220FBF742FF86
:1008A00003E00122F0E7032903D047F8015FBD8090
:1008B00099E736240A2180F8291089F803B0B3E7B4
:1008C0002424B1E712248AE77F2488E70A0C002059
:1008D000A0440020004700202DE9F041334F064698
:1008E000682038703248417801295CD9282101708C
:1008F0001E21304C81800122607F1146FAF744F9B5
:100900000025C0B3B4F842000321FAF76BF998B39D
:10091000FAF76EF988B3307810F07F01707805D05F
:10092000032903D0207901282BD039E0012805D0F4
:10093000032803D02079012820D031E011B1032908
:1009400007D00DE0012884F8245009D084F8255000
:1009500006E00121012884F8241001D084F8251034
:100960003078FAF739F9D8B1307878700F49022029
:10097000FBF7D8FE14E00BE008E005E0257131211B
:100980000BE02571122108E0222106E0132104E08A
:100990002079012804D125717F212820FBF7A6FEAC
:1009A0000A20A4F84600BDE8F081000000470020BE
:1009B0000A0C0020A0440020F8B50646164A002084
:1009C000ADF8000050780D46012823D93120107071
:1009D000124C1E209080207901281BD10122607FBB
:1009E0001146FAF7D1F840B16B460D4A2946304618
:1009F000FDF742FF010001D104E07F213120FBF728
:100A000075FE04E00649BDF80000FBF78BFE0A20E6
:100A1000A4F84600F8BD00000A0C0020A044002005
:100A20000047002070B5054625484178012946D980
:100A3000852101701E21234C81800122607F114697
:100A4000FAF7A2F8002670B3B4F842000221FAF7D0
:100A5000C9F830B3FAF7CCF850B1287800F07F002D
:100A600001280BD0022805D02079012816D023E0D8
:100A700022211EE0012084F8270001E084F827608D
:100A80002878FAF7A9F8B8B10F48C521017029787C
:100A9000417001460220FBF745FE0DE02671122150
:100AA00007E0132105E0FFE72079012804D1267132
:100AB0007F218520FBF71AFE0A20A4F8460070BDAE
:100AC0000A0C0020A0440020004700200448002118
:100AD0000222017042700122827081807047000002
:100AE0000A0C002010B5084C207F00280BD0E07FB6
:100AF00000F00EF800202077E077BDE81040FF21DD
:100B00000248F7F779BB10BDA04400209C380020B4
:100B1000084910B5497801290BD9074C21790129D9
:100B200004D1002121711121FBF7E0FD0A20A4F876
:100B3000460010BD0A0C0020A04400202DE9F04121
:100B40001446054669B1092927D13348017800299F
:100B500023D000210170BDE8F041FF212F48F7F7B5
:100B60004BBB2F4802274178012906D0022914D116
:100B700021782C4E102923D025E0054601782078D5
:100B800001F1400282420AD12046272904D141784E
:100B9000012901D1FFF756FB6F70BDE8F0817F2876
:100BA000FBD160788142F8D1A078782804D0FFF793
:100BB0006DFB03206870F0E71E20A8800420F9E791
:100BC00047706078B0772178174B184AF17700208A
:100BD0001F5C8F4208D1342901D0362902D1144933
:100BE000098829B9507003E0401CC0B20C28EFD32B
:100BF0000C2801D10B2050700A4814212B300746D5
:100C0000F7F7FAFA1422611C3846F7F7DCFA0120EC
:100C10003077A6F84250C0E7510B00209C380020E6
:100C20000A0C0020A04400206A780108B40B0020C0
:100C30007A0B002001490120487070470A0C0020FF
:100C400070B5154C40F22551204600F023F90028DC
:100C50000ED0204600F0ACF9C2B2104881890B04D6
:100C600006D44C044FF0000306D50A2A01D0838134
:100C700070BD41F400410DE00D2A09D0C1F30D040F
:100C8000074D491C89B22A558181C729EFD870BD0B
:100C900041F48041818170BD00380140880100200D
:100CA000041B002010B5044C0146204600F084F9D6
:100CB00020880006FCD510BD0044004070B5304CC3
:100CC00040F225563146204600F0E4F82D4D88B11B
:100CD000204600F06DF9EA89C0B2FE2A04D22A4902
:100CE0008854521CEA8101E00020E8813146204608
:100CF00000F0B9F840F224463146204600F0CAF828
:100D000040B1204600F054F9012068703146204679
:100D100000F0A9F840F226652946204600F0BAF80E
:100D200018B12946204600F09EF80821204600F020
:100D3000AAF8012806D10821204600F091F82046A3
:100D400000F036F90421204600F09DF8012806D174
:100D50000421204600F084F8204600F029F9022101
:100D6000204600F090F8012808D10221204600F02A
:100D700077F82046BDE8704000F01AB970BD000059
:100D80000044004088010020CC1B002070B5314D8C
:100D900040F225563146284600F07CF82E4C98B19A
:100DA000284600F005F9C2B2608A0021C82804D2A2
:100DB0002A4B1A54401C608200E061822182A1709B
:100DC0003146284600F04FF840F224463146284686
:100DD00000F060F840B1284600F0EAF80120A07069
:100DE0003146284600F03FF840F2266631462C4650
:100DF000284600F04FF818B13146204600F033F88D
:100E00000821204600F03FF8012806D1082120469D
:100E100000F026F8204600F0CBF80421204600F030
:100E200032F8012806D10421204600F019F82046A6
:100E300000F0BEF80221204600F025F8012808D174
:100E40000221204600F00CF82046BDE8704000F07A
:100E5000AFB870BD0048004088010020CA1C0020C7
:100E6000C943018070470A0A01219140C9430180AA
:100E700070470029818902D041F4005101E021F43A
:100E80000051818170470246002012880A4200D03A
:100E90000120704730B501F01F0201240025C1F385
:100EA000421304FA02F2012B0FD0022B0FD0838AD7
:100EB0004FEA11210088134204FA01F400EA040009
:100EC00001D000B10125284630BD8389F0E7038AAF
:100ED000EEE710B5C1F3421301F01F040121A14058
:100EE000012B07D0022B07D01430002A026805D04E
:100EF0000A4304E00C30F8E71030F6E78A4302605A
:100F000010BD000030B50446008A85B00D464CF691
:100F1000FF710840E98801432182A1894EF6F31050
:100F20000140A8882A8910436A890A431043A08196
:100F3000A08A4FF6FF410840A9890143A182684673
:100F4000FDF716FA1948844201D1039800E002988F
:100F5000A189090400EBC00101EB0010296801D54B
:100F6000490000E08900B0FBF1F06422B0FBF2F12F
:100F700009010B096FF018056B4300EB8300A3898F
:100F80001D044FF0320306D503EBC000B0FBF2F0B6
:100F900000F0070005E003EB0010B0FBF2F000F0FA
:100FA0000F000843208105B030BD0000003801402B
:100FB0008088C0F308007047C1F308018180704742
:100FC00010B500F02BF9BDE81040FDF737B900F07F
:100FD0004DBA000004480088034A0449121F1288D1
:100FE00042EA0040C8607047BC6C0040900B002093
:100FF00002F0EDBE02F024BF0A484FF0E022816803
:1010000019B99169084B594381609169826843F22B
:10101000856311441A44826088B202EB820140EA7F
:1010200001407047900B00200DE37A0570470000E7
:10103000034900200978C90700D00120704700004B
:101040002C0B0020034900200978890700D50120D6
:10105000704700002C0B002001460020A1F5E06243
:10106000B43A00D1012070470FB41FB50DF1230130
:10107000069800909DF822208DF804200DF10500BF
:10108000F7F7A1F89DE80F0000F03EFA1FBC5DF8ED
:1010900014FB0FB585B000208DF808009DF81820CE
:1010A00005998DF80A2000918DF809000DF11901BC
:1010B0000DF10B00F7F787F8684602F0BBFC09B0AA
:1010C00000BD0000074810B54178002909D1012171
:1010D0004170FCF7A9F9F9F7ADFFBDE81040FAF748
:1010E0006DB810BD900B002010B52A48284CC1687F
:1010F000E2792948F7F767F82748227827A16B3863
:10110000F7F761F82448627828A15D38F7F75BF8B3
:101110002148A27828A15138F7F755F81E482279BE
:1011200028A12B38F7F74FF81B48E27828A145385B
:10113000F7F749F8184862792CA12138F7F743F8F6
:101140001548A2792CA11738F7F73DF81248A27A72
:101150002FA15F30F7F737F80F48217A0A30F7F7F9
:101160004BF80D4800216B3800F8E81F41708C21C6
:101170000171A0214171142101725021417213218A
:1011800001738821417319210174417410BD00005D
:10119000FA770108900B00203B35002032313039BE
:1011A0003134302D535A3031000000003839323696
:1011B00020202020202000004443552020202020F3
:1011C0002020000048573A312E302E430000000006
:1011D00053573A312E30302E435F32343032303470
:1011E0005F383932365F3030000000007878787828
:1011F000787878780000000078787878787878784F
:1012000078787878787878787878787878000000C6
:101210005232583030303031000000002DE9F05F9C
:10122000644CDFF894B1654920785D4640F00100D8
:101230002070DBF80400F7F768F8F7F790FADFF8AA
:1012400080A1A0729AF8100060725E48808F010A37
:10125000E1722073E868F7F782FA010A6173A073FC
:1012600059480126022700780025DFF860910728F9
:1012700066D0D9F810008047022863D0E573DFF804
:10128000508198F8030001285ED000285ED0042029
:10129000FAF78CFA00B1677498F80400012857D067
:1012A000002857D00320FAF781FA00B127744F467F
:1012B0004849D9F80000F7F728F8F7F750FA010A7B
:1012C000A174E0749AF80E00C8B3002020750120C4
:1012D000FAF76CFA217860F3041121F0E000207035
:1012E0003020FAF763FA617860F300016170312011
:1012F000FAF75CFA617860F3410161700320FAF754
:1013000055FA617860F3820161700320FAF74EFAB2
:10131000617860F3C30161700420FAF747FA6178DD
:1013200060F3041161700420FAF740FA61784646D0
:1013300060F34511617098F8010088B90EE00BE088
:10134000E6739CE7E7739AE76574A5E76674A3E71D
:101350002674ACE72574AAE70120B7E7B07810B18E
:1013600041F0400001E021F0400020F0800060707A
:10137000A570DBF80C00F7F7F2F9A0803078A071C7
:1013800078688047E0711448257200780228207838
:1013900003D240F00200207006E020F0020020702E
:1013A00002D940F0040001E000F0FB002070BDE82D
:1013B000F09F0000CC350020380C002000002041B8
:1013C00028240020C80600206023002058000020A8
:1013D0008823002000401C46900B00200848094943
:1013E00010F8EC2FCA7042780A714279037902EB47
:1013F0000322CA80427A007A02EB002008817047FB
:10140000D03400202C0B002030B5164885B0016880
:10141000001D0068814223D01249134A103900246C
:10142000086120464FEA0D0300EBC00102EB4101C9
:10143000097B092903D1411C1955641CE4B2401CE5
:10144000C0B21228F0D3074812210C3084720B303E
:101450000546F6F7D1FE224669462846F6F7B3FE62
:1014600005B030BD200B0020E43500202DE9F0410F
:10147000214C0127207820B9FFF736FEFEF710FF38
:1014800027701E4D0026287890B195F8200020B1D5
:10149000401E85F82000BDE8F08119482E700168D3
:1014A000184A01F4E06111430160BFF34F8FFEE77A
:1014B0006088401C80B26080022807D36680FEF7F7
:1014C000DDFEEF71EE7600F055F8E680A088401C56
:1014D0000004000CA08004D0A680FEF7BFFEFBF73E
:1014E000C3F8FEF793FCFAF7E7FFF9F7E7FABDE870
:1014F000F041FEF7D3BE0000A80B0020A04400205E
:101500000CED00E00400FA050FB40098A0F5E061CE
:10151000DF3907D0A0F5E061343903D080B204B0E0
:1015200000F04CB812480188322901D30021018013
:101530000288009900EB0212516002889DF80410A5
:1015400000EB0212117202889DF80D1000EB0212DE
:1015500051740188DDF8052000EB011141F8092FD5
:10156000DDF809204A600188491C018004B07047F9
:10157000444100202DE9F0410D4C00270D4E0E4D49
:1015800010E0322800D367806088307004EB0010D0
:10159000001D0FC8FCF77CFA6088401C608028683A
:1015A000401C2860218860888142EAD1BDE8F08132
:1015B00044410020A00B0020A40B00200D4910B5D1
:1015C0000978C90710D00B4900230839A1F1140488
:1015D0000A68B0F5827F08D0A0F58070113803D179
:1015E00022F002000860238110BD22F00100086093
:1015F000E38010BD2C0B00202DE9FE4F15460E4652
:101600000746FBF7DFFADFF894C2A54C002F5ED047
:10161000012F7DD19CF80800E246002878D130786F
:10162000D6F8011040EA01206061F7F701FDFBF7F1
:10163000C9FA2A469BA0616900F03CFBD4E9050188
:10164000814266D0A061A5F10D00E16981460B18C9
:10165000C3F30A02D90A99A0E36100F02BFBFAF761
:101660005BF9218CE069DFF884B2B1EBD02F0BD0AD
:10167000C10A5844C70A2184FF0239469CA000F0E1
:1016800019FB3846FAF7C6F84FEAE97109EB917091
:10169000C0F38708371DA807B0F1804F0CD09BA07E
:1016A00000F008FB70190322FF210938F6F79DFDB1
:1016B00008F1010000F0FF0879480024426A02EBBB
:1016C0000B010091C1694FF0010B416275E0357962
:1016D000257072796270D6F806004FF6FF7800BA6E
:1016E00020F0FF03707A0343636071892181307BAE
:1016F000D6F80D7040EA0720E060378A27824FF065
:10170000FF36A6610026E6616662A4F8208001E04B
:101710004AE0BEE08CF80860CDE900100297294647
:1017200080A000F0C7FA2089228AE1688DE80700CE
:10173000627821788A48636800F0BCFABDE8FE4F01
:10174000F7F7A8BC5FF0000557F824100098FAF7E7
:10175000B9F8042808D06D1CEDB2032DF4D381A094
:10176000009900F0A7FA1DE00098006801901CB1F4
:10177000A8F10100844206DBDDE9001357F82420BC
:1017800081A000F097FA57F82410019881420DD0FB
:1017900085A000F08FFADDE9001357F824207AA025
:1017A00000F088FA8AF808B0BDE8FE8F0098001DA6
:1017B0000090032D03D2641CE4B24445C2D3FBF76E
:1017C00001FA1FFA89F15546BAF82C20301DF7F7B7
:1017D000E9FC334CA885024621897CA000F06AFA16
:1017E000FBF7F0F9E1686069884250D12089AA8D41
:1017F000904204D0BDE8FE4F7DA000F05BBA002708
:1018000085A000F057FA8D4E3046FAF703F8DFF85E
:10181000308230464146FAF755F8042807D07F1C3D
:10182000FFB2032FF5D3314686A000F043FA3768A4
:1018300031463B46424654A000F03CFA47451AD197
:101840007E4F00263F1D38466168FAF73BF80428B2
:1018500007D0761CF6B2032EF5D3394682A000F0ED
:1018600029FA3E683946334689A0626800F022FAB8
:101870006068B04202D085F808B095E7FBF7A2F99E
:10188000F7F7D6FB8BA000F015FAFBF7B1FDF9F7DF
:10189000F5FFBDE8FE4FFBF795B900008801002079
:1018A000DC1A00200A0D43757272204261673A25E6
:1018B000642C206C656E2025640A0D0057726974D3
:1018C000652D616464723A20736563746F722025BC
:1018D000642C2C6F6666736574202564202C7265F9
:1018E000636C656E202530640D0A000000600208FC
:1018F0003434437572722045726173652D2D6164B5
:1019000064723A202530780D0A0000000A0D6C61DF
:1019100073742D2D2D2D2D6261672121212121210F
:10192000210A0D000D0A3636365570642D2D747956
:1019300070653A2564202C7665723A25642C5462D1
:101940007974653A25642C204372633A25642C50DF
:1019500061673A25642C506C656E3A25640D0A0067
:1019600078780108213232212121212121212121D0
:1019700057726974652D4661696C2D616464723AB1
:10198000202530780D0A00006164647220253078CB
:101990002C2C5772697465202530782C2C72656167
:1019A00064202530780D0A000A0D20726561647686
:1019B000616C20213D20557064646174615B695DD8
:1019C0002921212121210A0D000000003132325548
:1019D0007064486561642E46696C654372633D2599
:1019E00030782C544372633D2530780D0A00000096
:1019F000557064486561642E46696C654372632066
:101A0000213D205443726320212121207265747589
:101A1000726E210D0A0000002121217570642D696C
:101A20006E666F21212057726974652D746F747012
:101A30006167202564200D0A00000000005802089C
:101A40004433221155706444617461466C616721AE
:101A50002057726974652D4661696C2D61646472EA
:101A60003A202530780D0A002121217570642D69F6
:101A70006E666F21212057726974652D4661696C0D
:101A80002D616464723A202530780D0A0000000050
:101A90003161646472202530782C2C57726974652A
:101AA000202530782C2C72656164202530780D0A51
:101AB0000000000032327570642D616C6C2077720A
:101AC000697465204F4F4B4B2121726573746172AD
:101AD0007421212121212121212121210D0A000010
:101AE00030B50D46094CC1B041F20D01A4F8051006
:101AF00001462A46E01DF6F766FB658040AA694666
:101B00002046F9F71FFB41B030BD0000221F002026
:101B1000FEE7000070B50E4D0224286F816A8847E9
:101B200030B1286F816A884700B10024204670BD1B
:101B3000084805210546FCF7DDFD0028F6D02620E3
:101B4000F9F742FE2846FCF7E7FD0124EEE7000026
:101B5000C80600206434002010B50C46801AF6F741
:101B6000E3FD2146F6F703FCF6F7F9FD80B210BD60
:101B70002DE9F041194D01EB4106294601EB8604A0
:101B8000904615F8262061880027CAB199B1142023
:101B9000B1FBF0F06080F6F7D5FD4FF06632104BE8
:101BA000F6F7CAFC6FF00B02F6F7A7FDF6F7FEFD9D
:101BB000A060C8F80000678005F82670BDE8F081D5
:101BC00022790844521CD2B222716080142AF5D1C5
:101BD000012005F826002771F0E70000480C0020DE
:101BE00066660A4010B50121CC022046FCF7A2FB34
:101BF0002046BDE810400021FCF79CBB07490020AF
:101C0000086007490878401CC0B208701E2803D835
:101C100002497F200839086070470000082C004006
:101C20007401002043E0322100BF00BF00BF00BFAD
:101C300000BF00BF00BF00BF00BF00BF00BF00BFAC
:101C400000BF00BF00BF00BF00BF00BF00BF00BF9C
:101C500000BF00BF00BF00BF00BF00BF00BF00BF8C
:101C600000BF00BF00BF00BF00BF00BF00BF00BF7C
:101C700000BF00BF00BF00BF00BF00BF00BF00BF6C
:101C800000BF00BF00BF00BF00BF00BF00BF00BF5C
:101C900000BF00BF00BF00BF00BF00BF00BF00BF4C
:101CA00000BF491E11F0FF01BED1401EC0B2002886
:101CB000B9D170470FB4054B10B503A9044A029877
:101CC00000F044F910BC5DF814FB0000313F01083E
:101CD000F00400200FB4084B10B504A902AA039821
:101CE00000F034F9044602A9002000F0C6FC2046AA
:101CF00010BC5DF814FB00007B26010830B528B14C
:101D0000144C031F002021680A4605E0084630BD38
:101D10009A4203D810465268002AF9D1002800D010
:101D200041680BD00468A3EB0005A54204D11B68F1
:101D30001C440346046002E0436000E023603AB1C3
:101D40001C68D51AA54203D115682C441C60526842
:101D50005A6030BD100C00202DE9F04782460F4C30
:101D600010480D4E0E4F001B4FF0000820F00705E5
:101D70004FF0010900221146504602F0E1FD002813
:101D800002D1306810B10020BDE8F0873C60C4E9A2
:101D90000058C6F80090EDE7140C0020844700209E
:101DA000100C00208067002002E008C8121F08C144
:101DB000002AFAD170477047002001E001C1121FCC
:101DC000002AFBD1704700002DE9FF5F82B000219F
:101DD000DDE90430020DDDF840B0034318D044F6CD
:101DE0001050A2F2FF3242431514119801281FD05F
:101DF000A5EB0B00401C5FEA000A4FF000064E4FB7
:101E0000DFF83891B046504615D5CAF1000413E00A
:101E1000119801244AA3012801D16FEA0B0102980D
:101E2000119AC0E90031C0E9024206B0BDE8F09F56
:101E3000CBF10000DFE704460021404A491842EB9D
:101E40000450CDE9001012E0E00707D032463B46CF
:101E500040464946F6F770FB8046894632463B4687
:101E600010461946F6F768FB06460F466410002C2C
:101E7000EAD1DDE90401DDE90023BAF1000F06DA59
:101E8000F6F75AFB42464B46F6F756FB05E0F6F7E7
:101E9000C5FB42464B46F6F7C1FB04460E46002200
:101EA000284BF6F7B9FD03D84FF0FF30014607E0A5
:101EB0000022254B20463146F6F797FAF6F793FDB8
:101EC000102409E0002C0ADB0A220023F6F7B4FCF8
:101ED000039B30321A55641E50EA0102F2D1641C91
:101EE000039AC4F111031444119A012A03D0012268
:101EF00008430DD10AE0084304D000204FF0110B35
:101F0000119072E7A3EB0B056D1E0DE05B4504DD40
:101F10004FF0000205F1010504E003DA4FF0000282
:101F2000A5F10105002AECD002981199C0E902310F
:101F3000C0E9004579E70000000014400000F03FD0
:101F4000300000000000F0430000E03F2DE9FF4FAB
:101F500095B09B468946064600250FE2252877D195
:101F600000242746F84A0121059400E0044316F8AE
:101F7000013F203B01FA03F01042F7D130782A28C4
:101F800011D06FF02F033078A0F13002092A16D853
:101F9000059A44F0020402EB820203EB4202104471
:101FA000761C0590EFE759F8042B0592002A03DA16
:101FB000504244F40054059044F00204761C3078FA
:101FC0002E2816D116F8010F44F004042A280DD04B
:101FD0006FF02F023078A0F13003092B09D807EBFE
:101FE000870302EB4303C718761CF3E759F8047B19
:101FF000761C30786C280FD006DC4C2817D0682867
:102000000DD06A2814D104E0742810D07A280FD19A
:102010000DE044F400140AE044F4801401E044F4B8
:1020200040147278824202D104F58014761C761C2A
:10203000307866280BD013DC582877D009DC0028CC
:1020400075D04528F6D04628F4D047281AD19DE10E
:1020500018E0632835D0642879D0652812D195E13D
:10206000702873D008DC6728F1D069286FD06E28FB
:102070000DD06F2806D1B5E073282CD0752875D007
:10208000782874D05A46179990476D1C75E1C4F3AF
:102090000250022809D003280DD0D9F800100428D6
:1020A0000DD00D6009F1040967E1D9F80010EA17B5
:1020B000C1E90052F6E7D9F800100D80F2E70D7083
:1020C000F0E719F8041B8DF8001000208DF80100CE
:1020D000EA46012003E059F804AB4FF0FF306107F6
:1020E0004FF0000102D40DE008F101018846B94229
:1020F0000FDA8045F8DB1AF808100029F4D108E05F
:1021000008F1010188468142FADB1AF8081000291B
:10211000F6D105985B46A0EB080721463846179A8A
:1021200000F094FA284400EB080507E04DE029E1AF
:102130000DE01AF8010B5A4617999047B8F10108BB
:10214000F7D25B4621463846179A13E142E00A224D
:102150000092C4F302524FF0000A022A08D059F844
:1021600004CB032A4FEAEC710AD00DE029E02AE003
:1021700009F1070121F00702F2E802C1914609E0E6
:102180000FFA8CFC4FEAEC71042A03D14FFA8CFC55
:102190004FEAEC71002907DA0A460021DCF1000C55
:1021A00061EB02012D2202E0220504D52B228DF8DD
:1021B0000420012203E0E20701D02022F7E7904645
:1021C00059E00A2102E010220DE010214FF0000A30
:1021D00000910BE010224FF0000A44F0040408279D
:1021E000009203E008224FF0000A0092C4F302526A
:1021F000022A05D059F804CB0021032A08D009E0AF
:1022000009F1070121F00702F2E802C1914605E059
:102210001FFA8CFC042A01D10CF0FF0C4FF00008CF
:10222000220728D5702806D0009B83F0100353EABC
:102230000A0305D00EE040228DF80420012208E0B8
:102240005CEA010206D030228DF804208DF80500EA
:1022500002229046009B83F0080353EA0A030AD146
:102260005CEA010201D1620705D530228DF8042015
:102270004FF001087F1E582804D034A003900EA808
:1022800002900DE036A0F9E753466046009AF6F753
:10229000D3FA84460398825C0298401E0290027032
:1022A0005CEA0100F0D1029806A9081A00F1200AA0
:1022B000600702D524F4803400E00127574502DD91
:1022C000A7EB0A0000E0002000EB0A01009005984F
:1022D0004144401A0590E00306D45B462146179A14
:1022E000059800F0B3F90544002706E001A85A4616
:1022F000C05D179990476D1C7F1C4745F6DBE003D6
:102300000CD55B462146179A059800F09FF90544C5
:1023100004E030205A46179990476D1C0099481EDA
:1023200000900029F5DC08E0029802995A460078EE
:10233000491C0291179990476D1CBAF10001AAF14E
:10234000010AF1DC65E10000092801003031323377
:1023500034353637383961626364656600000000E1
:1023600030313233343536373839414243444546CB
:102370000000000000F058F90544761C3078002871
:102380007FF4ECAD19B02846BDE8F08F620700D4A9
:10239000062709F1070222F0070CFCE80223E146B8
:1023A00003F000485FEA080C02D00FF2702C0DE039
:1023B0005FEA045C02D50FF2682C07E05FEAC47C98
:1023C00002D00FF2602C01E0AFF2700C4FF0FF383A
:1023D00023F00043CDF850C065280CD006DC45281A
:1023E00009D046281DD047283DD13DE0662818D0A9
:1023F00067287ED138E00021112F01DB112000E099
:10240000781CCDE9000106A90EA8FFF7DDFCDDE987
:102410000F010E9A03910021009207F1010A049125
:102420004DE04FF000400097CDE9011006A90EA83D
:10243000FFF7CAFCDDE90F0203920E9B11990022FF
:10244000DDF80CA00093049211B9791C00EB010A8D
:10245000B7EB0A0004D4C0F1FF3007F1010A049081
:10246000AAEB0700019044E0012F00DA01270021C8
:10247000112F01DD112000E03846CDE9000106A949
:102480000EA8FFF7A1FCDDE90F010E9A03910021D0
:1024900004910092BA4621070CD40399514500DA01
:1024A0008A46BAF1010F05DD009AAAF10101515CDB
:1024B000302908D0B84202DA10F1040F06DA0121FF
:1024C000CDE9011015E0AAF10101E9E7002805DCDA
:1024D000049901440491AAEB000102E0411C51451A
:1024E00000DD8A460499401A401C01904FF00040DC
:1024F0000290200704D40198504501DBCDF80480F8
:1025000000208DF84F0002980DF14F07B0F1004FF9
:1025100025D02B200E9002984FF0020800280CDAEC
:10252000404202902D200E9007E00A210298F6F713
:102530006DF93031029007F8011DB8F10001A8F1E2
:102540000108F2DC02980028EFD1791E0E9808707D
:10255000307800F0200040F0450007F8020D12A886
:10256000C01B00F107081498007800B1012000EBAF
:102570000A01019801EBE07105984144401A401EA0
:102580000590E00306D45B462146179A059800F0B3
:102590005DF805441498007818B15A461799904789
:1025A0006D1CE00324D55B462146179A059800F080
:1025B0004DF805441CE00498002807DBDDE9030121
:1025C000884203DD0098405C179901E0179930209C
:1025D0005A469047049805F10105401C0490019863
:1025E000401E019004D12E205A46179990476D1C29
:1025F000BAF10001AAF1010ADDDC05E017F8010BD0
:102600005A46179990476D1CB8F10001A8F10108CE
:10261000F4DC5B462146179A0598ABE62D000000D6
:102620002B000000200000002DE9F04104460025A9
:102630001E461746880404D405E039462020B047DA
:102640006D1C641EF9D52846BDE8F0812DE9F041E6
:10265000044600251E469046C80301D5302700E0F9
:102660002027880404D505E041463846B0476D1C54
:10267000641EF9D52846BDE8F0810A68531C0B603A
:1026800010707047F0B40C4905244A680E68531C5A
:1026900093FBF4F504FB1535B54203D1F0BC07A05C
:1026A000FFF708BB044D0835A85493FBF4F004FB76
:1026B00010304860F0BC7047E00A00204576656E37
:1026C000742071756575652069732066756C6C0A78
:1026D00000000000F0B58DB001F0BBF82E4E0025D3
:1026E0002E4C24E09DF824300AAA03A80899F7F795
:1026F000BFFA8DF81F5001203070079803AF00908B
:1027000097E80F0000F0D4F901280ED123481422D5
:1027100003A91438F5F757FD2048CDE901561438C0
:10272000016900910FC800F079F9FAF74BFA676870
:1027300027B309AB0AAA08A90020B8470028D1D1BD
:102740001CE000BF9DF824300AAA03A80899F7F7F7
:102750008FFA8DF81F50FEF76BFC30B1079803AE6F
:10276000009096E80F0000F033F9079803AE009050
:1027700096E80F00FEF778FCFAF724FAE66936B11E
:1027800009AB0AAA08A90120B0470028DAD100F055
:10279000B9FF0DB0F0BD0000E8000020C01400201B
:1027A00070B520211B48F5F727FD1A483021303835
:1027B000F5F722FD01F046F8FAF780FAFAF7B6FAD3
:1027C000144A1549303A0020FAF768FB10B113A0FB
:1027D000FFF770FA0F4A1049183A34390120FAF716
:1027E0005DFB10B113A0FFF765FA0A4C303CE568B9
:1027F00025B100231A4619461846A847646A002CDA
:1028000007D0A4460023BDE870401A4619460120AF
:10281000604770BDF01400204001002063616E31FC
:1028200020D0ADD2E9B3F5CABCBBAFB3C9B9A60DD0
:102830000A00000063616E3220D0ADD2E9B3F5CA60
:10284000BCBBAFB3C9B9A60D0A00000000B50D4965
:10285000A1B041F20B020020A1F80520401C80B27B
:102860002828FBD3502048800749087C401C087466
:1028700006A0FFF71FFA20AA69460248F8F762FC93
:1028800021B000BD221F0020A820002053656E64E7
:102890002063656C6C2074656D70200A0D0000006B
:1028A00010B51149A2B041F20C02A1F80520002098
:1028B00001F2EA2213180C18401C93F8973080B2EA
:1028C000E3710828F6D3082048800849087C401C9A
:1028D000087407A0FFF7EEF920AA69460248F8F746
:1028E00031FC22B010BD0000221F0020A8200020D3
:1028F00073656E6420626D735F73746174655F6984
:102900006E666F0A0D00000010B51249A2B041F2C8
:102910000A02A1F80520002001F2EA2200EB4003A0
:102920000C181344401C93F8213080B2E37128281E
:10293000F4D3282048800849087C401C087407A06C
:10294000FFF7B8F920AA69460248F8F7FBFB22B066
:1029500010BD0000221F0020A820002053656E64D7
:102960002063656C6C2074656D70200A0D0000009A
:102970002DE9F05F0024134EDFF84CB0DFF84CA0D7
:10298000054640F227474FF00109A04656F834109B
:10299000286888420FD106EBC400416809B1284677
:1029A00088472868B84204D15846FBF7B5FE8AF834
:1029B0000C90C5F80080641C64B2102CE6D3BDE80E
:1029C000F09F00000C050020AC34002028240020DB
:1029D0000FB4142210B502A90D48F5F7F4FB0C4C06
:1029E0001422214601F51270F5F7EDFB802109480C
:1029F000F9F747F90848016820468847142120461E
:102A0000F5F7FAFB0020206010BC5DF814FB000015
:102A1000E80C002000100140080500200FB470B53C
:102A2000214C0A9D607814280BD200EB800004EB47
:102A30008000142204A9001DF5F7C5FB6078401C36
:102A40006070059941F6EC4218480024B2EB114F32
:102A500010D19DF81B10102904D0132902D0112980
:102A600003D005E09DF81E1001E09DF81C10817058
:102A70000A210EE041F6EB42B2EB114F0AD19DF86C
:102A80001B108278914203D114210161847001E00E
:102A900032210161054800210C30FDF7F9F82C7056
:102AA00070BC5DF814FB00009C0D00209800002015
:102AB0000FB4142270B504A92748F5F784FB264DFE
:102AC00026484FF0FF366C68C461A0B2A0F574418F
:102AD000563903D0304670BC5DF814FB41F6EC412A
:102AE000B1EB144F03D0491EB1EB144F06D11A4974
:102AF000142201F17800F5F766FBEBE718498C42E8
:102B00001AD018498C4217D017498C4214D0174953
:102B10008C4211D016498C420ED016498C420BD0F3
:102B200015498C4208D015498C4205D014498C4275
:102B300002D014498C420CD10749142201F1B4008F
:102B4000F5F741FB0449AA7A00230B31204600F037
:102B500091FB0020BFE70000D40C0020980000206B
:102B600056F4261856F4011856F4071856F40818A7
:102B700056F40A1056F4121856F41D1856F41F088D
:102B800056F41A1056F41A1810B5134C13490020B5
:102B9000C4E900010421217260720520A072FF22A5
:102BA000082104F10B00F5F720FB0D4A32F8411F14
:102BB0005088E172090AC0F57A6021736073000AD7
:102BC000A073107908B1022000E00120E073BDE895
:102BD0001040014800F00CBF600D0020F4561018A2
:102BE000C80600202DE9F04101462E4C00250422A4
:102BF0000823022604F10B0001293CD002294FD101
:102C00002949C4E9005122726572A372FF2208218A
:102C1000F5F7EBFA254F0120E07237F8330F2073F8
:102C2000000A60737888C0F57A60A073000AE073C8
:102C3000B8882074000A6074B879A074204600F047
:102C4000D7FE0320F8F70BFBE672F888000A207322
:102C5000387A0A306073B7F80900A073000AE0738D
:102C6000B7F80B002074000A6074A574BDE8F04149
:102C70000C4800F0BDBE0E49C4E9005122726572D5
:102C8000A372FF220821F5F7B0FA1020E0720D20A0
:102C900020736573A673FF20E07325740620E3E7B5
:102CA000BDE8F081600D0020F456EB1CC806002042
:102CB000F456EC1C2DE9F04101462D4C0025042270
:102CC0000823022604F10B00012938D002294CD137
:102CD0002849C4E9005122726572A372FF220821BB
:102CE000F5F783FA244F0120E07237F8460F20737E
:102CF000000A60737888A073000AE073B8882074B3
:102D0000000A607497F82600A074204600F070FE58
:102D10000320F8F7A4FA97F82600C0F16400A7F89A
:102D20000700E6722073000A6073A573E5732574CB
:102D30006574A574BDE8F0410D4800F059BE0F4917
:102D4000C4E9005122726572A372FF220821F5F7CF
:102D50004CFA1020E072092020736573A673FF20DF
:102D6000E073257411206074E3E7BDE8F081000092
:102D7000600D0020F456EB1CC8060020F456EC1C35
:102D800070B50C4C05460C490020C4E90001042133
:102D9000217260720220A072FF22082104F10B0050
:102DA000F5F723FAE572280A20732046BDE8704043
:102DB00000F01EBE600D0020F45627182DE9F04FDC
:102DC00085B0054614216846F5F716FA714C0821BE
:102DD0000026042204F10B004FF0100B4FF00709FE
:102DE0004FF00208012D7CD0022D7BD16A4B924618
:102DF000C4E9006322726672A172FF22F5F7F5F949
:102E0000664D0127E772A8782073E8786073287907
:102E1000A0736879E073E8882074000A6074287AE7
:102E2000A074204600F0E4FD0320F8F718FA84F8B7
:102E30000B802889000A2073A87A6073E87AA0734F
:102E4000287BE073687B20746674A674204600F0CB
:102E5000CFFD0320F8F703FA0320E072277384F80C
:102E60000D80A87CA073E87CE073287D2074687DC9
:102E70006074A87DA074204600F0BAFD0320F8F726
:102E8000EEF94748FF22112180F887616846F5F77F
:102E9000ACF984F80BA0E87D2073287E6073A673DC
:102EA0009DF80000E0739DF8010020749DF8020079
:102EB00060749DF80300A074204600F099FD032083
:102EC000F8F7CDF90520E0729DF8040020739DF815
:102ED000050060739DF80600A0739DF80700E0737D
:102EE00001E03FE03BE09DF8080020749DF80900F8
:102EF00060749DF80A00A074204600F079FD03205C
:102F0000F8F7ADF90620E0729DF80B0020739DF8EC
:102F10000C0060739DF80D00A0739DF80E00E07327
:102F20009DF80F0020749DF81000607484F812B0B2
:102F3000204600F05DFD0320F8F791F984F80B902E
:102F40000A2121730B21617384F80E90E020E07355
:102F5000FF2020746074A0740E4800F049FD05B095
:102F6000BDE8F08F0F4BC4E9006322726672A17254
:102F7000FF220821F5F739F984F80BB031202073CE
:102F8000667384F80E90FF20E073267484F8118035
:102F9000A674E1E7600D0020F456EB1CC806002083
:102FA00020150020F456EC1C70B50B4C05460B495F
:102FB0000020C4E900010421217260720120A07286
:102FC000FF22082104F10B00F5F70FF9E572204606
:102FD000BDE8704000F00CBD600D0020F4560910F3
:102FE00010B5134C13490020C4E9000104212172DB
:102FF00060720720A072FF22082104F10B00F5F790
:10300000F4F80D4890F86C10E17230F8661F2173E7
:10301000090A61734188A173090AE1730179217476
:10302000407960742046BDE8104000F0E1BC00002B
:10303000600D0020F4561C18C806002070B5484DDD
:1030400048490020C5E9000104212972687207205F
:10305000A872FF22082105F10B00F5F7C6F82B2016
:10306000F8F7A4FB404C18B92C20F8F79FFB28B1C7
:1030700094F85B0020F00300401C03E094F85B0030
:1030800020F0030084F85B002D20F8F78FFB18B9BF
:103090000C20F8F78BFB28B194F85B0020F00C00B3
:1030A000001D03E094F85B0020F00C0084F85B0046
:1030B0002E20F8F77BFB002894F85B0020F030000E
:1030C00000D0103084F85B000B20F8F76FFB00286D
:1030D00094F85B0020F0C00000D0403084F85B0022
:1030E0000E20F8F763FB18B91A20F8F75FFB28B138
:1030F00094F85C0020F00300401C03E094F85C00AE
:1031000020F0030084F85C0094F85900012894F83A
:103110005C0020F00C0000D1001D84F85C0094F8E5
:103120005A00012894F85C0020F0300000D11030E3
:1031300084F85C0014F84F0FE87260780A30287346
:10314000A0786873E0780A30A8732079E873207B50
:103150002874607B6874BDE87040014800F048BC8A
:10316000600D0020F4561318C806002070B53E4DBF
:103170003E490020C5E900010421297268723C4CD7
:10318000A972204694F86C1090F86100642920F030
:10319000030000D1401C84F861002F20F8F706FBE3
:1031A000002894F8610020F0C00000D0403084F87E
:1031B00061001A20F8F7FAFA18B90E20F8F7F6FAB3
:1031C00028B194F8620020F00300401C03E094F85A
:1031D000620020F0030084F862000B20F8F7E6FAA2
:1031E000002894F8630020F0030000D0401C84F80D
:1031F00063000320F8F7DAFA18B90420F8F7D6FAD2
:1032000028B194F8630020F00C00001D03E094F84E
:10321000630020F00C0084F863002E20F8F7C6FA53
:10322000002894F8640020F0030000D0401C84F8CB
:1032300064000120F8F7BAFA002894F8640020F03E
:103240000C0000D0001D84F8640014F8610FE872CF
:1032500060782873A0786873E078A873BDE8704040
:10326000014800F0C5BB0000600D0020F4561910A5
:10327000C80600202DE9F0411F4616460C460546BB
:10328000F7F78AFA574A2846A91A574D90424FD065
:1032900022DC564AA0EB0201904276D00BDC544966
:1032A000401871D05349C8426BD12078A876A86BDA
:1032B00040F0080064E05048081825D0B0F5C02F51
:1032C0005FD13A4631462046F7F748F9002858D0F2
:1032D000A86B40F0020053E0B1F5202F46D0B1F5C5
:1032E000901F52D0B1F5A81F5ED0B1F5F01F48D1A4
:1032F00021463246032E00DD03223B48F4F763FFEC
:10330000A86B40F480403BE02078E870607828713A
:10331000A0786871E078A8712079E87160792872E6
:10332000A0796872E079A872A86B40F0010027E0EC
:10333000208868826088A882B4F904004FF47A611A
:10334000884202DDA0F57A6001E0C0F57A60E8828B
:10335000B4F90600884202DDA0F57A6001E0C0F50C
:103360007A602883A86B40F0040009E03A463146B1
:103370002046F7F7C3F8002803D0A86B40F01000F0
:10338000A863BDE8F08100E01CE0207885F8230008
:10339000607805F8240FA0786870E078A8706869F4
:1033A00040F020006861ECE7207905F8340F60797F
:1033B0006870A079A870E079E870686840F0400013
:1033C0006860DEE7207885F82700607805F8280F28
:1033D000A0786870E078A870286940F080002861C3
:1033E000CFE7000056F40818FC0C002056F41A1021
:1033F000AA0BE0F7000015F8000019F870B50F4CA3
:103400008318A34201D9032070BDA2B10124002377
:103410000BE005780E78AE4204D0FF2D01D00220DB
:1034200070BD0024401C491C5B1C9342F1D3012C4D
:1034300001D0012070BD002070BD00000000020816
:10344000F8B501210820FAF781FF03248DF8024026
:1034500014250F4F8DF803504FF48066ADF80060CF
:1034600069463846F8F786FB8DF802407400ADF8DF
:1034700000408DF8035069463846F8F77BFB31462B
:103480003846F8F7FEFB21463846F8F7FAFBF8BD58
:10349000000C01402DE9F0418846054614462249BA
:1034A0002044884202D90120BDE8F081CCB3E00776
:1034B00000D0541C224641462846FFF79FFF0028B3
:1034C000F2D0012080F31088F8F726FA3520F8F7BB
:1034D0009BF9E80AC002F8F79DF9074640F2E73089
:1034E000401E80B2FCD200260FE000BF08EB460170
:1034F00018F81600497840EA01212846F8F7C6F97D
:103500000746042804D1AD1C761CB6EB540FEDD34E
:10351000F8F7B4F9002080F31088042F02D00220BD
:10352000C2E7FFE70020BFE70000020810B54FF038
:10353000000140B1054C2046F6F77AFE2046F6F72A
:1035400061FB012010BD024CF5E70000006800405F
:103550000064004030B4022814D20B4A00EB800310
:1035600002EB83021569002D0CD00A7A8B7A042AAB
:1035700006D00C6801F10B022146AC4630BC604716
:103580004C68F7E730BC70478C0F002010B538B19D
:10359000044800BFF6F7F0FE042800D1FF2010BD5C
:1035A0000148F7E7006800400064004030B402289A
:1035B00015D20C4A00EBC00302EB83040122E3683E
:1035C0008A4013420BD09343064AE36000EB80032A
:1035D000483252F82320002A01D030BC104730BCBA
:1035E00070470000440F002010B518B1F6F752F9EB
:1035F000012010BDF6F776FDFAE7000010B583282C
:1036000012D10A4C207C01280ED0A4F13000C16AEE
:1036100009B1012088470120207404480021BDE839
:1036200010401430FCF734BB10BD0000F014002033
:1036300070B500291DD10F4E0546002406EB04107D
:103640000168A94203D100210C30FCF721FB641C66
:10365000A4B2022CF2D30848817F002909D0017C52
:10366000022906D100218177BDE870401830FCF7AF
:103670000FBB70BDEC000020F0140020044B00EBE9
:10368000C00203EB820200219160FFF74FBF0000F0
:10369000440F0020022811D2094900EB800201EBFF
:1036A00082018A68002A09D0054B00EBC001483B23
:1036B00003EB8101C96801B1012110477047000087
:1036C0008C0F002010B50446022817D2FAF7E5FF48
:1036D0000B4804EB840100EB8100C16809B120466E
:1036E0008847FAF7DCFF064804EBC401483800EBD2
:1036F0008100C168002901D00021C16010BD000017
:103700008C0F00202DE9F047254F4FF0000845466B
:1037100007F1300606EB05142078012802D00228B4
:103720002DD036E0A089062803D21E4931F81010AA
:1037300000E0C621201DFCF7ABFAF8B1FAF7ADFFA7
:10374000A089401CA08105EB450007EBC000D0F824
:103750000CC0BCF1000F04D000231A4619462846BD
:10376000E047022020704FF00109FAF798FF04F1BA
:1037700008000021FCF78CFA84F80E9009E004F1AF
:1037800008006721FCF784FA18B1A4F80C8084F8CB
:1037900000806D1CEDB2022DBCD3BDE8F0870000A7
:1037A000C0140020C47201082DE9F041022802D3A0
:1037B0000020BDE8F0810C4E00EBC00706EB87044B
:1037C0000125A560002565712371E27026F8271098
:1037D0002146E560FFF708FF18B10220A060012034
:1037E000E7E7A560E4E70000440F002070B5064657
:1037F000022807D20D4806EBC60400EB8405A86832
:10380000022801D0002070BD05F110000446F6F733
:103810000FFA21463046FFF7B9FEFF28F3D0012208
:10382000E96882401143E96070BD0000440F002048
:103830000EB58DE807006946014803F0F8F80EBDA3
:103840003412002010B500F089F8BDE8104000F0F7
:1038500033B810B500F042F8BDE8104000F088B869
:1038600030B54FF0FF34E8B1124A002352F833501C
:10387000854208D102EBC300416011B9002042F833
:103880003300002030BD5B1C142BEFD351B100235B
:1038900052F8335045B102EBC3056D6825B15B1C8E
:1038A000142BF5D3204630BD42F8330002EBC300A1
:1038B0004160E6E7B40F002010B54FF426710648CA
:1038C000F4F79AFC04492823A0310C2201F5F0708A
:1038D00003F086F8002010BDB40F00203EB5104C58
:1038E00004F5207514E06946284603F085F80021A8
:1038F000009A54F83100904207D104EBC1004368AC
:1039000033B19DE80700984702E0491C1429EFD322
:10391000284603F055F80028E5D000203EBD000001
:10392000B40F002000280CD00B4A002101EB41030A
:1039300002EB83039B682BB1491C89B21429F5D390
:103940000020704701EB410302EB830188600020F7
:1039500042F82300084670474C12002010B5F021B1
:103960000248F4F749FC002010BD00004C12002072
:103970002DE9F84300216846FCF78AF9009818B34E
:10398000012821D0DFF84880002500BF05EB450164
:1039900008EB810458F82160A76896B18FB1201D0B
:1039A0003146FCF775F901280BD1A06838B1606881
:1039B0000099091AB1FBF6F101FB06006060204690
:1039C000B8476D1C142DE1D30020BDE8F88300003A
:1039D0004C120020002803D002C00021FCF758B987
:1039E0007047002803D00068002800D001207047ED
:1039F0001CB50F490C68C4B1017A002304290ED00C
:103A0000D0F80020CDE90023427A52B100230429E6
:103A100009D0016800F10B020020A0471CBD4268DC
:103A2000F0E7837AF3E74168F4E700201CBD00006B
:103A3000C01400207CB50446FDF704FB38B9207A99
:103A4000042830D0D4F80000FDF706FB68B31C480A
:103A5000856935B3207A0022042828D0D4F80010D4
:103A6000CDE90012617A21B30023042823D0216814
:103A700004F10B020120A84798B1207A04281CD039
:103A80002568104E002400BF06EB04100168A9420F
:103A900003D100210830FCF7FBF8641CA4B2022C0F
:103AA000F2D300207CBD6068CEE701207CBD616858
:103AB000D6E7A37AD9E76168DAE76568E1E700004D
:103AC000C0140020EC0000200A4810B5418D49B117
